:020000040000FA
:10000000A8FA002009880200E5E90200F58702004D
:10001000F5870200F5870200F5870200F5870200E8
:1000200000000000000000000000000071890200D4
:10003000F58702000000000005890200F587020034
:10004000E98A0200E98A0200E98A0200E98A0200DC
:10005000E98A0200E98A0200E98A0200E98A0200CC
:10006000E98A0200E98A0200E98A0200E98A0200BC
:10007000E98A0200E98A0200E98A0200E98A0200AC
:10025000E98A020085F10200E98A0200E98A0200C7
:10026000E98A0200E98A0200CFF10200E98A02006D
:10027000E98A0200E98A0200E98A0200E98A0200AA
:10028000E98A0200E98A0200E98A0200E98A02009A
:10029000E98A0200E98A0200E98A0200E98A02008A
:1002A000E98A0200E98A0200E98A0200E98A02007A
:1002B000E98A0200E98A0200E98A0200E98A02006A
:1002C000E98A0200E98A0200E98A0200E98A02005A
:1002D000E98A0200E98A0200E98A0200E98A02004A
:1002E000E98A0200E98A0200E98A0200E98A02003A
:1002F000E98A0200E98A0200E98A0200E98A02002A
:10030000E98A0200E98A0200E98A0200E98A020019
:10031000E98A0200E98A0200E98A0200E98A020009
:10032000E98A0200E98A0200E98A0200E98A0200F9
:10033000E98A0200E98A0200E98A0200E98A0200E9
:10034000E98A0200E98A0200E98A0200E98A0200D9
:10035000E98A0200E98A0200E98A0200E98A0200C9
:10036000E98A0200E98A0200E98A0200E98A0200B9
:10037000E98A0200E98A0200E98A0200E98A0200A9
:10038000E98A0200E98A0200E98A0200E98A020099
:10039000E98A0200E98A0200E98A0200E98A020089
:1003A000E98A0200E98A0200E98A0200E98A020079
:1003B000E98A0200E98A0200E98A0200E98A020069
:1003C000E98A0200E98A0200E98A0200E98A020059
:1003D000E98A0200B9F10200E98A0200E98A020012
:1003E000E98A0200E98A0200E98A0200E98A020039
:1003F000E98A0200E98A0200E98A0200E98A020029
:10040000E98A0200E98A0200E98A0200E98A020018
:10041000E98A0200E98A0200E98A0200E98A020008
:10042000E98A0200E98A0200E98A0200E98A0200F8
:10043000E98A0200E98A0200E98A0200E98A0200E8
:10044000E98A0200E98A0200E98A0200E98A0200D8
:10045000E98A0200E98A0200E98A0200E98A0200C8
:10046000E98A0200E98A0200E98A0200E98A0200B8
:10047000E98A0200E98A0200E98A0200084B1B7837
:10048000002B4FF00003836018BF0222036008BFF7
:100490000122044B4360FF23C2710372704700BF07
:1004A000580C002028010800064A074B9B78026080
:1004B0004FF41672C3710023828008220372827186
:1004C000704700BF41530200580C0020064A074BFA
:1004D000DB7802604FF43472C371002382800822FB
:1004E00003728271704700BF49500200580C00200F
:1004F000064A074B1B7902604FF4B472C371FF23A5
:100500008280082203728271704700BF814B020013
:10051000580C0020054A064B5B7902609022C3719B
:10052000FF238280082203728271704753540200B5
:10053000580C0020054A064B9B790260A822C37123
:10054000012382800822037282717047815001006A
:10055000580C0020054A064BDB7E02607822C371EE
:1005600002238280082203728271704725E901000C
:10057000580C0020064A074B1B7F02604FF408729C
:10058000C37100238280082203728271704700BF0A
:100590006FE50100580C0020064A074B5B7F0260A4
:1005A0004FF49072C371FF2382800822037282711C
:1005B000704700BF09600200580C0020044B9A7F6E
:1005C000002303608360034B4360C271704700BF28
:1005D000580C002000010800044BDA7F0023036060
:1005E0008360034B4360C271704700BF580C00200A
:1005F00000010800064A9378D278134400228260F2
:100600000260044A4260C371FF230372704700BF57
:10061000580C0020880008002DE9F341C41D002873
:10062000064624F007040CBF0020204600F080FEA0
:10063000071E04DA6FF00B0002B0BDE8F0810EB9BE
:10064000FC42F7D4364D6989288903316B7B03302E
:100650002A7B89B280B21CF0A0FA0028EADB3C4475
:10066000A978EB78002E04F10304194424F0030464
:1006700000FB01F10CBF0020204600F0FFFF2044EA
:100680000EB90028D6DB2B790446B3B1697D194435
:100690006B791944FF29CDDC0330002E2A8AC9B2B8
:1006A00020F003040CBF0020204601F057F800287A
:1006B000C0DB04440EB9002CBCDB012000F02EFE90
:1006C000C8B1A97BB9B195F82C300734002B24F0C0
:1006D000070415BF402325234FF481722822002EE2
:1006E00014BF2046002005F079F90028A2DB04445D
:1006F0000EB9002C9EDBAB7CDBB12B7993B10734B8
:10070000002EA97C24F007040CBF002020460EF028
:10071000C5FB00288EDB04445EB9002C09DA89E7AA
:10072000580C0020012000F0F9FD10B1AB7B002B2C
:10073000E5D1724B1B6893B1A97981B10334002EC6
:10074000EA7C24F003040CBF0020204698470028D0
:10075000FFF670AF044416B9002CFFF66BAF684B80
:100760001B688BB1297D79B10334002E24F003047A
:100770000CBF0020204698470028FFF65BAF0444DA
:1007800016B9002CFFF656AF5E4B1F68B7B1697DF6
:10079000A1B10334002E2B7E24F0030408BF0020F7
:1007A000009318BF2046EB7DAA7DB8470028FFF6CE
:1007B00041AF044416B9002CFFF63CAF072000F00F
:1007C000ADFD98B1A97989B10334002EAA7E24F039
:1007D00003040CBF0020204601F032F90028FFF688
:1007E00029AF044416B9002CFFF624AFB6FA86F7F9
:1007F00095F825007F09A0B10334EB7F297F24F011
:10080000070419443B4644F00404C9B2224601F0EF
:1008100059F90028FFF60EAF044416B9002CFFF674
:1008200009AF95F82610002959D00734002E2A8DDB
:1008300024F007080CBF002040461CF0C3F9041E3A
:10084000FFF6F8AE444416B9002CFFF6F3AE1EB125
:10085000298D404618F0E0FA95F82010002940D084
:1008600095F82430002B3CD06A8C0734002E24F0FD
:10087000070802F124020CBF0020404692B21CF08F
:10088000A1F9041EFFF6D6AE444416B9002CFFF6BB
:10089000D1AE0334AB7F297F24F0070495F8240000
:1008A00019443B4644F00404C9B2224601F0FCF866
:1008B0000028FFF6BFAE044416B9002CFFF6BAAE0E
:1008C0003EB16A8C404695F82010083292B218F07A
:1008D0002BFD2B6B5BB176B12C630020ACE6884618
:1008E000B5E7002EF5D0002211461046EFE7002EA6
:1008F000F3D12046A0E62834FBD59BE66400002017
:100900006C000020680000201FB572B6194B5D6BAB
:10091000E5B9BFF34F8F1849184BCA6802F4E0627B
:100920001343CB60BFF34F8F00BFFDE7B4FBF6F47A
:10093000D3B20132002CF9D103F110026A4402F85B
:100940000C4C0A2233B901A8A847E2E7044600226A
:100950000A26EDE7013BDBB203F110040DEB0406C0
:10096000B0FBF2F402FB1400303006F80C0C204609
:10097000E8E700BF580C002000ED00E00400FA0595
:1009800013B5114C6846637B8DF80130237B8DF8DD
:1009900000306389ADF804302389ADF802300AF0E5
:1009A000ABFC18B1DB210320FFF7AEFF207E0AF07D
:1009B0000FFD08B1DE21F6E7E07D0AF003FD08B186
:1009C000DF21F0E702B010BD580C002070B50546DD
:1009D000002850D01AF0AEFE18B94FF0FF34204670
:1009E00070BD19F0DFFAB0F5FA7FF6D8234C032674
:1009F00023486563002500F00DFC2A222946A01C2F
:100A000084F83850257084F82C50256327F011F9AC
:100A100040F2011301212A46A67363801B23084676
:100A200021712381638140F20323A176A3811F23D7
:100A300023824FF40273638244F60113E382F723A7
:100A40006384FB23238508F005FC20B140F24F317D
:100A50003046FFF759FF08F019FC044610B140F288
:100A60005231F5E7EFF3108572B601F07FF8002DF3
:100A7000B5D162B6B3E76FF01504B0E7580C0020AB
:100A80008109000038B51446002840F0D080694D37
:100A900095F83830032B00F0C780B9B112B96FF068
:100AA000150038BD0139162900F2C180DFE801F0D8
:100AB0000C1D20355F68863B6B6E804147555A8C14
:100AC0008F9DA0A395A6AA001378AB700020FFF716
:100AD000A3FD0028B7BF012302236FF00B0085F8A8
:100AE0003830A8BF85F83830DBE71378EB70EDE7D6
:100AF0001379002BD3D05379002BD0D01288FB2A46
:100B0000CDD81A2A6388CAD91B3BE02BC7D82368E3
:100B1000A288AB60484B9A80D8E713786A799342F1
:100B2000BDD32B71D2E713782A799342B7D86B7172
:100B3000CCE713782A799342B1D86B75C6E713785E
:100B4000002BACD05378013BDBB2F82BA7D813882D
:100B50009278EB82394B9A70B8E71078687614F087
:100B600001F9B3E71378002B99D0AB76AEE70120FB
:100B700000F0D4FB237808B1012B90D9AB73A5E723
:100B800013882B82A2E71378AB719FE7072000F050
:100B9000C5FB10B92378012B81D9072000F0BEFBDB
:100BA00018B12378002B3FF47AAF2378EB748DE7EC
:100BB0001378082B3FF673AF2B7587E71388FF2B4D
:100BC0003FF66DAFAB7481E71378EB767EE7137871
:100BD0000E2B3FF664AF2B7778E72368184A2B6219
:100BE000636853602389138170E713786B776DE72F
:100BF0001378EB776AE71378AB7767E7137885F8B4
:100C00002A3063E792786178207808F023FB002887
:100C10007FF447AF6378012B7FF658AF18F0E2F806
:100C200000287FF453AF3AE74FF0FF3039E76FF019
:100C30002C0036E7580C0020600C00206E0C0020C1
:100C4000780C0020F8B50D46064630B329B311F0F4
:100C5000070422D1124F97F83830012B02D16FF0E0
:100C60000B00F8BD032B02D14FF0FF30F9E700F085
:100C700001FA0028F8D02846FFF7CEFC0028EEDB6A
:100C800025F013FD3046396B0BF01EFEFFF778FEA2
:100C90000323204687F83830E3E76FF01500E0E7DC
:100CA000580C002010B5074C94F83830032B03D1B2
:100CB0000BF026FE0CF0D8FF1CF023F9002084F87E
:100CC000380010BD580C002050B1074B03F114023E
:100CD00053F8041B934240F8041BF9D100207047DD
:100CE0006FF01500704700BF44260300074B10B596
:100CF00093F838403CB90BF0EBFC0320044900F0BA
:100D000005FB204610BD4FF0FF30FBE7580C0020DC
:100D1000F1040000074B10B593F838403CB90BF0D4
:100D2000EBFC0220044900F0F1FA204610BD4FF020
:100D3000FF30FBE7580C0020CD04000038B50B4D08
:100D400095F8384074B90BF0F9FC0949012000F01E
:100D5000DDFA2046074900F0D9FA0123204685F83C
:100D60002C3038BD4FF0FF30FBE700BF580C00209F
:100D70007D040000A9040000054B10B593F838402D
:100D80001CB90BF0A9FB204610BD4FF0FF30FBE76C
:100D9000580C0020054B10B593F838401CB90BF0E7
:100DA0008DFB204610BD4FF0FF30FBE7580C0020B4
:100DB000054B10B593F838401CB921F00AFA2046CB
:100DC00010BD4FF0FF30FBE7580C0020054B10B56D
:100DD00093F838401CB921F0FFF9204610BD4FF0C0
:100DE000FF30FBE7580C0020054B10B593F8384056
:100DF0001CB921F0F4F9204610BD4FF0FF30FBE79D
:100E0000580C0020054B10B593F838401CB921F060
:100E1000E8F9204610BD4FF0FF30FBE7580C0020EA
:100E2000074B10B593F838403CB90BF0A3FC0420F5
:100E3000044900F06BFA204610BD4FF0FF30FBE78D
:100E4000580C0020150500000A4B10B593F83840E7
:100E50006CB90BF0A9FC0520074900F057FA074BC5
:100E6000074A20461A60074B074A1A6010BD4FF028
:100E7000FF30FBE7580C002035050000640000201F
:100E8000055801006C000020B1190000054B10B599
:100E900093F838401CB920F055FA204610BD4FF0A9
:100EA000FF30FBE7580C0020054B10B593F8384095
:100EB0001CB920F04FFA204610BD4FF0FF30FBE781
:100EC000580C0020094B10B593F838405CB90BF072
:100ED00083FC0749082000F019FA0920054900F0B1
:100EE00015FA204610BD4FF0FF30FBE7580C0020EC
:100EF00055050000750500000A4B10B593F8384001
:100F00006CB90BF087FC21F05BF90749082000F071
:100F1000FDF90920054900F0F9F9204610BD4FF010
:100F2000FF30FBE7580C0020550500007505000058
:100F3000094B10B593F838405CB90BF089FC0749B0
:100F40000A2000F0E3F90B20054900F0DFF9204604
:100F500010BD4FF0FF30FBE7580C00209905000052
:100F6000BD050000094B10B593F838405CB90BF093
:100F70008DFC07490A2000F0C9F90C20054900F052
:100F8000C5F9204610BD4FF0FF30FBE7580C00209C
:100F900099050000D9050000074B10B593F83840BB
:100FA0003CB90BF0A7FA1120044900F0AFF9204634
:100FB00010BD4FF0FF30FBE7580C0020F505000096
:100FC000074B10B593F838403CB90BF0ADFA11203F
:100FD000044900F09BF9204610BD4FF0FF30FBE7BD
:100FE000580C0020F5050000074B10B593F8384069
:100FF0003CB90BF0C9FA1120044900F087F92046EA
:1010000010BD4FF0FF30FBE7580C0020F505000045
:10101000074B10B593F838403CB90BF09FFA1120FC
:10102000044900F073F9204610BD4FF0FF30FBE794
:10103000580C0020F505000008B5064B93F8383031
:10104000032B03D008F0DEFF002008BD4FF0FF3077
:10105000FBE700BF580C002002680020014B1A601B
:10106000704700BF940C0020014B1B68184700BF5D
:10107000940C0020024B1868003818BF01207047FC
:10108000940C0020F7B504462D4E071D2C48376000
:101090000CF00AFE0228054606D1294920461AF01E
:1010A000F6FD284603B0F0BD042842D13378092B61
:1010B0000AD0262B1ED0314620461AF064FEB0F529
:1010C000817F2DD3722112E005213E201AF0B2FD5E
:1010D0000028F0D1F37801A93279684643EA022367
:1010E000ADF800301BF06BFA0028CFD05321082058
:1010F000FFF70AFC1A213E201AF09CFD0028DAD1E5
:101100007368694601A8C3F30F23ADF804301123B7
:101110008DF806301BF0BFFA0028B7D06521E6E74E
:101120000028B3D0A17820781AF084FD0028B8D127
:10113000ACE70828B5D1024920461AF0E0FDB0E737
:10114000980C0020074B4FF0FF3141F6FF72C3E9C6
:10115000001205490022C1E900221F21C3E9021241
:10116000704700BF000000209C0D00203F280CD8D5
:1011700001380B4BC0F3421200F01F0053F822302D
:1011800023FA00F000F001007047FF2806D0403835
:10119000044BC0F3421200F01F00EFE7012070473C
:1011A000000000209C0D0020074B014600684968A4
:1011B0001A4603C240F48C221A6041F0107242F4C5
:1011C000FF625A60704700BF000000200246024BD9
:1011D0000068516803C370479C0D00200246024B13
:1011E0000068516803C3704708000020FD28084BC1
:1011F00016BF00F1FF303F20C0B2420900F01F00CF
:1012000003EB82039B6823FA00F000F001007047B3
:1012100000000020014B1860704700BFA40D0020A3
:1012200010B5FFF78FFF1FF046F9034B04461B680C
:1012300003B19847204610BDA40D002070B50C885E
:10124000C27CA6B2C4F30E04931C058804F11802F4
:101250001D44825AADB21A4443882A44013AB2FB73
:10126000F5F202FB054292B29342044B8BBF33402E
:10127000B34313439BB20B8070BD00BF0080FFFFE0
:101280004A1E062A08B50346084604D84FF4D17111
:101290001520FFF739FB094A914202D940F2A31108
:1012A000F6E711B903B1196008BD2BB11B68002224
:1012B000C3E901211A1D1A600430F5E7FAFFFF7F28
:1012C00010B5114B00EB41041A786389B3FBF2F3BC
:1012D00003FB0223013A1A44B2F5706F027928BF6A
:1012E00000231A448378B2FBF3F0194403FB102067
:1012F000091AB1FBF3F003FB101313446FEA4343E5
:101300006FEA5343638110BDA80D0020024B03EB2D
:1013100080035960704700BFA80D0020034B03EB0A
:1013200080035868003818BF01207047A80D0020BE
:101330002DE9F04F10F0070A85B0054604D040F2C1
:1013400061111720FFF7E0FA544F04464FF0010BEC
:1013500007F14806B146B04657F8043B8DF80BA09C
:101360003BB101A898479DF80A30082B01D9E82124
:10137000E7E79DF80B1081BB05B13160B94506F177
:101380000406E9D12DB30023DFF814E111221E4633
:101390008EF8003058F82200013A60B190F804A0AD
:1013A0008178BAF1FF0F64D14FF000078E420771C8
:1013B0003CBFCEB20123511CECD10BB18EF80060C2
:1013C000112640F6FF6A58F82670002F63D1013EBF
:1013D000F9D2601B05B0BDE8F08F9DF80AC04A1D28
:1013E000BCF1020FE64604EB420438BF4FF0020E98
:1013F00053000EF1FF300444CEF100002040BDF850
:1014000008406444CCF1000C013C04EA0C04B4F53F
:10141000803F01D3F82194E775B1C31A3360997006
:101420001C8083F803B09DF80C201A71019A4FEAD2
:10143000124C1A81A3F806C004FB01049EE758F879
:101440002C90B9F1000F06D099F804B0D34504BF31
:1014500099F802904F440CF1FF3CBCF1000FEEDA1A
:101460003944FF29A2D90BB18EF8006040F2271150
:1014700067E794460027F0E707EB410309F101090C
:101480003846A3F80AA0FFF71BFF5FFA89F1BB7883
:101490008B42F1D89BE74FF00009F6E7AC0D002036
:1014A000A80D0020034B03EB8003D86C00B18078BB
:1014B000704700BFA80D0020F8B54FF6FF73054632
:1014C0000380184B03EB8103D86CB8B1867803799D
:1014D000B3FBF6F206FB1233DBB219460A1D00EB32
:1014E0004202B2F902705488002F09DB0131B1FBCE
:1014F000F6F206FB1211C9B28B42EFD10020F8BD03
:10150000FF29FBD0C4F30E03C4782B8024B94FF419
:10151000D5711720FFF7F8F95380BDE8F8401BF0AC
:10152000F7BA00BFA80D00201D4B03EB810370B577
:10153000DC6C054644B3030404D54FF4DC7117207A
:10154000FFF7E2F9014620461BF0C5FAFF280146E5
:1015500004D02046BDE870401BF0DABAA078B5FB95
:10156000F0F300FB1353DBB219460A1D04EB4206ED
:10157000B6F90260002E09DB0131B1FBF0F200FB8D
:101580001211C9B28B42F0D1002070BDFF29FBD0EF
:101590008B4204EB42021CBF0023E3705580D8E766
:1015A000A80D0020094B03EB8103014610B5DC6C4C
:1015B00020461BF090FAFF28014604D02046BDE8E3
:1015C00010401BF0A5BA002010BD00BFA80D0020E0
:1015D000F8B5104B074603EB81030146DC6C20464F
:1015E0001BF079FAFF28054611D0E688238953EAD3
:1015F000064606D0014620461BF08AFA01463846C8
:10160000B04720462946FFF75BFE0020F8BD0520C5
:10161000FCE700BFA80D002038B50E4B04468279C8
:1016200003EB8203D86C08B9052038BD8278E179D4
:101630009142F9D24B1CE37100EB41035D89B3F990
:101640000A30002BF3DBA5801BF062FA206000203B
:10165000EBE700BFA80D002008B5074B03EB8103A3
:101660000146D86C1BF037FAFF2804D140F21E2146
:101670001720FFF749F908BDA80D002070B50446F2
:1016800010F003000E4603D04F211820FFF73CF95D
:10169000FFF7F6FD054624B1034831460460FFF725
:1016A000EFFD284670BD00BF3C0E00202DE9F14F34
:1016B000DFF870B01E4607460D46DBF80030904656
:1016C0009DF828A09DF82C901BB961211820FFF7E8
:1016D0001BF95246092140461BF057F84A4684B28E
:1016E000092130461BF051F881B2DBF8000021449B
:1016F0001BF0C6F9386018B9286001B0BDE8F08F5A
:1017000004445346414609222C6038681AF0E9FF28
:101710004B4609223146286801B0BDE8F04F1AF067
:10172000E0BF00BF3C0E002070B50E4604461BF023
:101730003FF8054630461BF03BF8044B2A1821467B
:101740001868BDE870401BF0BFB900BF3C0E002018
:10175000014B18681BF088B93C0E00201F2AF8B511
:10176000044613460ED89200033222F00303B3F569
:10177000803F2DD2184DACB1A00710D05F210920B9
:10178000FFF7C2F8FF2B4FEA420204D9FF339A4217
:10179000A8BF1A46E8E77C2AB8BF7C22E4E7297094
:1017A0006C602B8122F0030228230127120403FB23
:1017B00001F06B680025120CEEB28E4200D3F8BD2A
:1017C00014B126181F705E60104401352833F3E70A
:1017D0004FF0FF30F3E700BF400E0020144A002115
:1017E00038B553681478C8B2844203D8AB210920B5
:1017F000FFF78AF81846013128330578002DF2D01A
:1018000000218170012412898161051D44709208B4
:10181000C16100F12001446821F8022B994245F88A
:10182000044B1444F8D100234361037038BD00BF5A
:10183000400E00200A4B1B89B3F5FF7F4FEA93004F
:1018400006D25A089B1A9BB2984238BF1846704776
:10185000B3F5EE6F01D8FF22F4E740F27263F3E7CD
:10186000400E00202DE9F8434B7880460C4602F0EC
:10187000040602F0FB07D3B1DFB12E4BD4F804907D
:101880001D89B7BB0123AD084A46211D637004F1D1
:10189000280004F12003A761E76123F8025B984266
:1018A00041F8042B2A44F8D10023636101E0002FA2
:1018B000E3D0FF23A370002E18BF0226A3191B7DBF
:1018C000032B03D1022F1CBF0136F6B2A31901224C
:1018D0001A7506F10C02002304EB860624F8123078
:1018E0007268A3704046C8F80020A8F80430BDE82C
:1018F000F883002114226170A01826F09AF9B5F53A
:10190000FF7F0FD26B08ED1AADB209EB0502C4F8E8
:1019100004902584A2606384C4F80C90A58422619D
:10192000E384C6E7B5F5EE6F4FF0FF03EBD940F265
:101930007265EAE7400E0020F7B5D2000B68400060
:10194000002502F07802CDF8013000F006008B8807
:101950000243ADF805300D4B42F001021E785F687E
:101960008DF80020EBB29E4201D800240AE0C5EBBE
:10197000C5040722694601353C44204626F030F96B
:101980000028EFD1204603B0F0BD00BF4C0E002070
:10199000014B1878704700BF4C0E0020034B00210C
:1019A0001A785868C2EBC20226F043B94C0E0020E8
:1019B00010B50C4650B1830703D020214120FEF71B
:1019C000A3FF044B58601970FFF7E8FFC4EBC40095
:1019D00010BD00BF4C0E0020F8B504460D4616465B
:1019E000FFF7AAFF034630BB144A92F800C05768BD
:1019F000DAB2944501D807201CE0C3EBC3020133DF
:101A0000B85CB918024610F00100F1D1630022F071
:101A10007F02F60003F0060306F0780643F00103A8
:101A2000334313430A4602F8013B2B68C1F80130E7
:101A3000AB889380F8BD1220FCE700BF4C0E00205D
:101A40002DE9F84305460C46F720052191461AF08A
:101A50009CFE061E22DB1DB906FB04F0BDE8F883E0
:101A600015F0030703D098211920FEF74DFFDFF88A
:101A70003480C8F81050A5B2A8F81460BBB29D42DB
:101A8000EAD9B8F814C04B46D8F810000522F7215F
:101A900007FB0C0001371AF024FEEFE74FF0FF3090
:101AA000DCE700BF540E002007B5CDE900230B464C
:101AB00003490246081D1BF0D2F903B05DF804FB90
:101AC0006C0E002013B5064CCDE900230B460246F0
:101AD00004F1080104F10C001BF0C1F902B010BDC3
:101AE0006C0E0020024B014618681BF0AAB900BF1B
:101AF0006C0E0020024BD3E900211BF0D6B900BFC9
:101B00006C0E0020034B1B28D3E9022138BF1B2099
:101B10001BF0CBB96C0E0020024B0146D3E900202C
:101B20001AF0D2BF6C0E0020024B0146D3E902200E
:101B30001AF0CABF6C0E002008B54B1E032B03D948
:101B400023219020FEF7E0FE002801F1010114BFDF
:101B50000C230523C9B203EB8101034B013121F0B2
:101B60000101197008BD00BF7C0E0020124B01223C
:101B70004FF0FF3000211B685A60C3F80803C3F818
:101B80000015C3F804250D4B1B685A6040F6FE7221
:101B9000C3F808034020C3F80015094B0949C3F8EE
:101BA0000825C1F88800BFF34F8FBFF36F8FC1F8CE
:101BB0008801C3F808257047D41D0020D01D0020DF
:101BC0000020085000E100E00A4606483A2302F8E7
:101BD000033BC368C1F803300369536043699360F2
:101BE000704700BF800E0020024B5A8C02435A847B
:101BF0005B6A1847800E0020014B00215B6A184782
:101C0000800E002010B5154C16F08EFC15F064FF08
:101C1000208DFFF7F1FF237E63B12246104904F1C6
:101C2000190052F80C3BE36063685360A36893604B
:101C300021F092FE0B4B228D93E803000DF0B8F9D2
:101C4000236B18880DF0DEF8A36B94F8341094F829
:101C500035009847002384F83C3010BD800E0020EA
:101C6000C91B0000AC0E0020034B93F83C300BB1B5
:101C7000FFF7C8BF704700BF800E002070B5224C30
:101C80000646636C256B236495F88C3094F8480005
:101C90000BB10430C0B295F86D102EB9FF2803D1F6
:101CA00095F86C308B4201D016F0DAFA95F88C304A
:101CB00023B3E06C16F01AFD94F82C30E16C003B75
:101CC000206C18BF012384F87030D5E93A23C4E9A9
:101CD000182315F01BFE46B995F86D30033B012B18
:101CE00094BF2820002016F063FD95F86C100020AA
:101CF00016F0BEFD022384F83C3070BD206C16F057
:101D0000F5FC15F0E9FEE6E7800E00200138C0B2D0
:101D1000032808B504D940F267410620FEF7F4FD18
:101D2000014B185C08BD00BF000A030008B5094B51
:101D300093F83C20022A04D040F22D212720FEF700
:101D4000E3FDDA7A42F00102DA72BDE80840FFF7FB
:101D500059BF00BF800E002010B50E4CA26F137843
:101D600003F00303032B04D1D378022B01D100200D
:101D700010BDE06F1AF0BBFD0028F9D1A36F1B78EE
:101D800003F00303032BF2D00AF0E4FF80F001001C
:101D9000C0B2EDE7800E002038B51E4C0546D4F8E1
:101DA0008030984708B9012038BD94F83430002BB2
:101DB000F9D194F82C301BB9012D03D00020F3E7A2
:101DC000002DFBD194F88430DD06C3F3001001D55B
:101DD000FFF7C2FF636CD4F888201B78C3F30013AD
:101DE0002AB9B4F88C2013B1B2FA82F35B0994F8E3
:101DF0002C10628C39B1910705D5A36FD8780238C1
:101E000018BF0120D0E7002ACDD10028D6D183F019
:101E10000100C9E7800E00202DE9F341324C06464F
:101E20000F4694F83C30256B012B5FFA83F804D001
:101E300040F29D412720FEF767FD95F87C3053B1B5
:101E40000021042085F87C10FFF7CEFE94F82C309A
:101E50000BB185F87E80A16F0B7803F00303032B91
:101E600005D195F8823013B90220FFF7BDFEA26FAD
:101E7000137803F00303032B02D053782BBB012309
:101E800085F8823095F88C30CBB194F82C30226BE9
:101E9000003B94F84880D5E93A0118BF0123C4E912
:101EA000180192F86D0084F87030FFF72FFF0022C0
:101EB00003460E4902200092424615F0BFFC36B19F
:101EC00002B0BDE8F041FFF79DBE0223D8E7002F26
:101ED000F6D03046FFF760FF0028F1D102B0BDE830
:101EE000F041FFF7CBBE00BF800E0020D00E0020D7
:101EF00037B5724C0023256B8DF8053095F88C2092
:101F000094F848300AB10433DBB295F86C1028B964
:101F1000FF2B03D195F86D308B4202D0FF2016F0D5
:101F20009FF995F88230032B00F2B680DFE803F0CA
:101F3000023B94A794F88E306148ADF80630A5F8BE
:101F40005C300AF0DDFE80B1A16F4FF48070FFF7C6
:101F50004BFE0121A36F85F87D10DB781B2B1ED172
:101F600005F1100016F0ACF919E00DF105020DF1C4
:101F70000601E06F1AF044FCA067A0B195F8C730E5
:101F80008BB99DF805302BB9038001218370A06FB8
:101F900021F0EFF9BDF80610A06F21F084FC0123B9
:101FA00084F88F3001E0474BA36795F88330A16F29
:101FB000DB0003F008020B7803F0F303134395F8FA
:101FC0008420920002F00402134323F010030B70EC
:101FD000FFF7C2FE0028A06F14BF10230023027871
:101FE0001343037095F88B30002B58D04378002BA7
:101FF00055D0E06C16F07AFB94F82C30A06FB3FA51
:1020000083F35B0984F87030D5E93823C4E91823D9
:1020100021F0C4F9021EE16C18BF0122A06F16F076
:10202000BFFD18B9A16FE06C15F070FCA06F1AF03D
:102030007AFF95F86D10012016F01AFCA26F0123AB
:10204000118884F8E030A4F8841091781E4A84F84E
:102050003C30917003B030BDB5F85C300DF1050235
:102060000DF10601E06FADF806301AF0C9FBA0676C
:10207000002894D140F2CD212720FEF745FC1048DE
:102080000AF03EFE10B940F2D721F5E7A36FDB78E6
:102090001B2B84D1012163E740F2E521ECE716F028
:1020A00025FB15F019FDA06F21F078F9011EA06F36
:1020B00018BF012124F06BFBB8E700BF800E0020A1
:1020C000F80E0020100F0020040F0020064B10B562
:1020D00093F83C2002F0FF0422B91C760CF060FF5C
:1020E000204610BD0C24FBE7800E00200A4B0B4A53
:1020F00070B506460D461A60FFF7E8FF18B1DE21FD
:102100002720FEF701FC064C012104F1900021F08C
:1021100030F96664E56470BD800000207000002026
:10212000800E0020024B012283F8E120704700BF9F
:10213000800E00202DE9FF419C4C02AE0A9F86E8EC
:10214000030094F83C1001F0FF0511B90AB103B186
:1021500027B940F26D112720FEF7D6FB96E8030061
:1021600004F12C0C84F8E15084F8345084F8E250E7
:1021700084F8355084F8E05084F88F5065842585C4
:10218000C4F880306262A7638CE80300256B16F008
:10219000B9F815F0A1FC95F9740016F017F9A86AC2
:1021A00016F088FA286A16F017F995F89C0016F0D0
:1021B00039F995F87630002B00F0AE804D2015F0FF
:1021C000C1FF94F82C00002840F0A88095F86C20FE
:1021D000774B03EB820359684FF47A7301F5FA7178
:1021E000B1FBF3F16E3116F08BF9724B724E05F5BF
:1021F0008077186816F064FA6B69E367AB69C4F816
:10220000E43005F1F0031868083353F8041C324633
:10221000BB4203C21646F6D15968D5F80001236BBC
:10222000664A03C293F8862093F86C00A2F1260157
:10223000012903D993F88710262977D194F82C2007
:10224000002A70D193F802121AF05DFE064605F1DD
:1022500034073146384621F041FC314620F04DFC30
:10226000B5F8403095F86D10834228BF03463846D4
:1022700084F88E3021F0F8FB95F86D1095F88C609D
:102280000429B5F8488008BF032120F036FC0EB9B8
:10229000043080B2404528BF40465FFA80F884F899
:1022A000E8800BF01FFE30B10BF022FE404538BF36
:1022B00040465FFA80F894F82C6084F84880002E3D
:1022C00059D195F88B308BB1012395F86C0084F8C7
:1022D0007030D5E93823C4E91823FFF717FDFB2236
:1022E000034635490420009615F0A8FA0120FFF7AF
:1022F000FFFD002323606360A360B5F88030638036
:102300002B88238095F89C3023712B6F0BB1012211
:102310001A6004B0BDE8F081962050E795F86D2072
:10232000C42101205FE793F89A128DE7213A012A30
:102330000FD824290FD094F82C20BAB193F8263165
:102340005A0711D413F001017FF47EAF03F00201AC
:102350007AE724290AD194F82C203AB193F826215F
:1023600093F865301340EBE704216DE7032814BFB1
:10237000064604266BE795F88C3093B1012395F857
:102380006D00D5E93A6784F87030C4E91867FFF743
:10239000BDFC00220346084900920220424615F087
:1023A0004DFA0120FFF76AFCA3E700BF800E002072
:1023B000000A030080000020D00E0020E80E00205C
:1023C00008B5114B93F83C201AB9BDE80840FFF757
:1023D00019BC93F82C2042B993F83C30012B12D051
:1023E00040F20B212720FEF78FFA93F83C20022AB7
:1023F00002D040F20F21F5E71B6BD3F8D801BDE8FE
:10240000084016F0A9B908BD800E0020014B1876CF
:10241000704700BF800E0020014B93F8E00070472A
:10242000800E0020044B93F88F201AB9188DC0F34A
:102430000030704701207047800E0020024B188D3D
:10244000C0F3C020704700BF800E0020014B93F8FE
:10245000E2007047800E00202DE9F34182071E4DF7
:1024600006460F462C6B22D5D5F8883023B940F2AA
:102470008E412720FEF748FAB5F88C201846296CC3
:10248000033291F8018019F011FB0DF1020201A94C
:102490002864D5F8E4001AF0DDFA01981AF0C4FABD
:1024A000012238604146D5F8E4001AF06AFAF307D1
:1024B0000ED5D4E93A32013342F10002C4E93A328E
:1024C00094F88430012B0CBF0023012384F884305E
:1024D00002B0BDE8F08100BF800E00202DE9FF476B
:1024E000B44C002380468946276BCDE9023394F82B
:1024F0003C30022B04D040F211512720FEF704FAA1
:10250000238D590606D44020FFF776FB238D43F038
:102510004003238597F88C30B8F1000F00F050810C
:10252000A3B115F0E7FA88B9236C5A7872B11B7819
:1025300097F88420C3F3C0039A4207D1012384F89B
:102540003530FFF75FFB04B0BDE8F087236C5978A6
:10255000A4F88C1009B3D4F8E4001AF0E9F9C4F82F
:102560008800238D97F8832043F400732385236C20
:102570001B78C3F380039A4200F0C280256B95F864
:102580008230002B40D0022B11D102A9E06F1AF04B
:1025900059F928B940F20541AFE7C4F88810E0E7DF
:1025A000D5E93832013342F10002C5E93832002161
:1025B00094F82C3085F882103BB195F87E3023B129
:1025C000102085F87E10FFF70FFB95F87D309BB14A
:1025D000002685F87D600AF0A5FB10B940F21C4189
:1025E0008BE731460820FFF7FFFAD5E9383201338F
:1025F00042F10002C5E9383295F88330012B0CBF57
:102600000023012385F88330238D4FF0000A43F423
:1026100000632385216C97F884200D78C5F3C003EF
:102620009A426FD00025206C1AF07DFC97F88B3011
:10263000B3B194F82C3097F86C00B3FA83F35B09CC
:1026400084F87030D7E93823C4E91823FFF75EFB1C
:1026500000220346584900920420FB2215F0EEF8B0
:10266000B9F1000F00F0CA80012616F05BF91DB128
:1026700003A90220FFF7F0FEBAF1000F10D094F882
:102680002C3043B1B4F80720B4F805301343B7F841
:102690008020134304D0B4F809300133A4F8093082
:1026A000B8F1000F00F0C480B4F805300133A4F88D
:1026B0000530002384F8E23040480CF091FB02988A
:1026C00030B11AF0B1F9216B002202720BF036FB27
:1026D000039B33B1216B00221A720C2203980BF07A
:1026E000FBFA002E7FF42DAF238D1B063FF52BAF99
:1026F0008020FFF781FA238D43F08003238522E7B2
:10270000C24687E705F00305266B032D14D0F5B903
:1027100096F88430013B18BF012386F88430236C7F
:102720005B78002B3FF47FAFD6E93A32013342F1B8
:102730000002C6E93A3276E7238D0120002543F4F2
:10274000805386F87C002385FFF74EFAE0E74D784A
:10275000002DDDD0238D96F88C5043F480532385D3
:1027600015F006FD042894F8E83006D1002D14BFBA
:102770001B221F22934228BF1346226C52789A4292
:102780000BD8D4F88830002B3FF44CAF94F8E130EC
:102790006BB12020FFF730FA44E794F83430012081
:1027A00043F0100384F8343017F09CFC3AE74546B8
:1027B000AEE700BF800E0020D00E0020AC0E00203F
:1027C0000BB115F0ABF994F8E230013384F8E23044
:1027D000238D43F48063238597F86D30033B012BF1
:1027E00005D80025012017F07DFCAA461EE70BF056
:1027F00079FB82460028F4D1054617E794F82C208F
:1028000094F8E2303AB1628C120704D5A26FD27804
:10281000022A3FF429AF012B3FF626AF0120FFF734
:10282000BBFA064600287FF41FAFFFF761FB1EE7E7
:10283000B4F807300133A4F807303DE72DE9F04F35
:1028400004468BB01E4600230D461746069390F8AB
:102850006D801FF007FE94F8C0310B2B04D940F2B5
:10286000F2310620FEF750F8794A32F813B094F8A6
:1028700087308344442B1FFA8BFB3CD00E2B94F8FB
:10288000862038D0443A53425341039387F00103E2
:102890000493002F57D194F80432032B53D1039B98
:1028A000002B50D0B4F89832AB424CD1D4F80C3253
:1028B0002046B4F8DC2141F64B59C4F8F831E369FD
:1028C000C4F8FC31B4F852321344C4F800320FF0AB
:1028D000FFFCD4F8A03294F8AC224B458CBF4FF0EB
:1028E00000094FF0010942B9E26993421AD02088E9
:1028F00023F0B7FE16E00123C7E7208823F0AEFEE1
:1029000018B940F232713020ACE7B4F8A832B946B9
:102910006386B4F8AA328381B4F89832C7814381C0
:10292000013B0382D4F89C3284F87690E362B4F8D9
:102930009A322386D4F8A032E361D4F8A4326362D9
:10294000022384F80432B4F850A204F50873B4F8F2
:102950008090A5EB0A0A0593A5EB09090FFA8AF303
:102960000FFA89F9002B17DAD4E98E23C4E99223F0
:102970000023012284F81B324B4694F804A2354F01
:102980005FFA8AFABAF1030F00F2C881DFE81AF0A1
:1029900006002601640045013246EEE794F86D100A
:1029A00094F8D60120F0D0F88046E06A59464044B9
:1029B00017F0AEFA5946C4F80802E06917F0A8FA11
:1029C00094F8763007A9002B18BF4FF0020A504444
:1029D000C4F80C0208A815F0ADFF079BD4E99201DA
:1029E0000093DDE9082324F054FF814620461AF0C5
:1029F000BFFAD4F8543294F86D00D4F82CA00693A2
:102A000016F0C6F8069B00F52240D4F80812BB3B2E
:102A1000B1309A444FF47A73AAEB010A3031B0FB1B
:102A2000F3F0D044238EA8EB090803EB4101A8EB97
:102A30000000069094F86D001AF0A6FAD4F854221B
:102A4000069B38609B1ACC2B69D840F2D2415AE7DA
:102A5000180A03006C0F0020E36A5946D4F8FC0101
:102A6000184417F055FA5946C4F80802E06917F0FF
:102A70004FFA94F87630002B08BF4FF0000A50440C
:102A8000C4F80C0220461AF073FAB4F8DC31D4F81A
:102A90002C80D4F8FCA1002B40F09980002E00F08F
:102AA0009680D04494F86D0016F072F8D4F808328D
:102AB000A8F1BB0800F5224994F86D004FF47A7B29
:102AC000A8EB0308D4F8403209F1B1099844C31EB9
:102AD000D4E98E12012BA8EB0108B9FBFBF973D9DD
:102AE00016F056F800F2E730B0FBFBFBA8EB090844
:102AF00008EB0B000690D4F80812D4F8F831D4F89B
:102B00000022303194F86D0002FB0311238E03EB99
:102B100041011AF039FA0123386084F80432E3697C
:102B20004FF00008D4F80C2204F13400A3F5A2738E
:102B30003F6806999B1A84F820829F4228BF1F464F
:102B4000D4E99232C4F8D8715B1842F10002C4E9AA
:102B50008C3220F087FF0744A4F85052C4F8247246
:102B6000D4E98C23C4E992230EF0E4FD20B1D4F81B
:102B700024321E33C4F82432B4F8C81184F82882F1
:102B80004D1B2DB2002DC4BF022384F82832039BB5
:102B9000002B40F0C680002E40F0C48094F8043230
:102BA000002B00F0DC80E16904F50870D4F80C32E9
:102BB000C91A1FF071FF80B2002800F0D080149B6A
:102BC00003B118800120DAE04FF03E0B8EE7D044CD
:102BD000D4F80832A8EB030306938CE7D4F80C2250
:102BE000E169D4F8F801891A4B43D4F8001206932E
:102BF000B4F8DC319944CB439944D4F808323033EB
:102C000000FB0133218E94F86D0002FB093301EBC8
:102C100043011AF0B9F9386081E7E069584306903A
:102C20005EB3B4F8DC1141BB84F81B12D4F80C126B
:102C300001FB130A94F88630262BCDF818A003D098
:102C400094F88730262B09D1B4F89832EB1A1B047C
:102C500004D494F89B32002B18BF9846002A3AD02F
:102C6000B4F8DC31BBBBD4E98E23D4E990018242B5
:102C70008B4108D340F2265145E694F81B120029F7
:102C80007FF44DAFD2E794F86D00C31E012B40D9FD
:102C900015F07EFF00F522404FF47A7BB130B0FB97
:102CA000FBF000F1AB0BD4F8403294F86D00103B10
:102CB000D4E98E125A1AC31E012B92442CD915F056
:102CC00067FF4FF47A7300F2E730B0FBF3F0AAEB42
:102CD0000B0A50440690B4F8DC1140468944D4F8FD
:102CE0000C1201FB09F909F130094FEA490949467B
:102CF0001AF04AF9234A94F876301060002B3FF41A
:102D00000EAF06AB4946E0691FF03BFF84F81B029B
:102D100005E74FF4897BC6E73E20D8E740F23E51F5
:102D2000F1E5E6B1B4F8F01119B3B4F8F22194F872
:102D3000F431501CA4F8F22102FB033399420EDD5A
:102D400094F828325BB10023A4F8F20184F8283209
:102D50000BF0D4F800F00700013084F8F40104F51A
:102D6000087194F81C0218F053F820B940F287510A
:102D7000C9E50A46DBE7049B84F8183200200BB053
:102D8000BDE8F08F6C0F0020F0B5044685B018B98F
:102D9000A8213020FDF7B8FD072900F20681DFE801
:102DA00011F008004500450040000401F000F80063
:102DB000020190F8183253B3B0F81632B0F8802000
:102DC00093421ED1B0F8CC21D31AA0F88020A0F8ED
:102DD000CE312046D4E98C23C4E98E230FF098F934
:102DE00094F8D331002B00F0CA8022F052F9704BD6
:102DF0001B68002B00F0C380204605B0BDE8F04002
:102E000018479A1AA0F8CE21A4F88030E1E7B0F86C
:102E10001432B0F880209B1AA0F8CE31B0F81432EA
:102E2000F2E705B0BDE8F04015F090BD24F0C1FC1C
:102E3000D4E98E23801A61EB0301012871F10003AC
:102E400002DA40F21261A4E76FF0010383424FF00F
:102E500000038B4102DA40F213619AE7E5690DB194
:102E6000B0FBF5F594F88730442B14D094F8862005
:102E7000442A0AD00E2B08D0A2F1430672427241B6
:102E8000B4F81612B4F880303AB1B4F816320133FF
:102E9000A4F8163214E00122F2E72B449BB2CA1ABE
:102EA000150454BF4B1C01339BB2A4F8163294F89E
:102EB00019322BB9B4F81622B4F8CC319342E6D0CB
:102EC000B4F8523202AEB4F880500133394FA4F84E
:102ED0005232B4F8BA301D44B4F8B830013DED1A9E
:102EE000ADB23B685BB1B4F816120022204601393E
:102EF00089B29847B4F816321844A4F81602B4F808
:102F000016126B1A18041ED40023204600961A4687
:102F1000FFF794FC98B3012812D1B4F81622B4F844
:102F2000C811BDF808301344521A12049BB204D5DC
:102F3000EA1A12F4004F18BF0B46A4F81632D0E775
:102F400040F26A6125E794F88A3030460394002BFA
:102F50000CBF3E23082384F8A93001238DF80830E4
:102F60000BF0AAFC204622F096F8002394F81C02ED
:102F700084F8043217F0D2FE202384F81C3205B006
:102F8000F0BD012017F0AEF805B0BDE8F04019F033
:102F9000DABF90F80432042B01D0CE21F9E60023E9
:102FA00080F80432EBE7D421F3E6D821F1E600BF44
:102FB00088000020900000202DE9F04104460E46D4
:102FC000154690F8383103F0FF071BB10C2738463F
:102FD000BDE8F08101464C4817F07AFE2028804673
:102FE000F4D05822394604F5887024F022FE84F883
:102FF0001081C4F81461FF2384F8383136B10AF027
:1030000095FF00F00700013086F8F40102234FF02D
:103010000008A4F8483184F8408116F0CDFF00F193
:103020004906204621F046FE0146B6B2D8B31FF04D
:1030300019FA00F5CD61284689B216F069FF2844D7
:10304000C4F8440124F0B5FB30184FF00106A4F891
:10305000268041F1000184F81861C4E9540120463A
:1030600021F03EFED0B1A5F2AA453146204621F01E
:1030700091FD2D1AC4F81C514FF0FF326FF0004340
:10308000C4E9562304F5A07194F8100117F0C0FEAE
:1030900070BB4FF4E5713020FDF736FC3046AE3D95
:1030A00021F017FFE5E72046DFF8608021F072FD90
:1030B000AE30C4F84401B8F8040048B1E08C38B12F
:1030C0000AF034FFB8F80430B0FBF3F202FB13004F
:1030D000064424F06EFB361841F10001C4E9546146
:1030E000002DC9D0AE1941F10001C4E95661C9E70C
:1030F000D4E9542300212046C4E94A23C4E94C23DF
:1031000021F017FE63E700BF57D001006C0F0020CD
:10311000F0B5002385B0CDE9003303238DF80630E8
:103120006846FEF779FA88B11D4E01230027B37176
:103130000223CDE902778DF80E3002A8FEF76CFA73
:103140000546A8B10023B37105B0F0BD00981AF090
:1031500069F8E5E790F81C0218F06AF994F81C0287
:1031600084F8045217F0DAFD202384F81C32DFE7DC
:10317000029B002BE1D093F81C22202ADDD0188876
:103180004FF6FF739842DDD00221FEF70BFA04469A
:103190000028DFD14FF49A713020FDF7B5FB00BF56
:1031A0006C0F0020044B0022DA719A7142F2107207
:1031B0009A80FFF7ADBF00BF6C0F0020014BD871A4
:1031C000704700BF6C0F002008B514F0F3FF044BEC
:1031D0009A6882422ABF9879002080F0010008BDD9
:1031E0006C0F0020F0B5044685B090F8D33103F0A1
:1031F000FF05002B6ED190F80432032B6AD124F026
:10320000D8FAD4E98E23801A61EB0301012871F109
:1032100000035FDB6FF00103834275EB010304DA07
:1032200040F2BB513020FDF76FFBE269B4F880300B
:103230000AB1B0FBF2F2013313449BB2A4F814328A
:10324000B4F8CC31B4F814229B1A1BB2002B41DD28
:1032500094F81C0217F0E0FE00283BD0FF2384F80E
:103260001932B4F8BA300DF10E07B4F880501A4E86
:103270001D44B4F8B830013DED1AADB2336863B106
:10328000B4F8141200222046013989B29847B4F8E4
:103290001432184480B2A4F81402B4F81432EB1AB1
:1032A0001B0417D4B4F8141200230122204689B25B
:1032B0000097FFF7C3FA68B1012808D1B4F81432B7
:1032C000BDF80E2013449BB2A4F81432D6E740F2A6
:1032D0000261A7E705B0F0BD900000202DE9B343DF
:1032E0000446062900F28380DFE801F00428152552
:1032F0002C317C003F4B9B7903F0FF025BB90092BD
:103300000123B0F8CC11FFF799FA38B14FF4DA6124
:103310003020FDF7F9FA042384F8043215F060F93F
:1033200017F0D0FB0023B4F88020A4F85232A4F8A0
:10333000162284F8193202B0BDE8B083032380F866
:103340000432F8E723F0E6F9C4E99001F3E72A4BE9
:103350001B681BB10246D0E99001984794F86D3084
:10336000E569033BDFF88C90012BD4F80C3294BF55
:103370004FF028084FF000089D4208F5807888BF7C
:10338000ED1A99F8073098BF00251BB9636B9D4271
:1033900028BF1D46D4F8D87104F1340020F062FB38
:1033A0000744022017F096FF0221ED1B25EAE57580
:1033B000854228BF0546284617F0D2FF00B92F44A2
:1033C00042463946204620F0DBFBD4F8D831C9F814
:1033D0000800E069184417F04FFF0028ABD140F215
:1033E0007E3195E702B0BDE8B04319F0C1BD40F2AF
:1033F00084718DE76C0F002084000020012A70B5D5
:1034000005460C46164615D0022A18D042BB14F0C9
:10341000D1FE32460146204619F0D4FE2A46124912
:1034200094F8100116F04EFE40B940F2977130202A
:10343000FDF76AFA14F0BEFEC5F8540270BDD0F86C
:1034400054120122204619F0BDFE2A46064994F87E
:10345000100116F037FE0028F0D14FF4F561E6E7D1
:1034600040F2AE71E3E700BF892D0000014B988068
:10347000704700BF6C0F00200D4B0321186830B55A
:103480000D4690F8A52090F84B400132B2FBF5F3C1
:1034900003EB4303D31ADAB244FA03F3DB0703D492
:1034A000013911F0FF01F0D180F8A52030BD00BF37
:1034B000780F0020014B18681AF00EB8780F002022
:1034C00008B50AF065F9014B187008BD100000201E
:1034D000054B10B41C68827C836804F1420194F8A7
:1034E000410010BC1FF04EBA780F00202DE9F041CA
:1034F000064690461D460C46D9B91A4F386800F169
:103500005B0390F85A2000F1780190F87E001FF0DC
:1035100039FA7A680346507908280ED03A6892F84A
:103520004E100A1A504250413A6892F85620012A29
:1035300005D1B36863B9012006E02046F4E77AB903
:10354000002BF6D10028F4D100F00100BDE8F08195
:10355000B8F1000FEFD11DB13046FFF7B9FFF3E727
:103560000020F1E7780F0020024B18686C3002F061
:103570009DBA00BF780F002038B50F4CFFF7F4FF5D
:10358000656802F04DFA63682860186820B940F257
:10359000F7413220FDF7B8F91AF0F1F910B940F20D
:1035A000F941F6E715F0A2F8002015F001F963687B
:1035B00004221A7138BD00BF780F002038B5194DAC
:1035C00004466B681B79022B04D940F6EA013220CD
:1035D000FDF79AF92B68027C83F8A4201A44C1688D
:1035E000996692F8242183F820214268C3F8882044
:1035F000037A022B0ED014F085FE15F01FF914F09B
:1036000089F8094815F05CF8084815F053F808489F
:1036100014F0E2FE637C23B12B685B6E0BB10122D8
:103620001A6038BD780F0020440100205555550020
:10363000D6BE898E08B5FFF743FF034B586802F0EA
:1036400081FA012008BD00BF780F002038B505467B
:103650000C4609F0A1F9420704D4A37803F0E00373
:10366000402B30D009F098F9830704D4A37803F0F5
:10367000E003202B27D0237803F03F03242B22D80C
:1036800014F07CFD94F90030A278002B637802F0EE
:103690001F02ACBF1E214FF4967143EA02234B4335
:1036A0001A1AB2F5877F0ED398420CD8074B2946D9
:1036B00018682388A0F82131A37880F82331BDE869
:1036C00038401AF073BC002038BD00BF780F0020CE
:1036D000F0B5044687B0084663785A0671D422785C
:1036E00003F01F0352EA03236BD06188052968D9D0
:1036F000237A6268C3F30403134362D0324B1B681E
:103700004BB140B1984700285BD0304B01221B6879
:10371000D3F890305A762D4E227A3368C2F30402E1
:10372000D3F89050636805F11E008DF81420190A33
:103730008DF810308DF81110190C1B0E8DF8121029
:1037400004A98DF813301FF06AFA638840F2E24250
:103750005343A27BAB67D4F809302B60637B43EA09
:103760000223E27B43EA02436B60238A013BA5F814
:103770006230237AC3F3421385F89230336893F8AA
:103780002031EB756378257813F0200F03F01F03C9
:1037900014BF4FF496771E2745EA032307FB03F572
:1037A00022F0B8FF33680246D3F89060238A06F10E
:1037B0005000009506339BB2CDE901730B4611F022
:1037C000C1F907B0F0BD00BF24010020780F002030
:1037D00008B5074B93F900207F2A04D140F29D31B0
:1037E0003220FDF791F802707F221A7008BD00BFE9
:1037F0001000002010B504788EB004F00F0404A966
:1038000022461AF0FBF8FFF75BFE042C33D11B4C69
:10381000059A2368107893F8781088422BD1507855
:1038200093F87910884226D1907893F87A108842DC
:1038300021D1D07893F87B1088421CD1107993F86D
:103840007C10884217D1517993F87D20914212D192
:103850009DF8212093F87E309A420CD10DF10F0093
:10386000FFF7B6FF9DF90F3004A90093237B227A5E
:1038700060681AF096F803200EB010BD780F002093
:103880002DE9F04F044689B0062900F2C780DFE831
:1038900011F06200E9000700C500C500C50028005E
:1038A0006F4D14F041FE2F6897F854309E0701D1F8
:1038B000032036E06E68B379002BF9D00DF11F00BC
:1038C000FFF786FF9DF91F30022221460293304602
:1038D0002B7A0193FF23009307F142031AF051F86A
:1038E000E6E75F4D6E68B379002B00F097802F6894
:1038F00097F85420900717D50DF11F00FFF768FFC8
:103900009DF91F3030460622029321462B7A0193FF
:10391000FF23009307F142031AF033F80023092034
:103920002B7309B0BDE8F08FD10777D5530701D5C8
:1039300014F0FAFD0DF11F00FFF74AFF9DF91F205B
:103940002B6802922A7A42330192FF2200920622C9
:1039500021466868C2E7424D2B6893F85420570708
:1039600037D56968CA79002A33D0426893F85B007A
:103970001678864255D1567893F85C00864250D12D
:10398000967893F85D0086424BD1D67893F85E0026
:10399000864246D1167993F85F00864241D150792C
:1039A00093F8602090423CD1627C93F85A00161A3A
:1039B0007242724193F8560001284ED0002A4CD131
:1039C00093F84E30082B02D04A799A4245D014F031
:1039D000ABFD6E68B379002B3DD02F6897F854206B
:1039E000900720D50DF11F00FFF7F2FE9DF91F3063
:1039F00030460022029321462B7A0193FF23009345
:103A000007F1420319F0BDFF012309202B736B68F6
:103A1000DA79002A85D19B79002B82D114F084FDBC
:103A200046E70022C6E7D10715D5520701D514F0A5
:103A30007BFD0DF11F00FFF7CBFE9DF91F202B68CA
:103A4000214602922A7A423368680192FF2200924C
:103A5000002219F096FF0320D9E70A20D7E700BF1C
:103A6000780F0020644D81686E682A68B379807C85
:103A70000493F37992F84880059319F05CFC92F86E
:103A8000543088F0010807465B0740F1898092F8BE
:103A90004D30002B00F0848092F84E60082E00F02C
:103AA0008180304609F0F2FA002818BF8046002FC6
:103AB0007AD03046A16809F0F3FC06462B6893F8EB
:103AC00041900EB149F0020993F85420500746D5B1
:103AD000626893F85B101078884267D1507893F849
:103AE0005C10884262D1907893F85D1088425DD175
:103AF000D07893F85E10884258D1107993F85F100F
:103B0000884253D1517993F8602091424ED1617C23
:103B100093F85A20891AD1F1000B4BEB010B69681D
:103B20004979082945D093F84E305A1AD2F1000A43
:103B30004AEB020A002E3FD1B8F1000F3ED02046DA
:103B4000FFF7C6FC059B43B1296891F8561001297F
:103B50004DD011B95BEA0A0349D114F0E5FC2B689A
:103B600093F854309B073FF4A3AE14F0DDFC049BA4
:103B7000002B3FF49DAE2046FFF7AAFC10B9D5F804
:103B80000080EEB10DF11F00FFF722FE9DF91F200E
:103B90002B68029242332A7ACDE900920122D7E6BD
:103BA00076797BE7002689E73E4687E74FF0000BF2
:103BB000B5E74FF0000ABDE70120C3E73046C1E793
:103BC00098F85520023A012A3FF672AE002F3FF4D2
:103BD0006FAE0DF11F00FFF7FBFD9DF91F30029343
:103BE0002B7A0193FE23009308F14203D6E70028C5
:103BF000B3D00A2095E600BF780F00202DE9F043EE
:103C000087B0174C06460F460DF11700FFF7E0FD91
:103C100065682B79032B20D02B79062B0CBF4FF036
:103C200003094FF00109236803F1420814F0A0FAD8
:103C30009DF917303A463146CDF80C900293237A1D
:103C4000CDE900034346284601F0B0FF10B160689B
:103C500001F048FF07B0BDE8F0834FF00009E2E74C
:103C6000780F00202DE9F043324E87B005460F460D
:103C70007468A37923B90024204607B0BDE8F08317
:103C8000D6F8008098F8953033B90378002B0CBF34
:103C90000123022388F895302379062BDAB224D049
:103CA000072A14BF4FF001094FF002090DF1170068
:103CB000FFF78EFD14F05CFA9DF917303A4629465D
:103CC0000293337ACDF80C90CDE9000308F142035A
:103CD000204601F06BFF0028CDD06C7814F0100462
:103CE00006D1706801F0FEFEC6E74FF00309DDE77C
:103CF000A9690220FFF7AAFC0446B8B10022336884
:103D000083F896206A696AB15178C1F3031183F888
:103D100097101178527802F00F0241EA0222A3F8BC
:103D20009820A9E7FF2283F89720A5E7706801F0A3
:103D300009FFA1E7780F00200D4A536810B51979E3
:103D4000022904D841F293413220FCF7DDFD1979B4
:103D5000082902D941F29441F6E71B79126903F16F
:103D600080439268033BBDE8104052F82330184767
:103D7000780F002010B5054C637A2BB114F05EFD6E
:103D800013F0C8FC0023637210BD00BF780F002041
:103D900010B5054C23792BB114F050FD13F0BAFC8B
:103DA0000023237110BD00BFA016002010B5094CE0
:103DB000FFF7E0FF012263681A7100232268A2F86E
:103DC000213182F82331FFF7CFFB2068BDE8104096
:103DD0001AF0B8BA780F002008B5044B586801F003
:103DE000B1FEBDE8084019F084BB00BF780F002089
:103DF000062938B51C469DF8105019D908291DD838
:103E000002B1DDB143689BB912B94378DB0617D420
:103E10000C4B5B68186819F0D3FD00B135B92CB9AB
:103E200009F056F900F00104204638BD0120F9E7F9
:103E30009DF81430002C08BF1C46F5E70024F3E77A
:103E40000124F1E7780F002038B50D1E044614BF99
:103E500003200520104409F051FA094B587270B143
:103E60005DB9033C012C94BF5524502413F02AFC67
:103E70002046BDE8384014F0D5BC4024F6E738BDF4
:103E8000780F0020F8B53D4CFFF76EFB656801F038
:103E9000C7FD63682860186820B940F25441322099
:103EA000FCF732FD19F06BFD054610B940F25641A2
:103EB000F5E7236893F8A6306BB123681A6D93F881
:103EC000A710C3F8102193F854200A4383F8542014
:103ED000002283F8A620206890F8A430034493F8C9
:103EE0002471636880F820711A7952B11B79012B13
:103EF00007D000211AF05AF818B9BDE8F840FFF7CA
:103F000055BF23681E4A93F8A530D05C14F08AFA96
:103F1000236893F8A420134493F82461022E2BD035
:103F200004D8012E05D040F2FE71B8E7F31E012B34
:103F3000F9D801F06FFD314614F092F9284614F0DB
:103F4000D5FB3146012014F073FA7B1E2A46384611
:103F500059425941FFF778FF6268082100235171E7
:103F600021722168D3801372E37281F89530A372B5
:103F7000237303231371F8BD0D20DCE7780F0020B5
:103F8000300A030010B50A4C052120681AF00EF81B
:103F900018B9BDE81040FFF709BF2368012093F866
:103FA000201114F065FC63680B221A7110BD00BF6C
:103FB000780F0020124A10B5536800B931B918467D
:103FC00001F0C0FDBDE81040FFF7F0BE19790829E7
:103FD00004D841F263413220FCF796FC19790C2990
:103FE00002D941F26441F6E71B79126903F180437B
:103FF0005268093BBDE8104052F82330184700BF13
:10400000780F0020054B1A6892F85420920703D0CD
:104010005B68186801F02EBD58697047780F002062
:1040200070B5304D06466B681A79032A02D01A79AA
:10403000042A09D1186819F0A2FC044638B941F2E3
:104040009B313220FCF760FCFFF7DCFFF5E72B68C3
:1040500093F8543013B941F2A131F2E776B11FF071
:1040600051F930B16B681A79022A0ED841F2213128
:10407000E7E720461FF061F90028F3D16B681A7951
:10408000022A17D841F28131DBE71A79082A02D9CE
:1040900041F22231D5E71B7920462A6903F180439A
:1040A0001269033B52F8233098470C2812D941F289
:1040B000B431C6E71A79082A02D941F28231C0E741
:1040C0001B792A6903F180435269033B52F823307C
:1040D0009847EAE72B69DB68BDE8704053F8203069
:1040E000184700BF780F002038B5FFF78BFF044654
:1040F00020B940F21E513220FCF706FC0B4DFF2088
:104100002B6893F8201114F0ABF8204614F0EEFA67
:104110002B6893F82031033B012B94BF282000200B
:1041200014F046FB6B6807221A7138BD780F002027
:1041300038B5134C0E20236893F8201114F090F832
:10414000FFF760FF054620B940F20B513220FCF723
:10415000DBFB14F0CBFA236893F82031033B012BEF
:1041600094BF2820002014F023FB23682A46002156
:1041700093F82001FFF768FE636808221A7138BDC2
:10418000780F002010B5074C606801F0ABFCFFF71A
:1041900097F920680021A0301EF033F9BDE81040E7
:1041A000FFF704BE780F002010B504468AB0FFF771
:1041B00087F9237803F00F03072B23D169462046A4
:1041C00019F0AFFC684619F052FD9DF80030CBB9EC
:1041D0009DF80130DB0715D50D4C019922689DF83B
:1041E000110002F1780392F87E201EF0CBFB48B15B
:1041F00020680121A0301EF004F9FF216846FFF776
:1042000031FD08B9012000E002200AB010BD00BF56
:10421000780F0020F0B5504D85B004460F462B684E
:1042200093F894300BB9002626E043781B07FAD5A3
:104230000378002BF7D12B68D3F89000503021F091
:1042400050FB0028EFD12B68D3F89060B27D2AB9DB
:1042500063695978B37AB3EB111FE4D1636873B91A
:10426000002F6DD0012FDED16B68186819F0A8FB04
:104270000028D8D06B681E7A304605B0F0BD69685A
:10428000487908283CD002AA0DF1070108F0F0FF98
:10429000064620B940F6BF713220FCF735FB2B688B
:1042A0009DF80700D3F89070BB7DFBB1636902A94C
:1042B0005A78120918F0BEFD0028B4D02B68029875
:1042C000D3F89020BDF80C10D06011829DF8072023
:1042D000D3F89030DA722B68D3F8902001239374CE
:1042E00063695B78C3F303139372C5E7024602ABBD
:1042F00007F10C01F87A1EF045FB002893D0EAE79D
:10430000607CFAB1626919465278120918F092FD80
:10431000002888D0626929685278D1F89030C2F3B9
:1043200003129A7262681068D86092881A82D1F873
:104330009030627CDA722B680022D3F890309A7445
:10434000012699E7024606F10C01F07A1EF01AFBED
:104350000028F0D167E700BF780F002007292DE97A
:10436000F043064687B00F4690464568654C23D11A
:104370001DBB002A48D1D4E9001091F8543013F045
:10438000030218BF012213F00403827103D03378B3
:104390005A1E53425341C37191F894304BB1236874
:1043A000D3F89000503021F09CFA10B963680122D4
:1043B0001A7207B0BDE8F08335B32946707C18F057
:1043C000BAFF072F814664D1637A63B158B1B8F15F
:1043D000000F55D065681EF019FB636868715B7942
:1043E00023720123A37263685879082858D1716831
:1043F000707C20F0CCF86268054671680532707CEC
:1044000008F06CFE00285DD0236893F8540010F08B
:1044100003000AD06268394693F84C303046019563
:10442000927900924246FFF7E3FC00F001006268D7
:104430002368907193F8540010F0040009D093F8A9
:104440004D30394601953046D27900924246FFF709
:10445000CFFC2D4B00F0010065681B68E8711BB1B3
:104460004146304698472872726872B3717C23685F
:1044700083F87E10116899679288A3F87C2024E065
:10448000236893F820110129A4D1284608F008FFD9
:104490006072637A002BA6D0B9F1000FA3D099E720
:1044A00004AA0DF10F0108F0E3FE20B940F69331A4
:1044B0003220FCF729FA04A99DF80F0020F067F8D4
:1044C0000546A1E76368D88018726268137AB3B9A9
:1044D000D388003B18BF0123B06800283FF469AFC0
:1044E000072F7FF466AF517908293FF462AF002BA4
:1044F0003FF45FAF08F0F2FE0123E37259E70123B6
:10450000EAE700BF780F0020940000202DE9F74F64
:104510002F4D934607468A462A688168807C92F828
:104520004880019318F007FF6C7A88F0010806466E
:10453000CCB192F854305B071FD592F84D30E3B1FF
:1045400092F84E40082C23D0204608F09FFD00280A
:1045500018BF8046002E36D0EB7A73B31EF060FA97
:1045600000230446EB72019B8BF800408AF8006040
:1045700083F8008003B0BDE8F08F7B6813B16B68EF
:104580005C79DFE76B68186819F01AFA0028F6D131
:10459000CEB195F80A90B9F1000F14D14946B86828
:1045A00008F07EFE044668720028DCD01EF02EFA69
:1045B00008280AD06B685871D5E72046B96808F01A
:1045C0006FFF0446CFE70024CDE74C46CBE700BFA2
:1045D000780F00202DE9F043A24E87B004463768DB
:1045E00097F857300BB903257BE0D6F8048098F88C
:1045F000063033B998F807201AB998F80820002A2D
:10460000F1D02578012D77D0022D00F0D180002D3A
:10461000E9D197F854209007E5D01BB998F80830F5
:10462000002BE0D0637813F0100FC3F3001714BF12
:104630000822012232EA0303D5D10023A2688DF8B3
:1046400014308DF815308DF81630002A4DD00DF14C
:10465000160305AA0DF115012046FFF757FF336831
:1046600093F841509DF81430002B00F0E28045F0A3
:104670000205002F3BD00DF117004FF00008FFF7A7
:10468000A7F8D6E9003903F1420713F071FD9DF94F
:1046900017302A462146CDF80C800293337ACDE9B3
:1046A00000033B46484601F081FA00289BD0A169EF
:1046B0000120FEF7CBFF002895D0336883F8968061
:1046C0006269002A70D05178C1F3031183F8971002
:1046D0001178527802F00F0241EA0222A3F89820E2
:1046E0000225284607B0BDE8F083FF25C1E729462B
:1046F0002046FFF783FA76E797F820216378022AAD
:1047000019D103F01903192B7FF46DAF97F85430CA
:10471000590714D4356895F854309A072BD1A169FC
:104720000120FEF793FF00283FF45DAF33680122BC
:1047300083F89620C4E703F01803182BE4E76168B8
:1047400000232046B1FA81F11A464909FEF7CEFE50
:1047500000283FF448AFA36932689B7813F0E00368
:1047600004D192F84930002BD4D13CE7402BD1D171
:1047700092F84A30F7E70DF11700FFF729F877684C
:1047800013F0F6FC0023FF22214603939DF9173016
:104790000293337ACDE9000305F14203384601F074
:1047A00005FA0028BBD11EE7FF2283F8972097E780
:1047B00097F854309B073FF416AF637803F0180363
:1047C000182B7FF410AF0DF11700FFF701F813F06D
:1047D000CFFC0023FF22214603939DF9173002935B
:1047E000337ACDE9000307F14203404601F0DEF9D8
:1047F00000283FF4F8AEA1690120FEF727FF00284A
:104800003FF4F1AE336883F8965062696AB151782B
:10481000C1F3031183F897101178527802F00F0258
:1048200041EA0222A3F898205BE7FF2283F8972051
:1048300057E72046FEF74CFE00287FF41AAF336896
:1048400093F85530023B012B3FF6CDAE9DF8153065
:10485000002B3FF4C8AE9DF81430002B7FF4C3AE9C
:10486000FE2506E7780F002030B505468BB0FEF731
:1048700027FE2C7828466946294D04F00F0419F0CC
:1048800050F92B68072C16D193F82011684619F0BF
:1048900051F9002221466846FFF760FD2B6893F826
:1048A0002031022B32D017D8012B1AD041F21C2113
:1048B0003220FCF729F893F8542012F0060FE8D0C4
:1048C00093F8A420134493F82421012AE1D19621DE
:1048D000002021F030FFDCE7033B012BE6D8072C5A
:1048E00019E0062C02D00BD8022C0BD821466846C2
:1048F000FEF7C6FF0446FFF73DFA20460BB030BD79
:10490000072C09D013F010FE0324F4E7072CFBD189
:104910009DF80030012BF7D16846FFF75BFEE9E711
:10492000780F002038B5144D2C6894F8483013B334
:104930006FF00043D4E920129A4208BFB1F1FF3F63
:1049400019D022F036FFD4E92023904271EB030303
:1049500011D3012008F070FD68B12D6808F082FCC9
:10496000044622F026FF054BA4FB03341B1844EB3E
:104970000104C5E9203438BD780F002040420F0003
:1049800070B51E4D06462A6892F823115F294FEA3A
:10499000511096BF1A4B00241B1892F8210100F009
:1049A0003F0098BFDC7813F03DFD2B6893F9580069
:1049B00013F00CFDFEB12B682246996E012013F016
:1049C0009FFD2B68214693F89630022B0CBF4020A8
:1049D000FF2013F045FCFFF715FB2B68064693F804
:1049E000951019B902462046FFF72EFA3046BDE869
:1049F000704013F07BBE22467321DFE7780F002062
:104A0000300A0300F7B52C4C0746226892F82311B0
:104A10005F294FEA511097BF284B00251B18DD78FE
:104A2000936E13B10120FFF7ABFF2368D3F8880022
:104A300013F092FE236893F85420910703D593F85E
:104A40009610022905D052070FD593F89620012A17
:104A50000BD1EA1E012A26D893F85930012B14BF36
:104A600029460321002013F003FF266863689A3665
:104A70001868D7B918F0A4FF63680746186818F0DB
:104A8000A5FF21680246304691F8963091F8201132
:104A90000091394619F0A0F8236883F820510023CB
:104AA000A37203B0F0BD2946DCE718F09BFF014676
:104AB000304619F086F8EFE7780F0020300A03003F
:104AC00008B50120FFF79EFF024B06225B681A71B2
:104AD00008BD00BF780F002008B50020FFF792FF47
:104AE000024B05225B681A7108BD00BF780F0020D9
:104AF00010B50446FEF762FD237A032B0AD1194B49
:104B00001B68986E20B140F62F113220FBF7FCFE97
:104B1000FFF736FF237A012B06D003D9023B012B86
:104B200012D910BDFEF7A8FC0E4C236893F958006B
:104B300013F04CFC2368002283F89520FFF7A2F9BC
:104B4000BDE81040FFF7EEBE064B1B6893F89530AA
:104B50001BB9BDE81040FFF7BFBFBDE81040FFF72D
:104B6000AFBF00BF780F002008B5044B586800F0B5
:104B7000B9FFFEF7A5FC012008BD00BF780F00209B
:104B800008B5FEF79DFC054B00211868A0301DF00C
:104B900038FCBDE80840FFF709B900BF780F0020D6
:104BA0002DE9F3414C4D00230E4607462A6841F299
:104BB0007070116D53720B885381CB69A3F57A74B1
:104BC000844295BF4FF47A7040F2E240B3FBF0F3B9
:104BD000B3FBF0F398BF03F550639BB213848B8C47
:104BE0005384CB8C93844FF47F43D3844FF6FF736D
:104BF000138517B3012130461EF0A6FA014630781E
:104C0000C0092C6894F8483004F11402FBB118F084
:104C100092FBE0B10B6863618B88287A938004F182
:104C20000E0208284AD004F10D0108F021FB88B9D2
:104C300041F2EA313220FBF767FE694668691EF0EF
:104C400036F96B6969461878C0F38010D9E70023FC
:104C50006361E2E72C68637B04F11A0843F0020306
:104C6000637347B3002130461EF06EFA0368C4F840
:104C70001A308388A8F804302B6893F95810186DFF
:104C800008F056FD286815491EF05DFE2868144995
:104C9000036D2A301A88A0F8092093F88E30C37269
:104CA0001EF05AFE0221286801F02AFAFEF75CFC89
:104CB00002B0BDE8F08104F17800D7E794F87E30C7
:104CC0006373A36FC4F80E30B4F87C309380002374
:104CD000C4F81A30E383CFE7780F0020B1D3010086
:104CE0004FD3010008B5FFF745F8044B0020596980
:104CF000FFF756FFBDE80840FEF7DCBB780F002049
:104D00002DE9F04F06468BB0FEF7DAFB337803F05F
:104D10000F03082B05D04FF0010948460BB0BDE842
:104D2000F08F6946304618F099FE9DF80090B9F171
:104D3000000FF0D19DF8013003F00303032BEAD1FB
:104D40002B4C276897F84D30002B39D097F84E80C0
:104D5000637A002B38D1002507F1780397F87E207D
:104D600001999DF811001DF00DFE0DB90028D2D05B
:104D7000256897F8483095F841A042353BB1404648
:104D800008F0C8FB00281CBF05464FF0010A9DF83B
:104D900012B052460299584618F0CDFA2B460746F3
:104DA00058461DF0EFFDC8B120680121A0301DF06C
:104DB00028FBFEF7DFFF31460120FFF7F1FEACE7ED
:104DC000636893F80580C3E71DF020FE0828C2D071
:104DD000A0EB080320725D425D41BDE7002F9AD031
:104DE0000299404608F05CFB0028DDD193E700BF44
:104DF000780F00202DE9F8436C4D002306468946C4
:104E00006869D5F800800370437013F089FC074689
:104E100028B9032008F080FF3846BDE8F883032E48
:104E20006C6942D1237823F00F0343F0030323700E
:104E30000C23637008F1780168691EF03FF898F858
:104E40007E1068691EF04EF80021686921F09FFC11
:104E50002B6893F8482003F1420493F8418092B103
:104E600093F85420520740F1908093F84D20002A87
:104E700000F08B8093F84E0008F04CFB00281CBF1C
:104E800004464FF00108214668691EF009F84146C2
:104E900068691EF01AF8464BD3F80C32002B77D015
:104EA00040F23F613220FBF72FFD052EC2D123785F
:104EB000222223F02F03627043EA491141F00501D9
:104EC000217029680B6D1B6AC4F80F300A6D936A54
:104ED000180AE3741B0C2075637592F87600138E24
:104EE00000284CD04FF0640CB3FBFCF3DBB2A3758D
:104EF000D36A002846D06420B3FBF0F39BB241F2A2
:104F00007070E3751B0A2376D369A3F57A7C844518
:104F100095BF4FF47A7040F2E240B3FBF0F3B3FB7D
:104F2000F0F398BF03F550639BB263761B0AA37638
:104F3000938CE3761B0A2377D38C63771B0AA377C2
:104F4000D2F88F30C4F81F3092F8933094F82420B0
:104F500084F823300B6D22F01F0293F89A3003F08F
:104F60001F03134384F8243007F03CFD94F82430E9
:104F700003F01F0343EA401384F824305AE740F259
:104F8000E24CB1E740F2E240B6E76B68587973E76C
:104F9000052E7FF441AF2B6821681A6DC2F80A1004
:104FA000A188D1811B6D83F8098035E7780F002037
:104FB00000A0085010B500210320FFF71BFF18B90F
:104FC000BDE81040FEF7F2BE074C0321206818F040
:104FD000EDFF0028F4D00121084613F049FC636876
:104FE00009221A7110BD00BF780F002038B5184D86
:104FF0006B68186818F0C3FC044620B940F263518E
:105000003220FBF781FC6B680A22002128681A71A4
:1050100001F076F82B6805201A6D237892F88E40FF
:1050200004EA531404F001042146FFF7E3FE18B923
:10503000BDE83840FEF7BABE0421286818F0B6FF74
:105040000028F5D02B681B6D83F88E4038BD00BF5B
:10505000780F002010B5114C0C22012163682068E4
:105060001A7101F04DF800210520FFF7C3FE18B9B1
:10507000BDE81040FEF79ABE0621206818F096FFA2
:105080000028F5D02368012093F8201113F0F0FBDD
:10509000236801221B6D83F88E2010BD780F00203D
:1050A0002DE9F043054691B00E46FEF709FA2B783C
:1050B0009B4C03F00F03072B07D00125606800F01D
:1050C00041FD284611B0BDE8F08306A9284618F036
:1050D00028FD206806A99A3018F09BFD23689DF8EA
:1050E000181093F89620914240F05981032E03D175
:1050F00093F89720FF2A16D09DF81920150740F144
:105100004E810B9A93F897105078B1EB101F40F036
:105110004681127800F00F00B3F8983042EA002080
:10512000984240F03C8106A832460721FFF716F965
:105130006068C3881BB9037A002B00F0318100231B
:105140008DF814308DF815308DF81630089B002B33
:1051500047D00DF1160305AA0DF1150106A8FFF7BA
:10516000D5F9236893F841609DF814300BB146F0EF
:1051700002069DF818509DF81480012D9DF81570B9
:105180009DF816302FD0022D7FD0002D40F00781E2
:10519000236893F854309D0730D09DF81930980754
:1051A00071D5B8F1000F0BD106A8FEF791F938B907
:1051B000236893F85530023B012B1FD8F7B1FE2628
:1051C00063681B7A33B1574B1B681BB10D9808B14C
:1051D0000F999847314606A8FEF744FD70B10225A5
:1051E0003FE0FF26C5E79DF81900226800F0090C92
:1051F00092F89A10BCF1090F04D009B9012530E0EA
:105200000007FBD592F85420500711D463689B79AE
:10521000002BF3D0236893F854309A07EED09DF812
:1052200019309B0716D4FF2106A8FEF7E7FCE5E737
:105230006268D279002AE9D0424606A8FEF756F9FC
:105240000028E3D02068A0301DF0FDF80028DDD054
:105250000C2506E0B8F1000F06D0314606A8FEF78F
:10526000CDFCFEF787FD2CE706A8FEF731F90028F4
:10527000F3D1236893F85530023B012BBED8002FA1
:10528000BCD0FE21D0E7FF269AE7226892F854208E
:105290009107B3D0616889790029AFD09DF8195082
:1052A00005F009010929A9D1920705F0020568D581
:1052B000002D39D0B8F1000F2AD00DF11700FEF7FC
:1052C00087FA00210320FFF795FD0546D4E9003851
:1052D00003F1420712F04CFF0123324606A9039363
:1052E0009DF917300293237ACDE900033B464046EF
:1052F00000F05CFC002D81D000283FF47FAF2068D7
:10530000A0301DF0A0F800283FF478AF0B25A8E7E7
:10531000002BAED006A8FEF7DBF80028CDD1A8E719
:10532000780F0020280100200DF11700FEF750FA39
:10533000294603200125FFF75DFD0746D4E9003922
:1053400003F1420812F014FF9DF91730324606A906
:1053500003950293237ACDE900034346484600F0C3
:1053600025FC002F3FF47DAF00283FF47AAF206882
:10537000A0301DF068F80028C8D1606800F0B2FBCA
:105380006FE7002D3FF44FAFB8F1000F01D0314669
:105390004AE706A8FEF79CF80028F8D169E760689C
:1053A00000F0D0FB2AE700BF036D10B5044623B917
:1053B00040F263313220FBF7A7FA0222074942721A
:1053C0001B884381FF2380F827304FF6FF73038546
:1053D0001EF0B9FA0023236510BD00BFB1D3010050
:1053E000F8B5184F0E46012178610020FCF79CF8B3
:1053F000054620B940F687013220FBF785FA4FF4C5
:105400009472002122F015FC01210846FCF78CF86B
:10541000044620B14FF49472002122F00AFC3B694B
:1054200013B940F69101E7E7304618F09EF8284698
:1054300018F029FE24B12046BDE8F84018F023BE3C
:10544000F8BD00BF780F0020014B024A1A61704777
:10545000780F00202C010020034B044A1A60044BF3
:10546000044A1A60704700BF28010020D1360000AE
:105470009400002015420000036810B523B940F6DF
:105480005E113220FBF740FA044A13606C3353601C
:105490001369BDE810401B68184700BF780F002053
:1054A00008B5044B586800F04DFBBDE80840FEF716
:1054B0007DBC00BF780F002038B590F8403005461D
:1054C00013F0FD0F05F1420114BF0120002085F803
:1054D000410007F067FC95F84030023BDBB2012B3E
:1054E00094BF0123002385F8483016D807F0BAFE90
:1054F000044622F05EF9094BA4FB03341B184FF05D
:10550000000044EB0104C5E9203407F095FF20B901
:1055100040F602213220FBF7F7F938BD40420F0078
:10552000014936301EF012BA71D3010010B5084C93
:105530000222636820681A7100F0B0FC38B9206854
:1055400018F083F92068BDE8104018F0FBBE10BDCC
:10555000780F0020013808B5C0B20A4B41B10328CA
:1055600001D8185C08BD40F2B9113320FBF7CCF923
:10557000032802D818440079F4E74FF4507106204C
:10558000F4E700BF360A030008B517F053FB054ADD
:10559000D2E84F3F0133DBB2C2E8413F0029F7D1E7
:1055A00008BD00BF900F0020024BA0F10801586811
:1055B000FFF7EABF900F00202DE9F84F0D461E4679
:1055C00000213B4B9346046801601A789DF82870CF
:1055D0009DF82C809DF930909DF834A032B9A4F14B
:1055E00008015868BDE8F84FFFF7CEBF1A2204F152
:1055F000090022F01EFB0123A372BBF1060F4FD856
:10560000DFE80BF00433394E434E3D00E37A23F0DC
:10561000130343F01303E372012304F10E02414626
:105620002846237547F6FF7384F81890E38204F147
:105630000D0318F078F9E37A5B0736D5BA1E04F14A
:105640001C03012A8BBFAA6832681168E2618ABF15
:10565000E161B28892889A80E77600232372154927
:105660002046BDE8F84F1EF071B9E37A23F0150328
:1056700043F01503CFE7E37A43F01003CBE7E37A77
:1056800023F0120343F01203C5E7E27A4AF01A0A44
:1056900022F01B020AF01B0A42EA0A02E272BBE78E
:1056A0004FF484613320FBF72FF9FF23E376D4E72F
:1056B000900F0020B95600002DE9F04F05468DB03F
:1056C0000C4600200121FBF76DFF064620B940F291
:1056D000C7113320FBF718F9A83018F054FC18B1A3
:1056E00096F85430042B2FD1304617F033FF58BBB7
:1056F000B84C04F1080704F10C08AE6A9EB92846BC
:10570000FFF752FF02238DF804608DF805309DF8F5
:105710000430002063F307009DF8053063F30F2089
:105720000DB0BDE8F08FA96A0B68B942AB624FF0CB
:1057300000030B704B708B70CB70DED04145DCD01A
:105740006068FFF721FFD8E7AE6A36B3A24B9E42EE
:1057500026D0043B9E4223D006F13B0A4FF00008BE
:1057600007F0F2F88146B8F1000F40F02E8102A94F
:10577000504618F0D6F9B9F1000F16D004F10D001B
:10578000EF7A17F0100713D09DF8187005993A4674
:1057900016F08CF94FF0010828E005F1330ADDE737
:1057A0004FF001084FF0000ADAE704F11C00E7E7C8
:1057B000002EEFD09DF80830022BEBD0014695F873
:1057C0003230E52250461DF023FD95F83230074671
:1057D0000344504685F832301DF012FD95F83280B2
:1057E000A8EB000CDCF1000848EB0C08B9F1000F45
:1057F0002CD1042305F12301237007F11803AA7AA1
:105800005343E270221D0233637005F10B0353F81A
:10581000040B8B4242F8040BF9D195F814B095F8BB
:1058200015A007F0B3F8C1F3402958464946FFF7E1
:1058300091FE6073BAF1000F04D049465046FFF75D
:1058400089FEA073E7762CE0C8460027EB7AD806DD
:1058500001D45B213DE75907AA7A95F80DE004F1E0
:10586000060005F10E0C2FD5E97EFE292CD111235F
:10587000E27084F805E023701301023363700123A2
:105880002371D5F80E30C4F80630BCF8043083809C
:105890002173EB69C4F80D302B8CA4F811302B7EEA
:1058A000E3744C4F07F1080A56453AD12379022692
:1058B00005F1280066F34613237118F050F82846C6
:1058C000FFF772FE04273FE007F10A030321E270AD
:1058D00053432170023384F805E06370D5F80E302D
:1058E000C4F80630BCF804308380277327442B7E2D
:1058F0007B73EA7A12F0080002D004232371D0E708
:1059000002F00303032B01D12071CAE7520701D52E
:105910000123F3E7022BF1D00BB92171C1E7A221DA
:10592000D7E607F10C094E4515D105F1280018F00E
:1059300016F86A7D6AB92379042762F34613237146
:1059400002262846FFF730FE8DF804708DF80560BA
:10595000DDE60027F4E77EB3B8F1000F26D005F1AD
:105960002808404617F0FBFF31467868FFF70CFE29
:10597000AB6A0022534585F8322097D04B450BD1B6
:105980002379404662F34613237117F0E8FF284657
:105990000226FFF709FE95E79DF80830022B05D196
:1059A0002379012623F0680323718BE723790126ED
:1059B00066F34613237185E7EF7A17F01007C3D01B
:1059C000237966F346132371E1E700287FF43CAFA7
:1059D00007460EE7900F00209C0F0020343270B570
:1059E000054692B20C461E4617F0ECF825B1034A64
:1059F000556014745674147070BD00BF900F002071
:105A000010B5034C606817F0FFF8237C237010BDBD
:105A1000900F0020014B587C704700BF900F002072
:105A200038B5134D686817F0F5F8044620B940F210
:105A300047113320FAF768FFD5E84F3F013BDBB24F
:105A4000C5E8413F0029F7D104F108033422184684
:105A500022F0EFF847F6FF720121E462E283FF22B1
:105A6000627584F82320E27C61F34612E27438BD4B
:105A7000900F002038B5436A044693B90A4D686810
:105A800017F0C8F8606220B94FF4B0713320FAF70C
:105A90003BFFD5E84F3F013BDBB2C5E8423F002A60
:105AA000F7D1606A3B3038BD900F0020036810B515
:105AB00004465BB1596A49B101F10802934204BF3F
:105AC00000230360064B5868FFF75EFD216831B183
:105AD000034B08395868FFF757FD0023236010BDBA
:105AE000900F002038B5046805469CB11349204644
:105AF0001DF035FF124B00221A735A739A73DA7332
:105B0000EFF3108272B6A16A0C3399B9A362E36213
:105B100002B962B62C68616A49B101F108039C427E
:105B200003D0074B5868FFF72FFD00236362002363
:105B30002B6038BDE16A0B60E9E700BFB956000091
:105B4000900F002070B50668044656B3716A154D73
:105B500041B101F108039E4202D06868FFF714FDCD
:105B60000023736221684E7DB6B100232B726B72E5
:105B7000AB72EB72EFF3108272B6886A0A4B40B9CF
:105B80008B62CB6202B962B62046BDE87040FFF777
:105B9000A9BFC86A0360F4E708396868FFF7F4FC36
:105BA000266070BD900F0020980F00202DE9F0476F
:105BB0000468914606460D469A469DF820209DF8B9
:105BC0002C8024B94FF448713320FAF79DFE624FC0
:105BD0003B78BBB9B8F1020F0BD007D9B8F1030F6E
:105BE0000AD033685BB90020BDE8F087FFF75EFF9D
:105BF000F7E7FFF777FFF4E7FFF7A4FFF1E740F2DD
:105C00003D31E1E7636A0BB94021DDE783F811809C
:105C1000CB687BB1097C238E0B4440F272618B42CE
:105C200007DDFFF78FFF3368002BDCD040F25A31DD
:105C3000CAE723860123A3729DF928302376B8F1A1
:105C4000000F7BD122756B691BB15B78C3F3031323
:105C5000A375EB6913B15B88A4F819302B78E27A4D
:105C6000581E4142414161F300029107E27267D43C
:105C7000991E4A424A41E17A62F34101E17211F010
:105C8000020118BFB3FA83F1E37A18BF490961F33F
:105C9000C303E372AB681BB1E37A43F00403E3721E
:105CA0002B6A13B193F90030E3756B6843B104F1CB
:105CB0000D0304F10E029DF82410284617F033FE60
:105CC000AB688BB1A9F1020104F11C02012995BF57
:105CD000DAF800301968E361E16194BFBAF8043082
:105CE0009B88938084F81B90B8F1000F0DD00022A0
:105CF000636A1A705A709A70DA70A26A12BBA36251
:105D000016492046E3621DF02AFEAA698AB153783B
:105D1000927802F01F0253EA02230AD1A26A3B7270
:105D20007B72BB72FB720E4B7AB9A362E3620023F3
:105D30003360636A63B940F2971145E7627582E7A1
:105D4000012298E7E26A1360DAE7E26A1360EDE79E
:105D500000230120636247E7900F0020B95600003E
:105D6000980F002008B5431EDBB2032B0AD80E4A59
:105D70000428D35C03F10503DBB207D1980100F5D9
:105D8000C87008BDFD210520FAF7BEFD032803D128
:105D9000180100F5BF70F4E702280BBF981D581DCD
:105DA0008000C000EDE700BF400A0300014610B5C7
:105DB00004460E4814F08CFF202884F8170111D0F7
:105DC00021460A4814F084FF202884F81E010BD1D4
:105DD00094F8170114F0A2FF20B940F28F2121207E
:105DE000FAF792FD002010BD0120FCE7B3E00100AE
:105DF000014B1870704700BF110000207FB590F86C
:105E0000143103F0FF0223B140F2B7212120FAF749
:105E10007BFD0C78039214F0010318BF8D68CDE967
:105E2000012218BF0195A60707D504ADCE6805EB82
:105E300083050133DBB245F80C6C650707D504AD6B
:105E40000E6905EB83050133DBB245F80C6C013BB1
:105E5000114D80F81D314B68C0F8C830C0F8F830DB
:105E600040F27123A0F8FC30032315F8011B0C420B
:105E70000BD004A900EB820601EB8201013251F83C
:105E80000C1CD2B22B39C6F8CC10013B13F0FF0327
:105E9000EBD104B070BD00BF440A030090F8232189
:105EA0005F2A4FEA52112DE9F04F044689B000F203
:105EB000A980904B0B4493F80790B9F1040F04D1DB
:105EC00000234FF0030980F81F3194F9213102F0CB
:105ED0001F0294F822A1002B94F821314AEA0222F1
:105EE000ACBF4FF01E084FF49678DB0908FB02FAAE
:105EF00014BF4FF4967B4FF01E0B12F03FF9AAEB44
:105F0000000712F077F994F8212107EB0B03804684
:105F100012F0400F0193D04414BF32254FF4FA75AC
:105F20001CF0A0FA019B0544F62F03FB05F5724B0C
:105F300005F5742505F23F25B5FBF3F56DD994F809
:105F4000153103F0FF0A002B5FD1484612F018FE0E
:105F5000684B4FF47A7203EB8903DF6807F522433D
:105F6000B133B3FBF2F6AB365E4406EB45060644AE
:105F7000484612F005FE0190484612F009FE4946D7
:105F80008346204617F07BFE00F18C03019AA7EBB5
:105F90000B0733448DF808A08DF811A09B1A4FF41D
:105FA0007A72B7FBF2F7DF1BD4E92C320397843BFC
:105FB00042F1FF3213EB080342F100025B1B62F176
:105FC0000002CDE906324D4B1878FE2803D094F834
:105FD00054305A0701D414F095F88DF8100002A936
:105FE00094F81701C4F8D870C4F81861DDE90623E5
:105FF000C4E92E2314F00CFF38B940F2B16121201E
:10600000FAF782FC4FF000095FE712F0E9FA14F0AA
:1060100059FD012009B0BDE8F08F48464FF47A7A67
:1060200012F0AEFD334B03EB8903DF6807F2E7366E
:10603000B6FBFAF620365E4446442E4406444846F3
:1060400012F09EFD0190484612F0A2FD834649469B
:10605000204617F014FEA7EB0B0700F18C03019A02
:10606000D4F8D8903344B7FBFAF79B1ADF1BB94535
:1060700013D3A8F1100302A802945D1B94F81C31FD
:1060800003968DF81830022305958DF81030002303
:106090008DF81930FFF7F0F9BBE7184B93F800A023
:1060A000BAF1FE0F03D094F854305B0702D414F019
:1060B00029F88246A7EB0907504615F00BF951461F
:1060C000192F38BF1927874228BF0746384615F0D1
:1060D00047F908B100209DE7D4F8D8003844C4F847
:1060E000D8008238C4F8E00015F0C6F80028C0D106
:1060F000F0E700BF400A030040420F0011000020FB
:1061000001292DE9F34705468A4605D9022900F001
:10611000A28040F2FF7150E0D0E92C4712F04AF81B
:1061200095F8208106460AF0010041461CF00CFD5E
:106130008146404612F02CFDB4F16E0347F1FF3763
:10614000BAF1010F3CD1B8F1040F3CD0B8F1030F04
:106150003CD0B8F1020F0CBF4FF4A6744FF4FC749E
:10616000F618534B03EB880347F1000716EB0906BB
:10617000D5F810811B6A47F10007D8F81C9003F28C
:10618000E73318444FF47A73B0FBF3F0301A67F139
:106190000006041946F1000600F0FEFD05F1E803D3
:1061A000834216D04A46CDE90046D8E9700118F07E
:1061B0004AF9814523D240F276312120FAF7A4FB37
:1061C0004FF4FC74CCE740F6E834C9E740F286446B
:1061D000C6E798F8750090B1D5E93A7A00F032FE3A
:1061E00030B9B8F9E431A8F8E401DF194AEBE37AF1
:1061F0004A4638465146CDE9004618F024F92D4B61
:10620000D5F810211B6892F87610834210D9D36913
:1062100018440029D362D16A41F66A0318BF4FF4CB
:10622000FA73411A138699420DD340F29171C4E773
:1062300031B16425B0FBF5F305FB1303C31AE8E79E
:1062400040F2E245F6E7001946F10006C2E97006A1
:1062500002B0BDE8F087D0F8103113B940F29C715C
:10626000ABE7002683F8E86190F8201183F86C1002
:1062700083F86D10FF2483F86E400339D0F81001C5
:10628000012900F134008CBF0021012107F074FDC9
:10629000D5F8100118F0AFF8C5F8106185F816416F
:1062A00012F09EF902B0BDE8F04714F00BBC00BF3D
:1062B000400A0300A40F002008B50B4B30B10128A1
:1062C0000DD040F612012120FAF71EFB18601A6863
:1062D00041F669039A4206D940F61B01F3E740F6FE
:1062E000C4121A60F3E708BDA40F00202DE9F04F97
:1062F00004468FB01F469246BDF86060039121F0BE
:1063000058FA02902046049117F034FDD4F8CC904E
:106310008346002F00F03182002800F04E82204694
:1063200017F0BBFE80F00107FFB2BAF1000F00F0DA
:10633000FB80029B13F5FA630593049B43F100086D
:1063400000F074FD00F02EFD054604F1E80029463A
:10635000069000F0FDFCD4F8101111B1069817F06A
:106360006BFE1DB1B5F92420A4F80C21BBF1000F80
:1063700016D0D4F8F0B0B5B1A868059BD5E90021D6
:10638000CDE9003880185A4641F1000118F05BF859
:106390008345034608D240F262312120FAF7B4FA6D
:1063A000D4F8C8B0E7E72B46069300F045FDDDE9D9
:1063B00005239D18D4F8C82002F2CF7048F10008D8
:1063C0000344B3FBF2F35343EB1A68F10002C4E950
:1063D0003A32002E40F09F804FF0FF326FF00043C2
:1063E000C4E92A2301214FF0000B04EB0B030691B3
:1063F00093F8243118460593FFF7B4FC059B064635
:10640000184612F0C5FB00F522404FF47A738C3623
:10641000B130B0FBF3F0D4E92A32064400205B1B14
:1064200062EB0802012B72F100010699C0F29C8117
:10643000994570EB020200DB994604EB8B0BDBF80D
:10644000CC304B4594BFC4F8DC30C4F8DC9027BB9B
:1064500019B34900B4F90C0189B21DF0B5FBB4F8C9
:106460000C21D4F810314FEAE07C121A12B2A4F8D1
:106470000C2143B1A3F8E421D3E97021121841EBB8
:106480000C01C3E97021D4E93A32451948EB0C08F4
:10649000181842EB0C02C4E93A02BAF1000F05D019
:1064A000D4E93A23C4E92C58C4E93023039B4FF0C4
:1064B0000009C4F8D8602A462046C4E92E5883F85B
:1064C0000990434617F06CFC039B18725E60002F26
:1064D00000F04E810123039A1370029B049AD4E9C1
:1064E0002A01C31A61EB0201012B71F10002C0F213
:1064F0003D81B548984279EB010200DB1846801BCC
:10650000039B1861D4F8DC00B04234BF00200120A6
:106510000FB0BDE8F08F42F2107329464246E6FB09
:106520000312C4E92A125DE7002F47D06FF0004341
:10653000D4E92A129A4208BFB1F1FF3F00F00E8160
:1065400094F81C31234493F824613046FFF70AFC89
:106550000546304612F01CFB00F522434FF47A70DA
:106560008C35B1338DF820A0B3FBF0F31D44029BB2
:1065700008A813F1AB02049B099543F10003CDE990
:106580000C230223ADF8283014F0E0FB10B940F2E0
:106590008E4102E7D4E92A230C990127DDF8108007
:1065A000521A0D9963EB0103521B5146029D63F190
:1065B0000003002BB8BFD146D34616E7D4E93A1200
:1065C00002980027D4F8C830451AC818B5FBF3F56F
:1065D00003FB05F542F10008029A2D18A5EB020213
:1065E00048F10008AA2A0DD8D4F8B820521AB2FBF4
:1065F000F3F203FB0211691A5D19B1FBF3F148F1E3
:106600000008F0E694F824618DF820703046FFF71A
:10661000A9FB0546304612F0BBFA00F522434FF4C1
:106620007A708C35B133D4F8B8108DF82970B3FB7B
:10663000F0F32B44D4F8C8500993D4E93A030A1A6A
:10664000B2FBF5F26A431218204643F10003CDE98C
:106650000C2317F0A5FB29468DF8280008A81CF08C
:106660001BFA0146DDE90C58BDE652F8041B013364
:1066700001F12B06BE429FBF2B3F0BF101067F1A93
:106680005FFA86FBD9B28842EFD804EB0B0304EB28
:106690008B0993F82431D9F8CC2018460693079239
:1066A000FFF760FB069B0646184612F071FA00F5EC
:1066B00022404FF47A73079AB130B0FBF3F007F140
:1066C0008C031E443044824209D3D9F8CC30DF1BFE
:1066D000002F26DA4FF489615FE62F4666E094F8D2
:1066E0001D21D4F8C8305A4513D90BF10106AB422D
:1066F0005FFA86FB0AD904EB8B03D3F8CC302B333B
:1067000004EB8B021D46D2F8CC70E1E740F2224147
:1067100043E6AB42F4D85B009D42F1D340F23F41E7
:106720003BE615EB0805059B2046B94643F10008FA
:106730000027D4E92C2317F0ECFAD4F8C8305843DA
:10674000D4E93A321B18204642F10002C4E93A3239
:106750002A46434617F0DDFA014646E6029D012728
:10676000DDF81080514627E7814666E64846C6E6D2
:10677000039B1F70C3E90458C4E6BAF1000F7FF40D
:10678000D8AD0299D4F8C870D4E93A238D1AB5FB74
:10679000F7F57D4315EB020801F1AB05A5EB080504
:1067A00043F10003AF42059397D8EF1B002394F801
:1067B0001D0104F1CC029B4664E7BAF1000F3FF4DF
:1067C000FDAE5F46B5E500BF0040420FF7B50123BF
:1067D0001D4E00273370CDE900776846FAF71CFF9D
:1067E0000546C8B10023337003B0F0BD90F8E9014D
:1067F00014F01EFE94F8E90184F8E85114F08EFAC2
:1068000010B94FF4D7711BE0202304F5E07084F831
:10681000E93100F081FADEE7009B002BDDD093F830
:10682000E821002AD9D018884FF6FF739842D9D0B2
:106830002946FAF7B7FE04460028D7D140F2BF1127
:106840003520FAF761F800BFA80F002038B50A4BD1
:106850000D4653F82040084612F09AF9033D04F51E
:106860008564012D04444FF47A70B4FBF0F494BFB6
:1068700028200020204438BD740A03002DE9F84F79
:106880009A4691F8863017460546A3F10E02443B1E
:106890000C46012BD2B218D991F88760443E012EE4
:1068A0008CBF00260126012A98BF0126BAF1000FED
:1068B00003D0012120460DF08DFC94F8E831032B24
:1068C00064D8DFE803F004615B610126EBE727B9D8
:1068D0004FF40B713520FAF717F8012300272046F3
:1068E00084F8E83117F051FDDFF89491D9F80030C1
:1068F000002B4ED051462046984700FB077800F009
:10690000A1FA002847D10221B4F9E4011DF05CF995
:10691000B4F8E4311B1AA4F8E431D4E9702318EB7D
:10692000020243F10003121843EBE0700023C4E9B4
:106930007020C5E904202B7094F8863003F0FD0226
:106940000C2A2AD0A3F12601D1F1000B4BEB010B4D
:10695000442B25D094F88730A3F14402534253418D
:106960002046BBF1000F08BF9B461EF021FD10B171
:10697000BBF1000F16D000232B7219E00323D4F8CB
:10698000F07184F8E831AFE7E769ADE740F26621DE
:10699000A0E7B846B3E70020BFE74FF0010BD9E707
:1069A0000123DDE794F8E831012BDAB22BD12A720A
:1069B000002304F134006B721DF054F86860BAF1E2
:1069C000000F5AD0002E58D1394628461CF064F8E2
:1069D00086B220461EF0ECFC8246BBF1000F1AD1B5
:1069E000864218D308FB00F185F808B0D4E970326C
:1069F0005B1842F10002C5E90432B8F1000F04D17E
:106A000040F2B52166E70223B6E7394628461CF076
:106A100043F8504486B2314620460DF0DBFBD9F8EE
:106A2000003063B101212046984747433044D5E9FF
:106A3000043286B2DF1942F10002C5E9047200F0A7
:106A400001FAB0B97100B4F9E401B1F5803FB4BF07
:106A500089B24FF6FF711DF0B7F8B4F8E4311B1A94
:106A6000A4F8E431D5E904321B1842EBE070C5E923
:106A70000430D5E90423C4E97023BDE8F88F00BFD2
:106A8000540100202DE9B0430D46044618B9F42105
:106A90003520F9F739FF072967D8DFE801F0044FFF
:106AA0004F4B66555C6390F8E8310BB9FC21EFE77A
:106AB0000DF0D0FA00285BD02E4B1B680BB120469E
:106AC000984794F86D30DFF8B090033B012B99F8AC
:106AD000013098BF2825523DEFB2E5691BB9636BC1
:106AE0009D4228BF1D4604F134001CF0BBFF00F19D
:106AF0002B080220A5EB080514F0ECFB022125EA87
:106B0000E575854228BF0546284614F029FC00B9E2
:106B1000A8443A46414620461DF032F8C9F8040020
:106B2000E06914F0A9FB08B9EE21B1E7BDE8B04374
:106B30001EF0F8BBBDE8B04311F008BF01220021F0
:106B4000BDE8B04317F030BC012013F0CBFABDE82C
:106B5000B04316F0F8B990F8E831042B08D04FF4A0
:106B6000917195E740F2271192E740F22B118FE7E0
:106B7000BDE8B0838C000020A80F0020024B00224B
:106B8000C3E90022FFF722BEA80F0020014B587076
:106B9000704700BFA80F002038B5044620B940F266
:106BA00091113520F9F7B0FE90F8E83103F0FF05B8
:106BB00013B14FF4C971F4E790F8E931202B02D0FA
:106BC00040F29311EDE70146044814F081F82028C3
:106BD00084F8E90114BF28460D2038BD856A0000FD
:106BE00008B511F0E7FA054B5A6882422ABF1878B7
:106BF000002080F0010000F0010008BDA80F002077
:106C000038B50446042960D8DFE801F0031A161EDF
:106C10005B002F4B1B7803F0FF026BB9012117F0CB
:106C2000C3FBB4F880300133A4F8803011F0D8FCF5
:106C3000BDE8384013F046BF042384F8E831F5E797
:106C4000032384F8E83138BD41F64B55D0F80C32B7
:106C5000C269AB4290F81812C0F8F0218CBF002531
:106C6000012529B99A4219D000881FF0FAFC15E0D5
:106C700000881FF0F3FC20B940F212313520F9F7FB
:106C800043FEB4F8143200256386B4F816328381CB
:106C9000B4F80432C5814381013B0382D4F8083241
:106CA000204684F87650E362B4F806322386D4F89E
:106CB0000C32E361D4F81032636217F066FB0223F2
:106CC000BFE7BDE8384017F060BB4FF45571D5E71A
:106CD000A80F0020024B0022C3E90022704700BF2A
:106CE000B00F002008B5044B186810B9FFF7F2FF89
:106CF00008BD0C20FCE700BFB00F0020C3693BB902
:106D000083692BB9034B1B681B1A584258417047C3
:106D100001207047B00F002010B5D0E906436BB1D9
:106D2000D0E902219C611144DA680A44DA60826980
:106D30003AB1D3610023C0E9063310BD034A1460A1
:106D4000F5E7002BF6D0DA60F4E700BFB00F0020C3
:106D500008B5C16191B90F4A1368836103B1D86165
:106D600010600023C269C3609AB1D3687BB18168A7
:106D70008B420AD22D213720F9F7C6FD8B69886135
:106D80008361002BEDD0D861EBE75B1AC360002371
:106D9000D36008BDB00F0020014B1868704700BFDA
:106DA000B00F0020034B00201B6803B97047184642
:106DB0009B69FAE7B00F00200B4B002230B51B682F
:106DC00004464FF0FF35104623B911B9002808BF1B
:106DD000104630BDDA68A24203D3AA423CBF154632
:106DE00018461A469B69EFE7B00F002038B5036AD2
:106DF0001BB182689C68A24203D2CD213720F9F7EB
:106E000083FDC1698569D9619D6141B18B619969D2
:106E100041B1CB61C1680A44121BDA6038BD024936
:106E20000B60F4E7D960F9E7B00F0020014B0122B5
:106E30001A717047B00F0020014B00221A71704781
:106E4000B00F0020014B1879704700BFB00F002031
:106E5000F8B5264B0446084600211D680B466DB95F
:106E60005BB1984225D3013CB0FBF3F11C4403FB1A
:106E700001F5B4FBF3F48C420ED9F8BD2E690BB1C9
:106E80009E4207D226B94FF496713720F9F73CFDA0
:106E9000A98A3346AD69E2E7B5FBF3F603FB165664
:106EA00026B9B5FBF2F602FB1656DEB10139ED1A32
:106EB000E1E7451E1D44B3FBF4F4B5FBF0F5AC422D
:106EC000DBD3B3FBF5F605FB16374FB9B6FBF2F78C
:106ED00002FB176727B9B6FBF1F701FB17671FB174
:106EE0000135ECE72846C8E73046C6E7B00F00207A
:106EF00010B50F4C206820B161681FF015FD00230C
:106F00002360A3680BB10023A360237F022B03D16E
:106F100094F82030DB0705D511F006FB002323771A
:106F200010F0DAFD636A94F82000BDE810401847BD
:106F3000B80F00200123F0B5564C85B084F82830F6
:106F4000E36A1B7AFBB1216B94F8342091F8D830B6
:106F5000101E03F1FF3318BF0120022ADBB234BF39
:106F60000122022284F85800032BD1E93201C4E93E
:106F7000120159D8009204F13801474A0420D35C29
:106F8000FB2210F05BFC236BFF2093F8D81011F06C
:106F900067F994F86030032B4BD10023656EA36032
:106FA00094F834306E78012B5BD83146287817F08E
:106FB00067FA6368C0F3C002ADF80C0093F8A03024
:106FC00003F0010161F382004306C7B28DF80C00A3
:106FD00058BF236B9DF80D0058BF93F8C8306870F8
:106FE00058BF03F0010207F05003C7F301073B430A
:106FF00043EA810343EAC2032B70E36A1B7A002B46
:107000003AD0002E38D0A06E11F070FB0022A16E95
:10701000284611F0C5FD00283AD12946A06E05B0DA
:10702000BDE8F04010F072BC40F267410620F9F76D
:107030006BFC012B216B94F8340009D1097F11F00E
:107040001DFFA060A56855B940F28F114720EEE7FB
:1070500000900846D1E9322311F02AFFF1E72035EC
:107060009EE794F860302846032B02D10FF0E0FA37
:10707000C3E70FF0BFFAC0E7284611F037FB10F066
:107080002BFD0021284605B0BDE8F0401FF07FBB76
:1070900005B0F0BDB80F0020880A03002DE9F743C2
:1070A0000F4606467E4CA0B994F86030032B14BFFF
:1070B00062684026E46E1EBFD36E0133D36611F0C2
:1070C00081F801463046A04703B0BDE8F043FFF722
:1070D0000FBF2368002B36D0203394F83420597822
:1070E000012A32D8187817F0CBF96368C0F3C002D0
:1070F000C0F3801993F8A030ADF8040003F0010349
:107100009A42236B93F8C8800CBF0126002688EAB8
:10711000900000F001083FD0B9F1000F0CBF8825A6
:107120000825E36A1B7ACBB3B9F1000F36D1A9B3B6
:10713000A6B310F0DFFC88BB94F8203043F00303C3
:1071400084F82030C0E7636EC7E7022A21D19DF89A
:1071500004201B7822F03F0203F03F03134394F80E
:107160006020032A8DF8043008D103F00303032BB9
:107170000DD094F8203043F00103E1E713F0200F25
:107180000CBF08250C254FF00008C146C9E748256B
:10719000F9E74FF00008C1460825C2E794F83430FB
:1071A00013F0FD0F03D11FF0B5FAC4E91C0111F073
:1071B00009F815F04003014603D0E36E28469847CE
:1071C00082E7B9F1000F31D15EB3206810B3A26F2E
:1071D00045F01005236FB146D4F874C09B184CEBF2
:1071E000E272C0E90432B4F87C30003B18BF0123DE
:1071F0000376B8F1000F01D045F02005E36E284674
:107200009847B9F1000F27D023688BB9A1214720F7
:10721000F9F77AFB63681B6E002BEAD145F0100585
:10722000E7E76268536F01335367E2E79946E0E7A7
:1072300000216268197059709970D970D16BB9B911
:10724000D363136492F8393023B96068154931303B
:107250001CF07CFB00232360002F8AD194F834308B
:107260004BB1013B012B7FF62FAF40F2CA21CEE795
:10727000116C0B60E5E7FFF75DFE257F012D0CD15A
:1072800010F0A0FFE16802232A4601440648237754
:1072900003B0BDE8F04311F01DBB03B0BDE8F083BF
:1072A000B80F0020E7690200C80F002037B502239D
:1072B0003A4C94F8601084F82830E36A03291A7A6B
:1072C00008BF0820636818BF987F0AB10430C0B2B5
:1072D00093F8B01010F0C4FFE36A1B7A23B3A06EDA
:1072E00011F004FA94F834506B1E18BF012384F88F
:1072F00058306368D3E928019A7F93F8B0301B2A8D
:1073000003F1FF3338BF1B22022DDBB2C4E91201A7
:1073100034BF01210221032B30D8009102202049E3
:10732000CB5C204910F08AFA94F86030023B012BC4
:1073300029D960681FF0EBFA2060206830B36368D9
:107340002030D3E9282340E90623E36A1B7AFBB106
:10735000A16E10F0DBFA94F8343003F0FD03012B3A
:1073600019D1636893F8B030033B012B94BF2820F8
:10737000002003B0BDE8304011F01ABA40F2674176
:107380000620F9F7C1FA00232360D6E7606EDCE738
:1073900011F0ACF9DFE703B030BD00BFB80F00203B
:1073A000880A0300F00F002073B5254C054694F8B9
:1073B0006030032B04D102B0BDE87040FFF798BDE8
:1073C000A26822B940F2E2214720F9F79DFA012B89
:1073D0000CD0D4F88030206BD4E91C2100F1C80611
:1073E0009A18009641EBE37320F022F90023A36082
:1073F00035B194F8203043F0010384F82030DAE707
:1074000094F83430002BD6D0032BD4D0012B11D1DB
:10741000FFF74CFF237F012B0FD110F0FDFEE16839
:1074200002232A4601440748237702B0BDE8704092
:1074300011F050BA40F20231C6E702B070BD00BF91
:10744000B80F0020C80F0020034AD2F88030034450
:10745000C2F88030704700BFB80F0020044B054AC7
:10746000C3F884200022C3E919011A77704700BFCE
:10747000B80F002058010020034BD866D3F88400D1
:10748000596211F01DB900BFB80F0020014B002256
:107490001A777047B80F00202DE9F3410D9F15466C
:1074A000404C0C9A6760A3670E9F089B2763C4F843
:1074B0008030BDF824709DF82830A4F87C70002737
:1074C00084F86030137A0F9E94F81CE084F83450EE
:1074D000E26284F82070C4E91C01A3B106F1100334
:1074E00004F1380C06F120081868083353F8041C1E
:1074F0006746434503C7BC46F6D11168336A4B4023
:107500002365736A6365BEF1020F05D1032D3FD871
:10751000DFE805F02D3B2D3B106810F05DFF9DF876
:107520002C0010F07FFFE36A586811F0C3F8236B5A
:1075300093F9D90010F04AFF94F8343003F0FD03BA
:10754000012B0DBF236B0120636800200CBF93F853
:10755000D83093F8B030D4E91C67009332463B46EC
:107560001FF0F5F80028D1D102B0BDE8F081FFF797
:107570009DFE94F83400012805D870B1636893F833
:10758000B01011F075F90120EEE7FFF7D3FCF0E73A
:1075900040F25E314720F9F7B7F9236B93F8D81022
:1075A000EFE700BFB80F0020074B00221A7793F8CF
:1075B0002820022A06D1D3E91C21801841F10001BC
:1075C0001FF0D2B8704700BFB80F0020044A92F8ED
:1075D000203043F0010382F82030FFF789BC00BF60
:1075E000B80F002070B50B4C9D7FE66A367A0EB15D
:1075F0000435EDB293F8B030566812686376002314
:107600002176E3760123A576E0602377C4E904269A
:1076100070BD00BFB80F0020F0B5157A9C7B0DB18E
:107620000434E4B2576893F8D860126893F9D950DB
:10763000054BC3E90427012219765E769C76DD7638
:10764000D8601A77F0BD00BFB80F002070B456683C
:1076500093F8D840126893F9D9500E4BC3E9042629
:10766000FF225C7619764FF47A719A760A4ADD76B3
:1076700002EB84025468022204F5FA741A7700229D
:10768000B4FBF1F400F16E0103F11000214470BC71
:1076900011F020B9B80F0020880A030070B49DF8DB
:1076A0000C40CCB99C7F157A0DB10434E4B2566815
:1076B00093F8B0501268094BC3E9042600221976EA
:1076C0005D760146DA7602229C7603F110001A7785
:1076D000012270BC11F012B90824E4E7B80F0020B1
:1076E000034B186808B120307047586E704700BFD0
:1076F000B80F00200138C0B2032808B504D94FF4F0
:1077000050710620F9F700F9014B185C08BD00BF65
:10771000A00A03000138C0B2032808B504D94FF409
:1077200050710620F9F7F0F8014B185C08BD00BF56
:10773000220B03000138C0B2032808B504D94FF466
:1077400050710620F9F7E0F8014B185C08BD00BF46
:10775000980B03000138C0B2032808B504D94FF4D0
:1077600050710620F9F7D0F8014B185C08BD00BF36
:10777000700C0300F8B50C46074618B9E1211A2031
:10778000F9F7C2F825230B706FF4F973C518437A23
:10779000CB70B5F8B0318B8095F898314B7295F875
:1077A00099318B7295F89A31CB7295F8B5310B758A
:1077B0000821B5F8AE01F9F7F5FE95F8FC3106465B
:1077C000002B40F0AD8008B9F521D8E7D5F8BC20F2
:1077D0006B6990F800E05FFA82FCD8B2C3F30F2126
:1077E000C2F30F27C3F30743C2F30742BEF1000FF2
:1077F0005DD1A373617384F80FC062742073277422
:1078000095F8B000FFF776FFA07495F89001FFF7A8
:1078100071FFE074EB7F637595F8C730A375AB7F9C
:10782000A4F8193095F8C630A4F81B30AB8B6384EC
:10783000B5F8C430A38495F8243084F8263095F840
:10784000253084F8273095F8263084F8283095F8CC
:10785000CC3084F8293095F8CD3084F82A3095F86A
:10786000CE3084F82B3040F2E242337CA371737C3B
:10787000E371B37C2372737DE375B37D2376736804
:10788000B3FBF2F3A4F81D3095F89C31E37795F83B
:107890009D3184F8203095F89E3184F8213095F898
:1078A0002C3084F82C30012385F86331F8BD6374E3
:1078B00084F80CC0A27321746773E07395F890018B
:1078C000FFF718FFA07495F8B000FFF713FFE074FE
:1078D00095F8C7306375EB7FA37595F8C630A4F8AB
:1078E0001930AB7FA4F81B30B5F8C4306384AB8B80
:1078F000A38495F8CC3084F8263095F8CD3084F800
:10790000273095F8CE3084F8283095F8243084F864
:10791000293095F8253084F82A3095F82630A0E7EC
:1079200078B10378012B0CD117F8033C4BB1162327
:10793000074907F10A0085F806321CF004F84423D1
:10794000E37029463046BDE8F84016F041BE00BF5E
:1079500071E60100054B98429FBF00F53470044B5F
:107960001860002088BF1220704700BF00093D004A
:1079700014000020014B1860704700BF4010002029
:10798000044B1B681BB11B1A584258417047012019
:10799000704700BF40100020024B1868003818BF25
:1079A000012070474010002070B515461E46043077
:1079B00016F026FF31460446281D16F021FF049BD1
:1079C000064A04440133126804F597705B08934239
:1079D00038BF1346984238BF184670BD401000208B
:1079E0002DE9F04F8BB005460C46CDE90332037804
:1079F0000B708278437843EA0223C2784B7043EAE3
:107A000002401B0ACA706A798B702B7943EA022301
:107A1000AA79237143EA02411B0AA271637140F6FD
:107A2000C31398428ABF40F2E2420120B0FBF2F059
:107A300099428ABF40F2E2430121B1FBF3F1DDE953
:107A40000323934263D11CF02AF9014603299EBF08
:107A5000CB1CB3FBF1F35943A4F8091089B2EB79BD
:107A6000E3722B7A23736B7A6373AA7B0592A273FA
:107A70002BBB049B83B1A07840F2E24362784B4376
:107A800042EA0022E07842EA0042B3FBF2F002FB55
:107A900010330BB101236373039B83B1607940F210
:107AA000E24322794B4342EA0022A07942EA0042B3
:107AB000B3FBF2F002FB10330BB10123637340F20E
:107AC000E240A046AB46A24641434FF000090E22D9
:107AD0005FFA89F3059898421ED8207816F042FF85
:107AE0004FF6FF73984240F0B9804FF0000B01222F
:107AF0009D4BA17B1B68E2712272002940F0FA8045
:107B0000607B002840F064820BB0BDE8F08F039BDF
:107B1000002B08BF014699E709EBC9009BF80F301D
:107B200002FB094C28448AF80F300CF10803068A3E
:107B30000693ACF81160B7B2408AACF8130086B275
:107B40009BF8140016F016FE8AF819009BF8150031
:107B500016F010FE069B0E228AF81A00002F71D034
:107B6000A3784FF0FB0C607840EA0320E37840EA0A
:107B7000034007F1FA03B3FBFCFC07EB0C03013BEA
:107B8000B3FBFCF394F80DC09BB2BCF1000F08D01E
:107B9000814204BF07F10D039BB281423CBF053314
:107BA0009BB2FB2B02FB094C28BFFB231F44ACF804
:107BB0001530013FB7FBF3F3471E9BB20F44B7FBF1
:107BC000F0F058430F2828BF0F208AF81B00002E22
:107BD0003DD06379FB27207940EA0320A37940EA6E
:107BE000034006F1FA03B3FBF7F7F319013BB3FBCC
:107BF000F7F3677B9BB247B1814204BF06F10D03E7
:107C00009BB281423CBF05339BB2FB2B02FB094771
:107C100028BFFB231E44A7F81730013EB6FBF3F341
:107C2000461E9BB20E44B6FBF0F058430F2828BF07
:107C30000F208AF81C0009F101090AF10E0A0BF164
:107C4000090B45E75F739F738AF81B70BFE702FB60
:107C50000943DE751E768AF81C60ECE70821F9F707
:107C6000A1FC834600283FF440AF466F002E3FF44E
:107C70003EAF6FF404720E2716440DF12702214621
:107C800096F8B40117F0EEF858BBA27B96F8B41141
:107C900007FB02430132D97396F8B5111974B6F88F
:107CA000C410A3F81110B18BA3F8131096F8C610E6
:107CB000A3F81510B17FA3F8171096F89011C81EFD
:107CC000012898BF0421597696F8B010C81E0128E3
:107CD00098BF0421997696F8C710D976F17F197765
:107CE000A273D6F81162002E3FF401AF6FF4047353
:107CF0001E44C2E7B4F8096040F2E2425643B34280
:107D000034BFF31A00230593002398F81B20013396
:107D100098F81C0008F10E08824238BF024688F825
:107D20000220DAB29142F0D8204616F0DBFF049B25
:107D30000746DBB1A27831466378607B43EA0223D1
:107D4000E2780038009743EA02434FF0010218BF7F
:107D5000012016F0BEFF6B894FF47A7253439842AC
:107D600004D91120D0E600BF14000020039B002B93
:107D700067D0627931462379607B43EA0223A27996
:107D80000038009743EA02434FF0010218BF012078
:107D900016F09FFFAB894FF47A7253439842E0D8B4
:107DA00000274FF000094FF00E0AFEB20DF1270335
:107DB00029468DF826900AFB064806EBC6028DF888
:107DC000279098F80F000F3201930DF126032A44F3
:107DD00000935B4617F020F898F810209DF82730A4
:107DE000217A98F81C00069216F0D4FC40B19DF858
:107DF0002630069AE17998F81B0016F0CBFC58B9AA
:107E00000AFB0646059B294620461036009301963C
:107E1000DDE9033216F097FF0137A27BFBB29A42ED
:107E2000C3D8204616F05EFF069000260127A37BEC
:107E3000B34208D8002FF8D0B84600264FF00E0AFB
:107E4000BCE0039FADE70E2306EBC602294603FB09
:107E500006480DF127030F3298F80F0001930DF13A
:107E600026032A4400935B4616F0D6FF98F81C00C0
:107E700098F81080404530D294F808A042469DF80A
:107E80002730514616F086FC814630BB6279237953
:107E900094F806C043EA0223607BDDF818E00AF19B
:107EA000010243EA0C43003840F2E24CB4F80910F6
:107EB00018BF0120CDF800E00CFB01F1079216F08D
:107EC00008FFAB894FF47A714B43834205D3BAF173
:107ED000FF0F1EBF079A4F4622720E2303FB064375
:107EE000D87E80452FD994F8079042469DF82630D9
:107EF000494616F04FFC804628BBA27809F1010ADA
:107F0000DDF818C06378607B43EA0223CDF800C037
:107F10000038E27840F2E24CB4F8091043EA024338
:107F200018BF012052460CFB01F116F0D2FE6B89FE
:107F30004FF47A725343834205D3B9F1FF0F1CBF4C
:107F4000474684F807A00136F6B270E70AFB0649F7
:107F50000DF1270306EBC602294699F80F000F32F0
:107F600001930DF126032A4400935B4616F054FF5B
:107F700099F810209DF82730217A99F81C00069274
:107F800016F008FC40B19DF82630069AE17999F880
:107F90001B0016F0FFFB78B90AFB06432946204672
:107FA00010330193059B0093DDE9033216F0CBFEFD
:107FB000002818BF4FF000080136F6B2A37BB34289
:107FC000C4D8B8F1000F7FF49BADB8460026F5E7A2
:107FD000A07B00230E21DAB2904220D840F2E24387
:107FE000B4F80920A1785A43637843EA0123E17881
:107FF00043EA01439A4203DD049B002B7FF4B1AEB8
:108000006179237943EA0123A17943EA01439A4242
:1080100003DD039B002B7FF4A4AE002074E501FB7D
:1080200003451A46B5F81150F62D3FF69AAE01FBFE
:1080300002420133B2F81320F62ACCD991E600BFF0
:10804000F8B5224D2A681678002E3CD1D2E91043AB
:10805000D2E91472E41B63EB0203241843F100031A
:10806000012C73F1000204DA4FF4A3714220F8F7F7
:108070004BFC4FF0FF32A24276EB030302DA40F2F0
:108080004711F3E7D9B91AF0EDF92B6893F862308C
:108090000B2B03D940F2F2310620E8E70C4A1026F8
:1080A00032F813100144204689B211F031FF064422
:1080B0002B6858684008B04228BF3046F8BD3221CE
:1080C00002260846EEE70026F2E700BF4410002033
:1080D000A40A03002DE9F0410F4686B0054612F0D0
:1080E00011F897F8C7300446FA7F0021D7F89C8131
:1080F0006846934238BF1346264A013B126808FB84
:1081000003F3D66E1822B34238BFF61A1FF091FD62
:108110008DF8084006F1F00301932B78012B18D15C
:1081200006F5AF76019612F00BFED7F89C311B18BE
:1081300041F10001CDE90431019B694695F8240025
:10814000AB6312F065FEF0B940F2EC514220F8F753
:10815000DBFB2C7F002108FB04F42046FFF770FFB7
:10816000D5E91023A41800F1A50200F13E0043F167
:108170000003A41A63F10003CDE90443019B03EB60
:1081800040000190D8E710F02BFA12F09BFC06B0EB
:10819000BDE8F081441000202DE9F04104460E4670
:1081A00020073ED5384D0123A8682B716B7190F8DC
:1081B000C831022B09D10323344900F2F31000F82F
:1081C0002B3C002343721BF0BEFB12F0B9FDAF68DD
:1081D00042F2107C0023B7F8B6E13246D5F80080B1
:1081E000EEFB0C23121843EB0103C7E9762398F842
:1081F000003083B9404616F023FFD7F89C2198F849
:108200001C3031465343D7F898219A1A024408F19A
:1082100020001DF084FB21065EBFAB68012283F8BD
:10822000C921E2060CD5184DA868C17FA03017F00F
:1082300083FBAA68002382F8C931126E0AB32B733C
:10824000A3061CD5104CA068D0E9626590F8C71051
:1082500000F5C07017F070FB23681A784AB9A2685D
:10826000D2E962128E4275EB020202D25868FFF721
:10827000EBF8A268D2F87031013BC2F87031BDE86A
:10828000F0810123DBE700BF441000207577000078
:1082900038B50446154608465AB9032304F2F310CC
:1082A00084F8C83184F8FC510949BDE838401BF016
:1082B0004ABB0B7853B904F2112174301FF0FCFA59
:1082C00020B940F2AB414220F8F71EFB0023E5E75E
:1082D0007577000010B50446006807292CD8DFE840
:1082E00001F00414140A2B102328154B1B68BDE859
:1082F00010409B681847124B1B685B69BDE8104033
:1083000018470F4B1B681B69F8E70023037710F829
:10831000201B29B90CF0C8FC638A013B638210BDA5
:1083200019460CF09DFCF7E740F2BA514220F8F7ED
:10833000EBFA40F2BD51F9E74FF4B861F6E700BF40
:10834000840100203B4B2DE9F0411E6807469C68E4
:10835000337E357F012B3ED14FF0000835E0D4F855
:108360001142E4B16FF404710C442046314616F01A
:1083700043FE16F058FE40B3F5B9B6F93230B4F901
:10838000D211728E5B1AA4F8D2219BB2D4E9782163
:10839000D31841F10001C4E978313D7018E0B8F11B
:1083A000000F14D10135746FEDB284B16FF4047213
:1083B0004FF001081444D8E73178204616F0FAFD52
:1083C00018B194F8B531AB42E7D8002CC7D10024DE
:1083D0002046BDE8F081013594F8B531EDB2AB42ED
:1083E00005D93178204616F0E5FD0028D5D1D4F81E
:1083F0001142002CEBD06FF4047331461C4420462C
:1084000016F0FAFD16F00FFE0028F0D0B6F9323063
:10841000B4F9D211728E5B1AA4F8D2219BB2D4E9BE
:108420007821D31841F10001C4E9783100233B7071
:10843000CEE700BF4410002038B50D46B0B191F82A
:1084400090210C4B91F8B00003EB82039C6910F073
:108450009FFB45340444284604F2E73416F012FE2C
:108460004FF47A73B4FBF3F4204438BD4CF2620449
:10847000F1E700BFA40A03002DE9F04FBA4D04460E
:1084800091B088462F68A860384616F0D9FDD4F818
:108490009C313E7F5E43D4F89831F61A064420465C
:1084A00016F0F0FD2B693044984207D9B8F1000F5F
:1084B00004D10027384611B0BDE8F08F3978224644
:1084C0000CA816F0C8FD2B68DDF8348020461A7F12
:1084D00008F18E0116F01EFD0F210890B4F8AC01D2
:1084E000F9F760F80746002861D094F890010FF082
:1084F00081F807EB40077B7E84F8913104F1A001FD
:108500002B68204604F1B8091B7F009394F82130B2
:10851000E27F17F029FA2B6894F8C77004F5C07150
:108520001B7F3A4628730093204694F8C93017F011
:108530001BFA4846D4E978320133A3FB071342F112
:10854000000207FB02334A1E63F100031FF06DF8BF
:10855000E17F49B1D4E92A13D4E97802884272EB69
:1085600003032CBF0121002194F8C7204AB1D4E9AC
:108570007872D4E96203874272EB03032CBF0122B5
:1085800000222868D4F89C3190F81CC003FB0CFC36
:10859000002900F0C280D4F8E031D4F8A870DB1BC9
:1085A000FF2B07D940F2F1114220F8F7ADF998F806
:1085B0007430A1E7476807FB03C3C3F1000A002A30
:1085C00000F0AD80D4F8E071D4F88831A7EB030E49
:1085D000BEF1FF0FE6D8D4F898310769DF1BA7EB8F
:1085E0000C0C476807FB1EC700236B71002900F0C5
:1085F0009F8082F00103297930460993FFF720FD1F
:1086000029688346099B0A78012A40F0938094F8F0
:1086100090C1564800EB8C004FF47A7C806900F5DD
:10862000FA70B0FBFCF0D1E910C11CF16E0C41F105
:10863000000110EB0C0041F10001801941F1000133
:10864000059404F5DC7408F1E0080494089CCDE975
:10865000023400245346CDE90074CDE90698FEF7B4
:108660001BFF074600283FF424AF2B681B78012B23
:108670006AD0AC6894F8B00010F082FA94F8B02098
:108680003A4B03EB82034FF47A72DB6A03F2E7336F
:10869000B3FBF2F303EB4B0B5844FEF785FF0DF1F0
:1086A0002F00FFF74FFE804600283FF403AFD5F8B8
:1086B00000A09DF82F90504616F0C2FCD8F89C41BF
:1086C000D8F8983104FB09F4E41A0444404616F043
:1086D000D9FC2B69204498423FF6ECAE9AF8001082
:1086E00042460EA8C5F8148016F0B5FC0F999DF807
:1086F0002F2040468E31A61B16F00CFC2B688146BD
:1087000008F5DC7A1B78012B20D1014608F1B8036B
:1087100052463046FEF780FFCCE68A464FE70369B3
:108720004768FF1AD4F898313B44A3EB0C075BE78A
:10873000022360E7D1E91001301841F10001B0EBEC
:108740000B0061F100017BE72046A6E7642130467B
:1087500011F0DEFB841C43465246A4B24946301B4E
:10876000FEF740FFA6E600BF44100020A40A030065
:1087700010F0020F2DE9F047474E86B003D0B368E2
:108780003D2283F8F1213768B46897F81C9094F87B
:10879000B53109F1010296F80C809A4209D13B7873
:1087A0003BB994F8623123B9D4F878310133C4F875
:1087B0007831C30705D5384606B0BDE8F04716F056
:1087C00066BB0DF11700FFF7BDFD9DF8173005469C
:1087D00007F120003B771DF0ECF8824600284DD0D1
:1087E000B8F1000F0BD094F8393043B92B4904F19C
:1087F0003100D4E92823C4E902231BF0A7F8002D97
:1088000041D094F8B5314A46D4E96078029394F89F
:10881000C730019394F8C930009304F5C073D4E9CC
:10882000780117F057F810B1013748F100083A46BF
:10883000434604F1B80010F093FBBAF1000F03D0E7
:1088400029463068FFF746FC06B0BDE8F08773693B
:10885000AB4201D173791BB9FEF718FE0FF064FE2D
:1088600000212846FFF708FE88B90DF11700FFF731
:1088700069FD33689DF8172005461A77002DE6D16B
:10888000B8F1000FAFD1306816F001FBDCE7B8F1AA
:10889000000FB6D0A7E700BF44100020E769020030
:1088A0002DE9F74F0B6980460E46D1F814900193DD
:1088B00016F0C6FBD8F87440054614B16FF4047086
:1088C000044400220127DFF848B192468CB9002FFA
:1088D00040F09A8098F80010002940F095804046BA
:1088E000019216F0ADFB2D1A019A7BD540F27E5114
:1088F0004AE094F8C81103296FD8DFE801F00F02AD
:10890000172A94F8F11101F0FF00002959D094F8CA
:10891000F12141462046FFF7BBFC0122D4F8114269
:10892000002CD4D06FF404731C44CFE7D4F8D431B6
:1089300094F8F11101F0FF0C0029E8D1D4E9781086
:10894000013140F10000994270F1000348D33E220A
:10895000DFE7D4E97601019B834279EB010316D36B
:1089600094F8F1217ABB082284F8C8A184F8062281
:1089700098F800205ABB04F2112108F174001EF08F
:108980009BFF20BB40F2BD414220F7F7BDFFD4F86A
:10899000A41001F080000906E2D4D4F8841101F09B
:1089A000800150EA0103DBD1D4F8E40100F080003B
:1089B00051EA0003D4D194F8F11101F0FF0000292D
:1089C000CED10746AAE794F8F121D2B2CCE75946B6
:1089D00004F2FD101AF0B7FF9FE740F26E51D3E7A3
:1089E00067469BE7D8F810108D4202D340F27F51C2
:1089F000CAE7D6E90410491940EBE575C6E9041544
:108A000012B1404616F055FB384603B0BDE8F08F72
:108A100071E601002DE9F3410023444E0546446F01
:108A200030603371002C7ED06FF4047329461C44EF
:108A3000204616F0E1FA16F0F6FA90B3B5F93230A6
:108A40002846B4F9D2116A8E5B1AA4F8D2219BB2DF
:108A5000D4E97821D31841F10001C4E97831EB6EF3
:108A6000336116F092FB0746F0B9D6F80080022079
:108A700012F030FC0221D8E91B535D1B854228BF50
:108A80000546192D38BF1925284612F069FCE8B9AA
:108A90003369D8F838002B4428443361C8F83800CB
:108AA00014E0D4F81142BDE705F120001CF07CFF72
:108AB0000028DAD13068037F43B920301CF079FFF9
:108AC00020B930681A4920301CF0FDFF0FF01AFC65
:108AD000FEF7DCFC17491848FEF7CEFC3946204665
:108AE000FFF7CAFCC0B90DF10700FFF72BFC9DF89A
:108AF000073004463068037737B9002CEED102B056
:108B0000BDE8F04116F0C3B9002CF8D0214602B000
:108B1000BDE8F041FFF7DEBA3068203002B0BDE8B2
:108B2000F0411CF06BBF2846E9E700BF441000206D
:108B3000D58200007187000099810000014B024A34
:108B40001A6070478401002068010020014B1868FA
:108B5000704700BF840100202DE9F84F44680646A5
:108B60000D4694F88770002F40F0458103F00EFF0A
:108B7000C80740F13E8104F51678284641461AF0B0
:108B8000AEFD94F88C30002B40F0108194F88B30BF
:108B9000002B40F00B81B4F88050D4F81C9003F007
:108BA000FBFE94F85A32022B02D81BB91E2503E1B2
:108BB000042BFBD1C0431842C2B240F0188194F894
:108BC0005B32022B00F20681002BEFD01A4240F0FC
:108BD0000E8194F85DE20EF0C003C02B00F0078117
:108BE00094F8613294F8602242EA032294F86232E7
:108BF00003F00F0342EA0342FE2A03D894F86E32D0
:108C00001907D3D194F8643294F8630240EA032040
:108C100094F8653203F00F0340EA0340FE2804D8BD
:108C200094F86E3213F0F00FC0D1B4F866A2BAF126
:108C3000000F40F0D38094F86E321B07B6D1B4F821
:108C40006812002940F0CF8094F86E3213F0F00FD4
:108C5000ACD194F86A3203F1FF3CBCF11E0FA5D8E9
:108C600094F86CC2012B94F86BB24BEA0C2B94F87D
:108C70006DC24BEA0C4B02D0BBF5C87F96D3B4F85B
:108C800071C240F2E24303FB0CF39B458EDA94F889
:108C90006FB2BBF1000F89D094F870B2BBF1000F36
:108CA00084D0ACF1040C40F67C4B1FFA8CFCDC4504
:108CB0003FF67CAF1EF0800F3DD194F86EC21CF0E1
:108CC0000F0F1AD0B3FBF2FE02FB1E32002A7FF414
:108CD0006DAF94F85DB294F85C220BF00F0B42EA92
:108CE0000B225244013A92FBFAF292B20EFB02F2CC
:108CF0000CF00F0E72453FF659AF1CF0F00F1AD072
:108D0000B3FBF0F200FB1233002B7FF44FAF94F86B
:108D10005F0294F85E3200F00F0043EA00230B4438
:108D2000013B93FBF1F39BB2534394F86E22B3EBF8
:108D3000121F3FF63BAF94F8742294F8733243EA63
:108D4000022394F8752243EA0243B3F5FA7FFFF455
:108D50002DAF99457FF62AAF94F8771294F87622D2
:108D600042EA012294F8781242EA014293423FF625
:108D70001DAFB4F879325D1B2DB2002DB8BF6D4226
:108D8000ADB2B5F5804FBFF411AF2A231B4904F2F1
:108D9000C52084F887301AF0D9FD30461AF0CFFF8D
:108DA0000023A4F87C323846BDE8F88F1EF040FE60
:108DB00000287FF4F0AE25252322002140461EF036
:108DC00038FF1F2384F80A5184F80B31322384F8CA
:108DD0008730E2E7042B3FF4F9AEE7E6BAF1FB0F88
:108DE0007FF62DAFE2E6FB297FF633AFDEE62025E6
:108DF000E2E71A25E5E70127D5E700BFE9E9010029
:108E00002DE9FF410546486800230C4601AA694642
:108E10007830CDE9003316F06BFA20B94FF40471C5
:108E20001320F7F771FD6368019FDE6903F13408D1
:108E3000D7F8A031013E9E4228BF1E4619F012FB12
:108E4000636893F8C0210B2A03D940F2F23106205F
:108E5000E7E7164931F812100144D86989B211F0D8
:108E600057F8044640461AF0FDFD0444D7F8A40123
:108E700002A91034029B6400B44228BF34468442E5
:108E800038BF0446284664F317030293019B8DF80C
:108E90000B60C6F30F26B3F8B231ADF80C60ADF835
:108EA0000E301AF091FC04B0BDE8F081E40A030032
:108EB0002029F7B50646154628D1476897F8873028
:108EC0002C2B23D1002401AA694607F17800CDE9B3
:108ED000004416F00DFA20B94FF40D711320F7F786
:108EE00013FD304687F88740A7F8C4401AF037FFD3
:108EF000019880F8FC510DB180F8C84100F2F310E0
:108F000003491AF020FD002003B0F0BD0220FBE76A
:108F10007577000010B490F887302A2B1AD190F89A
:108F2000CD32BBB990F88632A3B9B0F87C22B0F844
:108F3000CE31C4691A444B1E234492B2B3FBF4F3FE
:108F40009A42A0F87C2205D3034900F27E2010BC8F
:108F50001AF0FCBC10BC704715E701002DE9F04F7A
:108F600081468BB00846D9F8048098F887302C2BBE
:108F700040F0698106A91AF06EFC002305AA04A935
:108F800008F17800CDE9043316F0B2F920B940F2C7
:108F9000A3311320F7F7B8FCB8F8803042F2107212
:108FA000BDF825000499C31A1BB2002BB8BF5B4261
:108FB0009BB2B3F5804FB8F8263038BF002702FBCC
:108FC00003F328BF1E27CB65002F40F00C81BDF8AE
:108FD00020209DF82450DDE90543C4F8B8319DF800
:108FE0001F3043EA0223BDF8222042EA05420B610A
:108FF000A4F8B201C4F89821079AC87DC2F31702F9
:10900000C4F8A8214A7D0093D1E9011315F061FE4F
:109010006061DDE904140B698A7DC87D0093CB682B
:10902000496815F056FEB8F88030BDF82510D8F81C
:109030001C20C91AC4F8BC0084480CB241F3C031EA
:10904000A4FB024302FB0131079BC3F31703E4189F
:109050006FF07F4341F10001E31841F100029842B3
:1090600077EB0203DDE90402D8E990AB92F82C50CB
:1090700038BF2027D2F8983190F815C04668002DE7
:1090800041D085681D4406FB0C55956105695B1B45
:1090900065EB050513EB0A034BEB05051B1941EBCB
:1090A0000505C2E97A35002F40F09D80002908DAD5
:1090B000731E1B1BB3FBF6F399B206FB0144C2E916
:1090C000781720301CF00DFC0546DDE90403426FE3
:1090D000002D00F0A380DAB16FF4047CD3F898611E
:1090E00003F211219444DCF898E1764513D8DCF8BA
:1090F0001152A5B355F8792C6FF4047E9642AE4414
:1091000038D8F446F3E70CF1FF3506FB0535BCE72C
:1091100040F2C6213DE7C3F81122416715F0C9FFAF
:10912000DDE90402436F5BB353F8793CD2F89861F0
:109130009A1B944227D3F61A43682644B6FBF3F6EB
:10914000B6B285B3203000211CF085FC049B93F857
:10915000240011F061FFC0B940F2FD3119E783F836
:10916000115283F8125283F8135283F81452CCF838
:109170001112D3E7C3F811520025CCF81112CDE734
:1091800040F2293105E70026DBE704980023524628
:109190002030CDE9013350F81C3C03FB164300930B
:1091A0005B460BF0CFFC049B5A8E01321644059AA5
:1091B000A2F8D4611A7E012A15D05A6F3AB16FF421
:1091C00004711068511828B940F20331E1E64FF4F8
:1091D0004071DEE6D1F8982150F8790CD1F89C1155
:1091E000121A8A4217D30024484688F88740A8F804
:1091F000C4401AF0B4FD57B10598154980F8FC71C8
:10920000274680F8C84100F2F3101AF09CFB38465C
:109210000BB0BDE8F08F01221A76E4E7C3F8112203
:1092200003F21123436715F044FF059B01220498C4
:10923000A3F8D421203052465B460094CDE9015575
:109240000BF080FCCFE70227E1E700BFFF86930425
:109250007577000008B5034610465A1E032A10D839
:109260004A1E032A0DD8084A0129517014BF0A2149
:1092700000211071937091721946F8F75DFC00207F
:1092800008BD6FF01500FBE7D6080020054A537AA9
:1092900020B143F0040300205372704703F0FB0336
:1092A000F9E700BFD608002010B5044616F0E8FB29
:1092B00008B9002010BDE04316F0E2FB0028F8D00A
:1092C000E31683EAA4635A1E1A42F2D0E3B25A1E8E
:1092D00013405A1E1342ECD0A0B21AF0C9FC0B285E
:1092E000E7D820461AF0C0FC1828E2D8A3B2B3EBA6
:1092F000144F04D184EA142313F0FF1FD9D0044B78
:1093000063405A1E1A4214BF01200020D2E700BF5A
:10931000D6BE898EF0B5070C164BA7F5AA4203EA14
:109320009023543A012A20D927F4004042F6AA2279
:10933000801A18BF0120002216211F24164687EA32
:10934000060562EA0505013511D0DD0301394FEA52
:109350005303ADB245EA56064FEAC4354FEA54040A
:10936000ADB245EA5202EAD1F0BD0020E3E70020A9
:10937000FAE700BFE0FF3F00F8B58D1F40F67A4CDA
:109380000746BDF82460ADB21046BDF8182065450B
:109390003BD8841FA4B264458CBF00240124254619
:1093A000AFBB1D4F3F796FB15CB96FF450654D197C
:1093B000062D06D86FF450640419062C8CBF0024C7
:1093C00001242546FDB1814224D803FB0666B6F58B
:1093D000FA7F1FDCA2F10A0340F676449BB2A34257
:1093E00018D816F0CBFC42F2107300FB06F15A437A
:1093F000B2EB410F0ED9BDF81C50BDF820008542DC
:109400008CBF002501252846F8BD0024C7E797F842
:109410007570C8E70025F6E770100020304BF0B5F6
:10942000B0F860700C4611461A88B0F85E6085B0DE
:1094300097425D8828BF1746964228BF16461B2EC6
:109440002ED0B5F5A47F2DD040F6480301AA9D4249
:1094500028BF1D4616F0F2FCBDF80A309F4228BF17
:109460001F46BDF80C30AB42E78028BF2B46238156
:10947000BDF806309E4228BF1E46BDF808309D420A
:10948000668028BF1D46A580FF232370E3881B3B11
:109490009BB2E02B08D940F219613920F7F734FA72
:1094A0001B2FCED105B0F0BD63881B3B9BB2E02BD8
:1094B00002D940F21B61F0E7238940F64812A3F578
:1094C000A4739BB2934202D940F21D61E5E7A388E1
:1094D000A3F5A4739BB29342E4D940F21F61DCE789
:1094E00070100020F0B502780346DFF894C001F157
:1094F0000C060A700025427840F2712E4A7082787C
:109500008A70D0F80320C1F80320B0F80720A1F832
:109510000720427A4A7294079CF8200001F1240443
:1095200081F8490002F0010048BF0130520744BFF2
:109530000130C0B2EAB2904207D89CF8393081F8C5
:109540004830002381F84A30F0BD03EB05120135A5
:1095500057890EFB07F746F8047B97890EFB07F740
:10956000B760D78924F8027B178AA780578A67815A
:10957000978A2782D78AE782128BA283DAE700BF15
:10958000701000202DE9F341002304460E461746D3
:1095900000F10A08CDE900336846F8F73DF808B154
:1095A000002015E0009DA542F6D03046EB1C16F0D9
:1095B000D4FB3946AA7819F0E5F90028ECD005F17A
:1095C0000A036A7A4146607A19F0DCF90028E3D090
:1095D00002B0BDE8F0810000054A134692F8202051
:1095E00053F8211B11F8030BC0F3801019F0CAB90E
:1095F000DC1500202DE9F7430F4611218046164661
:109600001D46F7F7CFFF044600283AD0694640468A
:1096100019F008FA20B14FF49D613920F7F774F979
:10962000DDF8048098F8DB309B072CD528461BF02A
:10963000A4FD04F15B01A8B1144B1B6813B940F2FF
:10964000F441EAE72A463046984740B9A4F8586002
:10965000A4F85B7084F85A50FF2388F82C3103B0CB
:10966000BDE8F0830A4BD3F80090B9F1000F02D1A6
:1096700040F2FA41D1E72B4604F17D023046C8475B
:10968000E3E70220EBE71A20E9E700BFB40100207E
:10969000B8010020012821D8022B0DD1A2F57A7043
:1096A000104B98421CD8A1F57A70984218D88A427B
:1096B0008CBF1220002070470B48824210D8012B2B
:1096C00007D140F252739A420AD9A1F6C410074B4F
:1096D000EBE7042BF9D140F6C313F4E712207047EF
:1096E00030207047A7F970028FFD7002CBF3700233
:1096F00007B50E4AB2F85430ABB1013B6946A2F847
:10970000543019F08FF920B140F241613920F7F758
:10971000FBF8019A0120B2F89E300133A2F89E3086
:1097200003B05DF804FB1846FAE700BF7010002094
:1097300010B504460A4814F057F80A492046FCF7C9
:109740005DFB204613F067FF38B12046FBF7B4FEFF
:10975000204614F046F8002010BD1220FCE700BFA0
:109760008C100020941000202DE9FF4106788046DF
:10977000012E40F0988031460020F7F713FF054690
:1097800020B940F626613920F7F7BEF8B8F8043062
:10979000002B40F0828013F0DDFE00287FD195F889
:1097A0001431002B7DD12846FFF7C2FF0446002864
:1097B0006FD1584F31463046F7F7F4FE97F838101E
:1097C000064619B110B940F64261DCE73A7F002342
:1097D000CDE9023312F001031CBFF86A0290520770
:1097E00041BF04AA02EB83037A6B43F8082C0029DB
:1097F00045D096F81431002B41D0B8F80230002B38
:109800003DD13B7F3046BA6A009302ABB97F13F07B
:1098100082FFA0B3304614F0BCFB06F14003804643
:1098200005F14002683653F8041BB34242F8041BAA
:10983000F9D12846FFF77CFF024610B140F664617B
:10984000A1E7B8F10C0F07D10146284614F06DFDD1
:10985000F8B940F6686196E7B8F1000F02D040F61B
:109860006D6190E77B7F2846296D43F0040385F8FE
:10987000543014F036FD60B940F66F6183E7B8F8F4
:1098800004202846B8F8021014F04FFD002808BF45
:109890000724204604B0BDE8F0811124F9E73A24FA
:1098A000F7E70C24F5E701210020F7F77BFE0546DA
:1098B00010B940F6826166E714F0FAFA044600280F
:1098C000E7D195F8543095F8A62022B195F8A72055
:1098D000134385F8A600053B012BDAD82B6D13B98D
:1098E00040F692614FE701210846F7F75BFE2946F3
:1098F0004FF49472064612F0D9F80423316D3046C5
:1099000086F8543014F0EDFC0028C2D140F697617F
:1099100039E700BF70100020114BF7B59C7E06465A
:10992000DD7E9F8B14B903F037F80446A5B903F028
:1099300033F8054614B9092003B0F0BD0028FAD069
:10994000304601A98DF804408DF80550ADF8067039
:1099500019F0F6F80020EFE7002CF1D1EBE700BF9B
:10996000341500202DE9F04399466C4B044685B030
:1099700018680F461B790021029020461646684D54
:109980008DF80C3003F086FE664B20462780C4F825
:10999000F831AB6840F8343F14F021FD804602F006
:1099A000F5FF2B7C10F0200FA4F83E8084F83C30AB
:1099B0005D4B0EBF1B22AA8869881B6814BFA4F8E0
:1099C0005E10A4F85E20A4F860201BB194F9741016
:1099D00038469847554F3B79003B18BF012384F820
:1099E0007530534B1B681BB107F10801208898475D
:1099F000012363864F4B1B6813B14F49208898475A
:109A00004E4B1B6813B14E4920889847AB8804F130
:109A100014006A8869780333033201919BB2297874
:109A200092B2009104F11801F7F740FE636923B97F
:109A300041F2AF013920F6F767FFA36913B941F28C
:109A4000B001F7E716F0F8F82062B9F1000F04D082
:109A500004F06CFA20F07F40A06296F84A2006EBF2
:109A60004202B2F82A80404616F088F96FF450633B
:109A700001469844B8F1060F49D90023908C40F272
:109A8000E24284F8763016F079F9FDF7E1F940F218
:109A9000E2430146E1612046C4F8D011A4F8D43174
:109AA00096F84A20E96806EB4206338EA384F38ECB
:109AB000E38414F091FC02A904F18E0019F0AFF8D0
:109AC000FF2384F8FC31FB6D23B1012204F58D7175
:109AD000204698472046FFF71FFF054604F026FA68
:109AE0000C230121B0FBF3F202FB13032046DBB28F
:109AF0005A1DD2B2082A96BF0D3384F89A2084F8F2
:109B00009A3003F0C7FD284605B0BDE8F083012375
:109B100084F876304FF47A73BCE700BF592603000F
:109B200034150020C610002098010020701000207D
:109B3000B0010020AC010020AA100020A8010020E4
:109B4000B4100020034B044A1A60044B044A1A6004
:109B5000704700BFA40100202D4A01008C010020A5
:109B6000BD460100014B024A1A6070479001002077
:109B70005550010010B503210020F7F713FD0446EE
:109B800070B90321F7F7D0FC044620B940F24D31FB
:109B90003920F6F7B9FE034B93F960101AF0B4FFC1
:109BA000204610BD7010002038B518F0EAFE0025E0
:109BB00003F078FA234C02F0FDFE19F0A5FE03F045
:109BC0000FFE05F07DF903F03FFE012002F0B6FE26
:109BD0001D4B1E4A29465D831A601B229D839A8075
:109BE000F9229D771D761A4B22835868194A1B89E2
:109BF00022601422E06104F12400238484F861507F
:109C0000A4F85450A576A580A5751EF012F801237E
:109C100042F2107204F13A0084F8565084F824306D
:109C200084F83930C4E90A221CF00EFD04F1440026
:109C30001CF02FFD0022002384F87050C4E91A2381
:109C400038BD00BF701000203415002003021B0037
:109C5000220B03001B004801044B41F64C521B2110
:109C60005A611974C3E90222FFF79EBF3415002020
:109C700073B5394D0446AB6840F8343F13F009FB27
:109C8000064602F083FE2B7C10F0200FE68784F856
:109C90003C30324B0EBF1B22AA8869881B6814BF58
:109CA000A4F85E10A4F85E20A4F860201BB194F91B
:109CB0007410208898472A490B79003B18BF01236C
:109CC00084F87530274B1B6813B1083120889847FA
:109CD00094F875302046002B41F64C5318BF4FF4D2
:109CE0007A73E361FFF718FE064648B10221208827
:109CF000F7F76EFC60B340F2D3513920F6F704FE5B
:109D000001236386184B1B6813B1014620889847CE
:109D1000164B1B6813B1002120889847697804F11D
:109D20001400AB886A8801910333297803329BB20F
:109D3000009192B204F11801F7F7B8FC636913B906
:109D40004FF4BE61D9E7A3691BB940F2F151D4E7E2
:109D50000926304602B070BD34150020980100205D
:109D600070100020B0010020AC010020A8010020EC
:109D70002DE9F34105460E461AF007FF002800F0D2
:109D8000AF8028461AF096FF30B1B6F80130013B9B
:109D90007F2B01D9122404E028461AF08FFF20B946
:109DA0000C24204602B0BDE8F081284613F0BDFA2D
:109DB0000028F5D128461AF091FE80460028EFD100
:109DC000284606F0A7FC0028E4D042F21073B6F84B
:109DD0000170F17828465F431AF054FF042130786F
:109DE000F7F7E0FB044606213078F7F7DBFB002CA1
:109DF00078D038B141F6F3113920F6F785FD0446E5
:109E000090F8BD80414E3368002B6DD04034204621
:109E10001BF0ABFD002867D020461BF062FD002838
:109E200062D1B8F1000F08D0394B20461B68984723
:109E3000002859D041F60721DEE73649424633680B
:109E400020464969984700284ED041F60C21D3E7B7
:109E500028461AF02FFF40B902210DF10600F7F74E
:109E60002BFB064658B90D249BE728461AF034FF11
:109E70000028F1D1284B1B79002BEDD18AE7002176
:109E800003F0B4FBBDF806302846314633801AF0A3
:109E900041FF28461AF020FFA8B9296A28461AF07F
:109EA00025FF01463046FFF7E3FE044600287FF415
:109EB00078AF3A4631462846F9F77EF8044620B195
:109EC00041F6382198E70121ECE7134BDB6D002BBD
:109ED0003FF467AF024606F58D713046984760E75C
:109EE00042245EE700288AD128461AF0D7FE0146B0
:109EF0000028ADD13A462846F9F75EF80446002816
:109F00003FF44FAF41F6152176E700BFA4010020D2
:109F1000A0010020341500207010002008B5027840
:109F2000032A12D80A4B07D101220A4883F861207C
:109F300003F0CCFE002008BD012A06480EBF012216
:109F40000022002083F86120F2E71120F3E700BF30
:109F500070100020F1960000074B02889B889A42FF
:109F600008D3B0F803309AB222B1044A0020A2F814
:109F700054307047112070473415002070100020B5
:109F80002DE9F3411E4F064697F86130A3BB0C2024
:109F900002B0BDE8F08106EB85036946B3F80380A3
:109FA000B3F801004444A4B218F03CFD00BB019B8F
:109FB000B3F89E2042451DD3A2EB0802A3F89E20D1
:109FC00093F8A82042B993F8A9202AB1B3F89E309B
:109FD00013B9684604F070FC01353278ABB29A428E
:109FE000D9D8B7F8543000201C44A7F85440CFE724
:109FF0000220CDE71220CBE700252C46EDE700BF7D
:10A000007010002008B503F0AFFB15F0A8FF024B5D
:10A0100083F8600008BD00BF70100020014B93F969
:10A020006000704770100020B0F90020F8B514B23D
:10A0300092B202F5A0639BB2B3F5206F36D8B0F9A7
:10A0400002301DB29BB203F5A06189B2B1F5206F59
:10A050002CD802F2F64140F2BE5089B2814227D894
:10A0600003F2F64189B2814222D8002C4FF00A0057
:10A07000C4BF093214B2002DC8BF093394FBF0F4F9
:10A08000C8BF1DB203F0B4FB0A2167B2064695FBB8
:10A09000F1F1384649B203F09DFB074B1B684BB109
:10A0A000A01B40B208B198470020F8BD3020FCE763
:10A0B0001120FAE71846F8E79C010020034B5A8864
:10A0C00002801B7883700020704700BF3415002089
:10A0D0007FB5837806461A2B09D8042B05D90122AF
:10A0E00002FA03F3314A134205D112251AE0292B53
:10A0F00001D03B2BF9D13088B0F5706FF5D26946AD
:10A1000018F090FC88B9019B93F8182102F0FF0524
:10A11000C2B9B27883F81921FF2283F81821684662
:10A1200019F0CBFB284604B070BD09213088F7F741
:10A1300039FA0446002837D002A9B0F8AC0118F06B
:10A1400071FC08B10C25EDE70821B4F8AE01F7F772
:10A1500029FA20B940F628113920F6F7D5FB037803
:10A160001BB994F8C831032BECD1039B93F82E2133
:10A17000002AE7D194F8F02102F0FF05002AE1D18E
:10A18000B4F8B021A3F8302194F8B42183F8322137
:10A19000027D83F83321B27883F8342184F8F021EA
:10A1A000FF2283F82E21BDE70225BBE720003804FB
:10A1B0000188A1F11B039BB2E02B0CD8428844F22A
:10A1C0004810A2F5A4739BB2834204D8034B00202D
:10A1D00019805A8070471220704700BF701000200D
:10A1E000034B1A885B88028043800020704700BFC1
:10A1F0007010002038B50478427804F001038578A7
:10A2000004F0020452EA030101D1112038BDBCB9A7
:10A21000002DFAD0002B08BF144601E0002425468B
:10A22000204615F0EEFE0028EFD0284615F0E9FE96
:10A230000028EAD0054B00209C76DD769883E5E780
:10A24000002BEBD114461D46EAE700BF3415002071
:10A2500013B50088694618F0E5FB18B102242046C2
:10A2600002B010BD684615F0CDFF0028F6D0019869
:10A2700090F82A310BB13A24F1E790F8D23003F08C
:10A28000FF04002BF7D190F8C9309B0706D1FF23BC
:10A2900080F82A31684619F010FBE0E70249CA301D
:10A2A00019F05AFBDBE700BF054502002DE9F84332
:10A2B00003780446032B03D912252846BDE8F8830A
:10A2C0004378032BF8D8437E85780BB9012DF3D161
:10A2D00015F0F80FF0D1A80751D5022DECD1504B55
:10A2E0005B79002BE8D002F057FB35EA000340F021
:10A2F000928094F8029019F0010506D0012322699A
:10A30000A168E078FFF7C6F9054619F0020F07D0FB
:10A3100002232269A168E078FFF7BCF90543EDB29A
:10A3200019F0040F07D004232269A168E078FFF731
:10A33000B1F90543EDB2002DBFD1B9F1050F0FD131
:10A3400094F804900423E16862694846FFF7A2F993
:10A3500000285ED1E3784B455DD1A36899425AD17C
:10A36000237E013B062BA7D801210020F7F71AF91D
:10A37000814638B940F627513920F6F7C5FA690702
:10A380009AD0B0E7A83013F0FEFD18B199F8543018
:10A390009A0742D194F819C0E278BCF1000CA17878
:10A3A000A06818BF4FF0010C012AB4F8009014BF48
:10A3B000B2FA82F2022294F818E018BF5209CB07D1
:10A3C0001ED54B0727690BD56669BB19984207D282
:10A3D00043089F4228BF1F46C31B9E4228BF1E46FC
:10A3E0000F4B19775A77A3F81E9083F820E083F873
:10A3F00021C083F82410C3E90A07C3E90C865CE78F
:10A40000022902D1D4F81080EAE74B0748BF266939
:10A41000E6E7054651E711254FE70C254DE700BF5C
:10A42000701000202DE9F041044688B0002002F0B1
:10A4300085FA23788DF8043063788DF80530A37899
:10A4400003F001058DF806305B0748BF013502F0C7
:10A45000A3FA9DF8063083434AD10DF1070003A902
:10A4600004F1030840F2712E0E468446DAB295429A
:10A4700019D8214B93F8202093F839308DF81C20FF
:10A48000A2788DF81D3032F0050333D112F0050F9C
:10A4900030D01A4CDAB2954217D801A8FFF706FF60
:10A4A00008B0BDE8F08103EB8302013318F80270B5
:10A4B00022440CF8017B9788D2880EFB07F70EFB2D
:10A4C00002F246F8047B7260D0E710F8012B012AF3
:10A4D00010D88A680E46A2F6C412A24206D8326884
:10A4E00004310133A2F6C412A242D3D93020D7E7F7
:10A4F0001120D5E71220D3E770100020CBF37002B3
:10A5000000B589B0437940F271218DF80430837928
:10A510008DF8053001238DF8063003788DF807306B
:10A52000B0F801304B430393B0F803204A430D4980
:10A5300091F820100592A2F6C4128DF81C1000218B
:10A540008DF81D1008498A4209D8A3F6C4138B421E
:10A5500005D801A8FFF7AAFE09B05DF804FB30207A
:10A56000FAE700BF701000203C369C002DE9F04F48
:10A57000437A04468FB0980705D5944A127912B9E8
:10A5800043F001036372657A690704D112263046ED
:10A590000FB0BDE8F08F15F0F80FF7D102F0FCF91D
:10A5A00035EA000340F0928094F8483053B9012D09
:10A5B000ECD1A369864AA3F25373934200F26E81F1
:10A5C000012602E015F00106F3D1AA0745BF731C6E
:10A5D000B2464FF0FF0ADEB26B070AD5B31D7D4AC3
:10A5E00054F82330A3F6C413934200F25781013686
:10A5F000F6B204F1080704F122054FF000095FFAF2
:10A6000089F846452BD823789A1E022A5ED9012B59
:10A61000BCD813B9A378012BB8D86378032BB5D86D
:10A6200094F84930013B062BB0D8684E0121002038
:10A63000F6F7B8FF96F838300546002B5FD10121B8
:10A640000846F6F7AFFF002818BF054605F1A80039
:10A6500013F099FC074600286BD00C2697E7C245FB
:10A6600036D07B680493049A3B6993428ED80120CC
:10A6700069882A89EB89B5F814B00390288C059174
:10A680000290688BCDE900B00020CDE90623FEF7EB
:10A6900073FE002800F00281B8F1000F2AD028884C
:10A6A000059988427FF472AFE988069A91427FF457
:10A6B0006DAFAA89079B9A427FF468AF6B8A5B45AE
:10A6C0007FF464AF3B68049A9A4213D011265EE788
:10A6D000012E0FD13A694048A2F57A73834200F205
:10A6E000DD807B68A3F57A71814200F2D7809A42BF
:10A6F0003FF64CAF09F10109043702357FE7A83076
:10A7000013F041FC00289AD06FF00043D5E92A12DB
:10A710009A4208BFB1F1FF3F91D1637A2846E268BF
:10A72000009304F11803617812F0F5FF0746002842
:10A7300085D0284612F014FF08B13A2627E72846AC
:10A7400012F008FF0028F8D1B37E43B9CDE90933F0
:10A7500006238DF82A3009A8F6F75EFFB8B100216C
:10A760000DF12200F6F7A8FE8046002800F0948044
:10A7700001232246BDF82210FFF7F4F8064620B95F
:10A780004046FCF709FA67B188B10646CBE0099B61
:10A7900093F8A520802ADED093F8BD30002BDAD0C4
:10A7A0005BE70028F1D16178284612F06BFF04F1D5
:10A7B000030AA27821782846534612F00BFF00289E
:10A7C0006ED1002F66D11220DFE700BF701000208D
:10A7D0003CF67002CBF37002A7F97002637A8DF831
:10A7E000247013F00102E16818BFA0690A911EBF2E
:10A7F0000B9001208DF824009F070DD5022B09D165
:10A80000901D54F820000C909DF8240040F00200A8
:10A810008DF824000132D2B2580709D5063254F817
:10A8200022200D929DF8242042F004028DF824206D
:10A8300003F00503052B0ED10B980D9A831899424E
:10A8400009D24B08834228BF0346C91A0B93914291
:10A8500094BF0D910D9209A92846FBF7CFFA94F801
:10A8600048102846003918BF012112F0B0FE94F8B4
:10A870004910284612F091FE284612F0B2FF4146D8
:10A88000284613F02EFD00287FF481AE07264AE00B
:10A890000B2648E0122646E00D2678E6302676E6BE
:10A8A00017B92846FAF708FE5346A27821782846B9
:10A8B00012F0F5FE94F80990B9F1020F05D002F0FC
:10A8C0006BF809EA000909F005094946284612F023
:10A8D00067FE17B9042385F85430C5F850805246F6
:10A8E000A07815F03AFA0146284612F0F3FE2378D4
:10A8F00033B95246A1784046FEF744FE0028C7D13E
:10A900000121284612F001FF0121284612F000FF24
:10A91000002F3FF463AF0421284612F085FE002883
:10A920007FF435AE0C26B8F8000002F0A5F900213E
:10A93000B8F80000F6F74CFE00283FF428AE41F2CC
:10A940007D313920F5F7E0FF10B5437994B0032B42
:10A9500057D823F0020302798DF80630D0F806307C
:10A960008DF80420CDF807304389027BADF80B3019
:10A9700001238DF8052040F271228DF80D300388F7
:10A980005343049341884A430792A2F6C412847B3E
:10A99000417B41EA0421ADF82810047CC17B41EAE7
:10A9A0000421ADF82E10847C417C41EA0421ADF8ED
:10A9B0003410047DC17C41EA0421ADF83A10417D98
:10A9C000847D41EA0421ADF84010C17D007E41EA5A
:10A9D00000210E48ADF8461000218DF84C108DF87E
:10A9E0004E100B4990F820008A428DF84D000AD88D
:10A9F000A3F6C4138B4206D801A8FFF7B7FD14B025
:10AA000010BD1220FBE73020F9E700BF70100020D6
:10AA10003C369C0030B5044695B0002001F08EFF16
:10AA200001A92046FEF75EFD054601F0B5FF9DF841
:10AA30000D4034EA000302D0112015B030BD14F0EF
:10AA4000050F1ED014F0F80F1BD101F0A5FF8443B1
:10AA5000F2D104AB0C49E2B2954203D801A8FFF74A
:10AA600085FDEAE7DA681846A2F6C4128A4206D8DB
:10AA7000026804330134A2F6C4128A42EBD93020B2
:10AA8000DBE71220D9E700BFCBF3700273B50623D2
:10AA90000024CDE900448DF806306846F6F7BCFD89
:10AAA00008B1002610E0009C94F8A530802BF4D06B
:10AAB00094F8BD60002EF0D094F80931002BECD151
:10AAC00094F8A430002BE8D101210020F6F76AFDAC
:10AAD000054620B941F2B0313920F5F715FFA8300D
:10AAE00013F051FA244B93F8383083B3F0B195F852
:10AAF0005430053B012B19D8284613F04AFA044676
:10AB000010B141F2BB31E7E72846FAF74DFC95F862
:10AB100054302246214623F00403284685F8543059
:10AB200013F003FC80B94FF49E51D5E7012108468C
:10AB3000F6F738FD054610B941F2C731CCE7A83029
:10AB400013F021FA68B90C24204602B070BD30B968
:10AB5000002EF8D0FF2384F8A4300024F4E7002E60
:10AB6000F8D1284613F015FA04460028ECD12846FF
:10AB7000FAF71AFCE8E700BF701000202DE9FF414A
:10AB8000077804460E46EF2F04D91226304604B04B
:10AB9000BDE8F081B0F80130ADF80C309DF90C2023
:10ABA0009DF80C30002AF0DB9DF80D209507ECD1C4
:10ABB000D80660D4990603F0030259D5002AE4D1DF
:10ABC0001D0703D503F06703012BDED16378180757
:10ABD00011D42179E278E07942EA0122617942EAEE
:10ABE0000142A17941EA0021207A41EA00418A42EA
:10ABF000CBD81F2AC9D9627A013A062AC5D8A27AC7
:10AC0000032AC2D813F0040102D1023A012A03D860
:10AC1000E27A012AB9D811B9A27C032AB5D813F077
:10AC20001001227D37D0012AAFD1237E012BACD871
:10AC3000002940D06378D90703D501F079FD0028B9
:10AC400040D06378227D03F01803082B4AD1022AF2
:10AC500038D11FFA87F803214046F6F7A3FC0546D2
:10AC6000002845D012F061FB00284DD00C268DE75E
:10AC7000032AA5D189E713F0600F86D103F00F02F4
:10AC800003F00703052BA1D0931E012B9ED9002AA8
:10AC90007FF47BAF9AE7022A04D103F06F03092BFC
:10ACA0007FF473AFA37D013B022B3FF66EAFE37DD4
:10ACB0000F2BBAD969E701F06FFE820707D4237D15
:10ACC000022B01D1112661E7A37D022BFAD001F0FE
:10ACD00063FE4307AED4237D032BF3D0A37D032B68
:10ACE000A8D1EFE7022AB4D0237F002BB1D0E9E747
:10ACF00003214046F6F718FC0546002843D0234BB5
:10AD000093F9601019F000FF002138461AF0B6FBE5
:10AD100028BB284619F0BFFF21463070E074284652
:10AD200005F050FDE37E0646002B3FF42FAF0028D0
:10AD30007FF42CAF0246E96C6846F6F793FD324685
:10AD4000E86C012111F0BEFFE96C68460422F6F7B9
:10AD500089FD32463146E86C11F0B4FF16E7403009
:10AD60001AF003FE0028D4D0637813F0330F7FF479
:10AD70000CAFA77D2846296A19F0B8FFFCF7CAFC7A
:10AD80008742C6D072E7072600E700BF7010002098
:10AD900030B502798BB00346042A5CD84488B4F5F8
:10ADA000804F58D82D4800211044ADF800108DF880
:10ADB0000810827C457B42F010028DF81D1042EA9B
:10ADC0004502C57D007F42EA850242EAC00202F0E8
:10ADD0001F028DF80020BDF80020ADF809201A8868
:10ADE0008DF80E40240A8DF80B20120A8DF80D10F4
:10ADF0008DF810108DF80C208DF80F405A7BD3F889
:10AE000007008DF811205A79059002A88DF81220BC
:10AE10009A798DF81320B3F80B209B7BADF818209E
:10AE20008DF81A307F238DF81B3001238DF81C30EC
:10AE30008DF81E308DF81F108DF820108DF823101E
:10AE40008DF824108DF821108DF822106946FFF737
:10AE500095FE0BB030BD1220FBE700BF220B0300B4
:10AE6000F7B5B0F801200546B0F803309A4202D990
:10AE7000122003B0F0BD052AFAD9052BF8D9B0F895
:10AE80000530002B40F09C8003210078F6F78AFB08
:10AE90000646002800F0968019F004FF0028E7D14C
:10AEA000304619F019FF0028E2D1304619F0F6FEBD
:10AEB0000028DDD1304619F0F9FE01460028D7D12F
:10AEC00028781AF0DBFA0446002852D106212878A7
:10AED000F6F768FB0746002852D1BCB92F78062048
:10AEE00011F02DFEBFB200285DD006213846F6F7DE
:10AEF0001BFB002857D080F8BD400446354B204648
:10AF00001B68984706F12803C4F88830E28D94F84E
:10AF1000300094F834104FF6FF7301F0FF0700295A
:10AF200054D19A4294F8351046D0002814BF3B27DC
:10AF30002327A06811F054FFB5F80320014640F222
:10AF4000E24073794243204600971AF0E3FA002862
:10AF50003AD004F14001284615F00BF873793046D9
:10AF6000237419F098FE014620461AF0E5FA0020F5
:10AF70007FE740301AF0B5FC0028A7D00C2078E716
:10AF800090F8BD303BB1014628781AF0BEFD114B58
:10AF900038461B68984706F12803C7F88830002315
:10AFA00087F8BD3099E704213846F6F7BDFA044624
:10AFB0000028A3D107205CE7002918BF0927B8E7BC
:10AFC000112056E7422054E7452052E79A42ACD17F
:10AFD0000927AEE78C0100202DE9F743074603213E
:10AFE0004078F6F7DFFA0546002800F0B880042123
:10AFF0007878F6F7D7FA044606217878F6F7D2FA89
:10B0000006462CB1C0B141F6B2313920F5F77CFCCF
:10B0100018B90C2003B0BDE8F083044690F8BD9049
:10B020003B7804F14008DB07404640F18B801AF082
:10B0300058FC18B10020EDE78146F1E7284619F0E9
:10B0400031FE0028E5D1284619F046FE0028E0D15F
:10B05000284619F023FE0028DBD1284619F026FEE9
:10B060000028D6D13B78C3F34003A373B9F1000F96
:10B0700032D06B794046627B237495F846301B09C9
:10B0800063F30712627309F0C5FC0028C2D156B100
:10B09000B9F1000F07D014F0CFFD344BC6F8900083
:10B0A0001B7E86F8A33014F0C7FD206002F03EFF3F
:10B0B00020F07F406060284612F037F90028B9D0B0
:10B0C000B9F1000F32D02A4B40461B689847002840
:10B0D000B0D041F6054198E7A06811F059FE00286C
:10B0E00097D1E28D94F8300094F834104FF6FF7346
:10B0F00001F0FF07002934D19A4294F8351011D09D
:10B10000002814BF3B272327A06811F069FE6B7944
:10B11000014600972046226F1AF0FCF90028A8D1BA
:10B12000452077E7002918BF0927EDE7114B4A466C
:10B130004046596909F07AFC00283FF47BAF41F69C
:10B140000A4162E7B9F1000F04D003B0BDE8F04353
:10B150001AF0DDBC03B0BDE8F0431AF09EBC4220FB
:10B1600058E79A42CCD10927CEE700BF70100020E3
:10B17000A001002034150020037813F0F80F73B5F8
:10B18000044640F0AA8013F0010307D142780F2A49
:10B1900000F2A5808278012A00F2A180B4F809208B
:10B1A000B2F5FA7F80F09B80B4F80B2043F6F6717D
:10B1B0000A3A92B28A4200F29280627B1F2A00F21F
:10B1C0008E8002F01702172A03D10C24204602B009
:10B1D00070BD4BB9E51CCDE9003305238DF8063071
:10B1E0006846F6F719FA38B105216846F6F764F9AA
:10B1F000054688B90724E9E700986378827A9A427D
:10B20000EED100F10C012B46A278C07A17F0BAFB00
:10B210000028E5D00B24D9E7324B0146BDF80000E9
:10B2200005F150061B689847BDF8003030462B8169
:10B23000237883F00203C3F34003EB742378C3F352
:10B2400080032B756378AB72A378EB722378C3F31A
:10B250000003AB75637B2B76D4F80330EB60B4F856
:10B2600007302B82A27A637A43EA022342F21072F9
:10B27000A5F88830B4F80B305343C5F88C3009F08A
:10B28000CFFB58B10521BDF80000F6F7A1F9002861
:10B29000B0D041F64C713920F5F736FB284612F054
:10B2A000DEFA044680B130461AF0F7FB10B141F6E1
:10B2B0005271F0E70521BDF80000F6F789F9002882
:10B2C00083D041F65371E6E7074B1B68002B3FF430
:10B2D0007DAFBDF80000984778E7112476E7122487
:10B2E00074E700BF9001002094010020014914F090
:10B2F0006EBD00BF781000200278034672B142781C
:10B3000062B142881A2A09D982881A2A06D90068A5
:10B31000034A106000209B8893807047122070477A
:10B320003415002002680020014B9A60704700BF6E
:10B330003415002002680020014BDA60704700BF1E
:10B34000341500200378A3F10A02112A9BBF024A98
:10B350000020122013747047341500200378FF2B4F
:10B3600016D14378FF2B13D18378FF2B10D1C378EC
:10B37000FF2B0DD1037923F0E0021F2A08D113F02F
:10B38000E00F05D05B09034A002082F820307047A7
:10B3900012207047701000200378012B9DBF03F02E
:10B3A0000103034A0020122098BF82F83930704709
:10B3B0007010002002680020014B5A61704700BFE6
:10B3C00034150020014B18760020704770100020C3
:10B3D000014B587600207047701000202DE9F04F87
:10B3E00004468BB00078049113F0BCFAA37B0821CB
:10B3F0000393F6F7D7F80646002842D0466F002E92
:10B400003FD06FF404714FF000084FF00E09771829
:10B4100046460DF12602214697F8B40113F022FDAD
:10B42000A0B9039D0135EBB2039397F8C730002B09
:10B43000FB7F18BF0126002B18BF4FF00108D7F87B
:10B440001172FFB16FF404721744E2E79DF82630E1
:10B4500009FB0342B2F8112052B109FB0343B3F8D0
:10B460001330002BEBD197F83030002BE7D003E0FE
:10B4700097F8D820002AF0D00C2630460BB0BDE853
:10B48000F08FB046039B1F2B00F2EA802378EF2B4E
:10B4900000F2E680B4F8092040F67C41131F9BB20D
:10B4A0008B4200F2DD8094F80EE000230E20D9B22A
:10B4B0008E4554D87EB1A178637843EA0123E178C0
:10B4C00043EA0143944903F18073FF3B23F07F4338
:10B4D0008B4200F2C580B8F1000F0FD0617923795B
:10B4E00043EA0123A17943EA01438B4903F18073C5
:10B4F000FF3B23F07F438B4200F2B280E379002BC5
:10B5000000F0AE80237A002B00F0AA80E37A072BAC
:10B5100000F2A680237B012B03D9BEF1010F00F2BC
:10B520009F80637B022B059355D000F2998040F2F7
:10B53000E243A04626464FF000095343069304F128
:10B540000F0307935FFA89F2964517D801F024FAA2
:10B55000039B06460E2B40F29B8009268DE700FBDD
:10B5600003410133B1F81170B1F81310002F18BF67
:10B570000126002918BF4FF0010898E7F07BEF285B
:10B580006ED80023D9B28E4527D896F810A00AF1BC
:10B59000FF331E2B64D80E2303FB0941B1F81120A1
:10B5A000B2F5805F5CD2B1F81330B3F5805F57D24B
:10B5B000B1F81500FB2853D8B1F81710FB294FD864
:10B5C00096F81BC0BCF10F0F4AD8377F0F2F47D812
:10B5D00052EA03050BD111264FE7914205D00E2107
:10B5E000079D5943695C81423AD00133CAE750EA6A
:10B5F0000105F0D05CEA0705EDD042EA000B5BEAFA
:10B600000C0506D0002AE6D00028E4D0BCF1000FDB
:10B61000E1D043EA010B5BEA070505D0002BDAD045
:10B620000029D8D0002FD6D0BC45E34638BFBB4652
:10B63000DA45D0D3059D3DBBA0B1024494F802A0E9
:10B64000069D013AB2FBF0F0627842EA0A2294F8D1
:10B6500003A042EA0A42B5FBF2F25043604501D929
:10B6600012260AE781B10B446279013BB3FBF1F189
:10B67000237943EA0223A27943EA0243069AB2FB02
:10B68000F3F35943B942EBD809F101090E3659E7F2
:10B690000DF0C8FB05460DF065FE94F80EE00021A4
:10B6A0004FF00E0CCBB29E450CD840F2E243B4F8FA
:10B6B00009005843E37A0B2B30D940F2F2310620CF
:10B6C000F5F722F998F819200F46002A83D0531E67
:10B6D000134280D198F81A30002B3FF47CAF03F16D
:10B6E000FF3919EA030F7FF476AF16423FF473AFC8
:10B6F0001E423FF470AF0CFB0143B3F8113083429C
:10B700003FF669AF0CFB0743013108F10E08B3F8AF
:10B710001330AB42C6D95EE700FF0F00A04A0027F6
:10B720004FF0960802EB4303BA46B9463D46598CA2
:10B730000EF0EEFB8346A37BFEB2B34231D82078F5
:10B7400013F010F90821F5F72DFF00284FD0466FB0
:10B75000002E4CD06FF404730DF1260221461E44D6
:10B7600096F8B40113F07EFBC0B9594603903046F9
:10B7700014F00FFC039B07463046194614F009FCF1
:10B7800007F19603B9441B1A984538BF984696F8B6
:10B79000B5319A4503FB075538BF9A46D6F8116272
:10B7A000D6E70E23594601375E4306F10F022244C5
:10B7B0001046059214F0C5FD0390FCF7E1F800284F
:10B7C0003FF44EAF059A00212644104614F0B9FD0F
:10B7D000039B03F196029944121A904538BF904694
:10B7E000327C924502FB035538BF9246A3E7237B88
:10B7F000012B08BF0AFB09F5B8F5BE7F98BFE735F6
:10B80000FCF7CAF838B9B4F8093040F2E2425343C1
:10B81000AB42FFF4E0AE207813F0A4F80821ADF8B5
:10B820002400F5F7BFFE0546D8B9082109A8F5F7A9
:10B8300043FE054608B907261FE613F066F805F132
:10B84000200009F0E7F8064660B10821BDF82400A1
:10B85000F5F7BEFE00283FF410AE42F277713920B2
:10B860002EE7012695F86870002F7FF405AE0920B9
:10B870004FF00E0A11F063F994F80E808146A27B16
:10B88000FBB29A420AD8C14580F08580002ED2D101
:10B890000821BDF82400F5F79BFECCE70AFB034323
:10B8A0002846D97B13F075F818B108F1FF385FFA14
:10B8B00088F80137E3E709FB0648284698F80F1097
:10B8C00013F067F88246002850D109210DF12600B7
:10B8D000F5F7F2FD824610B942F2A171BFE712F00E
:10B8E00010FEBDF82430AAF8AE31BDF82630AAF813
:10B8F000B03198F80F308AF8B4316B6FCAF8113252
:10B900000AF211236B67049B013703EB4606BAF872
:10B91000B0317380A17BFEB2B142CCD801232B7031
:10B9200023782B75A2786378E67843EA022362795C
:10B9300043EA0646237943EA0223A279AE6043EA4A
:10B940000243EB60E2796A75227AAA75627B002A6B
:10B9500014BF01200020E87540D140F2E240B4F865
:10B9600009704FF00E0C4743104626E0B0F8B03196
:10B97000D0F811B2039312F0C4FD039BBDF824204C
:10B98000AAF8B031AAF8AE2198F80F30CAF811B26F
:10B990008AF8B431B7E700274FF00E09BAE700BFC5
:10B9A000220B03000CFB0042B2F8132022B1B7FBBC
:10B9B000F3F203FB12727AB90130C2B291420DD98F
:10B9C0000CFB0042B2F81120002AEBD0B7FBF6F2D4
:10B9D00006FB1272002AE5D00123EB75B4F809309A
:10B9E00040F2E2424FF000080E275343A5F85420DE
:10B9F0002B656B60237B2B76A37B5FFA88F6B342C3
:10BA000029D8E37A286D0B2B3FF657AE6C4A02EB30
:10BA10004303598C0EF07CFA2B7E80466E6F002B10
:10BA200040F09C80002E68D06FF4047906EB090783
:10BA30001E463846414614F0ACFA97F8B531C7F8BF
:10BA40009C01D7F8117200FB0366002F55D06FF4EC
:10BA5000047E7744EDE707FB0646284608F1010817
:10BA6000F17B12F096FF014610B942F2F671F6E64C
:10BA7000337C80F8B531B27C737C43EA0223A0F8B2
:10BA8000C430327DF37C43EA02238383EB7D80F86C
:10BA9000D43080F82C30B6F8153080F8C630B6F8BF
:10BAA00017308377707E14F05EF981F89001B07ED4
:10BAB00014F059F981F8B000F37E81F8C730337F74
:10BAC000CB77A278637843EA0223E27843EA024321
:10BAD0006279C1F8CC30237943EA0223A27943EAA0
:10BAE00002434B626B68C1F8D0308B626B7D81F88A
:10BAF000C930AB7D81F821307EE76B6F2E616BB171
:10BB00006FF4047C634493F8B521D3F89C11C3F817
:10BB1000986101FB1266D3F81132F0E7DEB92B69A8
:10BB20006A7DE87D0093D5E9011313F0D2F82B6903
:10BB3000AA7D0646E87D0093EB68696813F0C9F8B2
:10BB40006B6FB3B36FF404721344C3F8BC605861F5
:10BB5000D3F81132F5E742F62A0180E6AEB16FF470
:10BB60000477F7190026B1463846414614F011FA19
:10BB700097F8B531D7F8117281449E4238BF1E46FE
:10BB800027B16FF404700744EEE7B14609FB06F6EF
:10BB90006F6F2E61002FC2D06FF404710F444146C5
:10BBA000C7E96669384614F0F4F9D7F81172361A05
:10BBB000F0E723780026049A1370A37B53705CE4AB
:10BBC000220B03002DE9F0470446BEB000780F4673
:10BBD00012F0C8FE082194F80E80F5F7E3FC054644
:10BBE00008B3456FFDB16FF40472AE180025A94685
:10BBF000214696F8B40113F0FEF868B996F8C730FC
:10BC000008F10108002BF37F5FFA88F818BF4FF0A6
:10BC10000109002B18BF0125D6F8116226B16FF477
:10BC200004731E44E4E7A946B8F11F0F4FD82378E8
:10BC3000EF2B4CD8E379072B49D8237A012B02D973
:10BC4000A37B012B43D8637A022B04D1112528460C
:10BC50003EB0BDE8F0873AD894F80EC0264622469A
:10BC60000023D9B28C4534D8B9F1000F15D0A27891
:10BC7000637843EA0223E27843EA0243604A03F12D
:10BC80008073FF3B23F07F43934220D8638940F6C3
:10BC90009B72053B9BB2934219D8002D00F0A78000
:10BCA0006279237943EA0223A27943EA0243544AA0
:10BCB00003F18073FF3B23F07F43934207D8A389AE
:10BCC00040F69B72053B9BB2934240F29080122556
:10BCD000BDE7D17BEF29FAD803EBC3012144B1F8CA
:10BCE00010E0BEF5805FF2D2498AB1F5805FEED2F6
:10BCF00092F814A0BAF1070FA8D8507DBAF1000F3E
:10BD0000A4D001380628A1D8BEF1000F05D1002922
:10BD10009CD0012501330932A3E74FF00109002926
:10BD2000F8D0F6E7317D1A4608428FD0717D08427F
:10BD30008CD003EBC3012144098AFB2986D802EB8E
:10BD4000C202013309362244528AFB2A3FF67EAFF3
:10BD5000DAB29445E6D82B464A4609A92046FBF7B5
:10BD60003FFE054600287FF472AF01A909A8FFF73E
:10BD700035FB054600287FF46AAF207812F0F2FD0B
:10BD80004FF6FF73984204D142F281513920F4F703
:10BD9000BBFD0821F5F706FC804620BB42F283512B
:10BDA000F4E706EBC606404609F101092644F17B9B
:10BDB00012F0EFFD10B942F28851E7E7B37D80F849
:10BDC000D530F37D80F82D30A27B5FFA89F696425C
:10BDD000E7D323780DF106017A70B81C52003B704E
:10BDE0000FF064FE33E7A946EEE709252FE700F0E0
:10BDF000D3FDB8F10E0FF8D894F80EC00023A7E7D2
:10BE000000FF0F00024B1B6803B118471120704759
:10BE10008801002038B5038804469AB20B80B2F539
:10BE2000706F3ED28278012A3BD8C078FF2838D084
:10BE30002179032901D1237B9BBBA57A637A43EA4D
:10BE40000523E57A43EA0543184DAB4229D850BB98
:10BE5000032928D182F0010505F0010572B10921FD
:10BE60002088F5F79FFB78B90B212088F5F79AFB1E
:10BE700078B12946BDE8384015F099BE0DF062FA58
:10BE80000028ECD10C2038BD2946BDE8384015F01B
:10BE900044BE0C212088F5F785FB0028E9D102205B
:10BEA000F1E71220EFE71120EDE700BF00093D00A8
:10BEB00037B5002504460DF106010DF105008DF89A
:10BEC0000550ADF806500DF045FA074B28465A8844
:10BED00022801B78A370BDF80630A4F803309DF8CB
:10BEE0000530637103B030BD341500202DE9F047F3
:10BEF00003788CB00546EF2B04D9122630460CB0DF
:10BF0000BDE8F0874378EF2BF7D88378013B1E2BF1
:10BF1000F3D80279C37843EA0223427943EA024321
:10BF20005D4A03F18073FF3B23F07F439342E4D8E3
:10BF3000C38840F67C42043B9BB29342DDD8037A2F
:10BF4000013B1E2BD9D8B0F8093040F6FE72013BF8
:10BF50009BB29342D1D8B0F80B30013BFA2BCCD82E
:10BF6000467B002EC9D0731E3342C6D100F014FDAB
:10BF7000864301D01126C1E7AB7B012BBDD8EB7BFB
:10BF8000022BF7D0B9D82B7C013B062BB5D86B7CA4
:10BF9000013B0E2BB1D8AB7C0F2BAED8EB7C012B29
:10BFA000ABD8002B70D12B7A287CB3FBF0F100FBCF
:10BFB0001133DBB2002BA0D16C7CCAB2A1429CD35E
:10BFC000AB7C01D0002B98D0121B5343DBB2142B57
:10BFD000D0D8EB7B002B5DD140F2E243EA88E978D0
:10BFE0005A432B7941EA03216B7941EA0341B2FBC1
:10BFF000F1F301FB1322002A4CD1B5F80B10B5F870
:10C0000009200A44013A92FBF1F253439BB2984251
:10C01000B0D30121687819F031FA0746002800F002
:10C02000F981C28D4FF6FF739A4240F0F381EB7CA9
:10C03000002B90F83420806814BF3B24232410F098
:10C04000CFFE3B7C009401463A6F384619F062FA05
:10C05000002800F0E181B5F80930B5F80B00019334
:10C06000AB7CC0B22A7C0093297A6B7C1AF05BF817
:10C07000804600283FF47EAF0B2010F060FDAB78C7
:10C0800083420BD90D2639E71BF0D2FC00288AD158
:10C09000252633E70123BAE700FF0F000A2128789D
:10C0A000F5F780FA002840F0B9810A212878F5F7E1
:10C0B0003BFA04460028E5D019F095FF032384F8E5
:10C0C00038302B7884F839300123A97884F83C3053
:10C0D00084F83A1084F83B102B7A84F83E3084F8C8
:10C0E0003D30EB7C003B18BF012384F857302B7C9C
:10C0F00084F85430AB7C84F855306B7C84F856302F
:10C10000B5F80B3084F858302A79EB7843EA0223EB
:10C110006A7943EA02436366A87A6A7A42EA0022AD
:10C12000A4F85A20E87B48B940F2E24CEA880CFBBC
:10C1300002F2B2FBF3FC03FB1C2323B9B0F10008AD
:10C1400018BF4FF0010884F86E80687B13F00BFE77
:10C15000012984F86F0003D9AE7B003E18BF012689
:10C1600084F89C604FF0FF3200264FF0FF33084602
:10C17000A4F8DA60E681C4E9042340F2E242EB88E5
:10C180005343A4F8FC20C4F8F83013F09DFDC4F824
:10C19000A00001F0CBFEA4F8A4006B783146D4F8DF
:10C1A000A00084F8A630267613F066FD3146C4F868
:10C1B0001401B4F8A40019F0B3FF94F85730C4F890
:10C1C000180194F86F1094F8580084F81C31267701
:10C1D000E67603B1043012F043FB04F15C0394F8FB
:10C1E0003A20064694F83E1094F89C00029304F11D
:10C1F0006003CDE90063EB8819F0CAFF94F83E10A4
:10C2000094F83A000096D4E9173219F03CFF94F8FC
:10C210006E2094F83E30A066039294F85520029266
:10C2200094F85620019294F854200092D4F8F82003
:10C23000616E19F060FF2065204619F096FFA4F8A2
:10C240006C0004A801F0E0FA20B942F6AC61392094
:10C25000F4F75AFB04A9204616F0E1FC94F8573095
:10C260006BB304F1400805F1140305F124014246C3
:10C2700053F8040B8B4242F8040BF9D1182108AE95
:10C280000DEB0100F4F7F0FE06AB04F1A8020DF18E
:10C29000300E03CB9446C4F89000C4F89410334693
:10C2A000083203CB734542F8080C42F8041C1E46C2
:10C2B000F5D104F18002614640460BF065F994F82F
:10C2C000573094F83E2094F83A1094F89C0002936A
:10C2D00094F86F300193E36D0093236E19F0E3FE41
:10C2E000D4F8F83000F56179994509D90A21287800
:10C2F000F5F76EF900283FF43DAE42F6EC61A6E793
:10C3000004F1C80A504608F085FB064648B10A21E8
:10C310002878F5F75DF900283FF4F0AD42F6F361B7
:10C3200095E795F8028008F1FF384FFA88F8B8F1E0
:10C33000000F0ADA01224946504608F077FB06460C
:10C34000002859D042F6187181E70B2106A8F5F7AD
:10C35000B3F8064610B942F6FC6178E75FFA88F850
:10C3600019F048FFBDF8183008F10101A6F8F230C5
:10C37000C9B286F8F01094F8573086F8EC302B7874
:10C3800086F8F430D4F8A00013F076FC96F8F0109C
:10C39000C6F8E400B4F8A40019F0C2FEC6F8E8003C
:10C3A00094F86F300022304686F8D830FB7B86F850
:10C3B000D9300023C6E9322394F86E304FF0FF32B3
:10C3C0003377B4F85A30B38194F85830B37394F893
:10C3D0005430F373636E7361D4F8F830B3610023A3
:10C3E00073744FF0FF331BF020F9D4F8983046F8FF
:10C3F000F83FC4F8986096E7D4E93A32293342F11D
:10C400000002C4E90C3294F8573087F830302B78AA
:10C41000FB8573E5422671E545266FE50C266DE543
:10C420000279C37843EA0223427943EA0243224A6B
:10C4300003F18073FF3B23F07F43934230B5044602
:10C440008BB002D912200BB030BD038940F69B722D
:10C45000053B9BB29342F5D8837A1E2BF2D8C28853
:10C4600040F6FE71531E9BB28B42EBD8F72A01D9DE
:10C470001120E8E7C57A15F0F80FF9D100F08CFA31
:10C4800035EA0003F4D1A378013B1E2BDAD8237BD5
:10C49000012BD7D8637B022BEAD0D3D8A37B012B07
:10C4A000D0D801A920460AF063FE0028E0D001A8F8
:10C4B000FFF71CFDC7E700BF00FF0F0008B5052010
:10C4C00000F048FA18F06EFF014B024ADA6508BD29
:10C4D000701000201D94000008B5052000F03AFA05
:10C4E00005F078FF014B024ADA6508BD70100020A4
:10C4F0001D94000008B52B21012001F0D7FC182065
:10C5000000F028FA07F0B6FE034B044A1A60044B09
:10C51000044A1A6008BD00BFB4010020C929010007
:10C52000B0010020D751020008B52B21012001F0F5
:10C53000BDFC182000F00EFA05F058FF034B044A2A
:10C540001A60044B044A1A6008BD00BFB401002001
:10C55000C9290100B0010020D751020008B52B21E4
:10C56000012001F0A3FC192000F0F4F918F0CCFD33
:10C5700002F09AF908F048FD014B024A1A6008BD22
:10C58000B0010020D751020008B52B21012001F095
:10C590008DFC192000F0DEF918F008FF02F084F994
:10C5A00008F032FD014B024A1A6008BDB0010020BC
:10C5B000D751020008B5054A2421054B01201A6015
:10C5C00001F074FCBDE8084005F01CBFF901020051
:10C5D0008801002008B503F083FFF6F7E3FD024869
:10C5E000BDE8084003F066BFE410002008B5FAF784
:10C5F00071FBFAF7C3FAFDF711FD01460248BDE8E9
:10C600000840F8F7EDBE00BFE410002008B503486D
:10C6100008F036F8BDE80840FDF794BAE4100020B1
:10C62000044808B500F5847112F062F9BDE80840CD
:10C6300002F032B9E4100020054808B500F5847115
:10C6400012F056F902F028F9BDE80840FFF7B2BF32
:10C65000E4100020044808B500F5847119F0B6FC18
:10C66000BDE8084008F022B8E4100020054808B5ED
:10C6700000F5847119F0AAFC09F01EFABDE8084023
:10C6800008F0CABCE410002008B516F078F9064896
:10C6900000F58471F5F72AFD022010F065FA0020FC
:10C6A000BDE8084010F060BAE410002008B501228F
:10C6B000064B83F80A2203F01BFF05F02DF8FFF765
:10C6C000E3FFBDE8084001F0E7BA00BFE410002036
:10C6D00010B5064C064904F5037015F09EFD04F5EF
:10C6E00004700449BDE8104015F097BDE410002027
:10C6F000BC010020C401002010B5094C094904F513
:10C70000037015F08AFD04F50470074915F085FDE6
:10C7100004F505700549BDE8104015F07EBD00BF69
:10C72000E4100020540200205C0200204C02002093
:10C73000014B93F80A027047E410002010B5094C31
:10C74000094904F5037015F068FD04F50470074904
:10C7500015F063FD04F505700549BDE8104015F0BE
:10C760005CBD00BFE41000200C0200201402002079
:10C770002402002010B5094C0D2000F0EBF8084908
:10C7800004F5037015F049FD04F50470054915F032
:10C7900044FD2420BDE8104000F0DCB8E410002087
:10C7A0002C0200203402002010B5084C0D2000F0AF
:10C7B000D1F8074904F5037015F02FFD04F5047056
:10C7C0000449BDE8104015F028BD00BFE41000206A
:10C7D0003C0200204402002010B50A4C1D2000F04D
:10C7E000B9F8094904F5037015F017FD04F5047054
:10C7F000064915F012FD04F505700549BDE8104025
:10C8000015F00BBDE4100020FC0100200402002004
:10C810001C02002010B50A4C1C2000F09BF80949AE
:10C8200004F5037015F0F9FC04F50470064915F0E1
:10C83000F4FC04F505700549BDE8104015F0EDBCA9
:10C84000E4100020EC010020F40100201C02002074
:10C8500010B50A4C1E2000F07DF8094904F503705C
:10C8600015F0DBFC04F50470064915F0D6FC04F560
:10C8700005700549BDE8104015F0CFBCE41000205C
:10C88000DC010020E40100201C02002010B50A4C4D
:10C890001F2000F05FF8094904F5037015F0BDFC96
:10C8A00004F50470064915F0B8FC04F50570054957
:10C8B000BDE8104015F0B1BCE4100020CC01002010
:10C8C000D40100201C02002038B5094C0D4601F0AF
:10C8D000B7F9D4F80C02C4F8045115F096FCFDF732
:10C8E000BBF901F03BFB012384F8183238BD00BFCF
:10C8F000E4100020014B93F818027047E410002068
:10C9000010B50D4CD4F8100215F07FFCD4F81402C9
:10C9100015F07BFCFDF748F9202000F029F82F20C6
:10C9200000F026F8262000F023F8292000F020F857
:10C93000002384F8183210BDE4100020014B83F866
:10C9400019027047E4100020014B93F81902704758
:10C95000E4100020C2080549012300F0070003FA93
:10C9600000F08B5C18438854704700BF180000200B
:10C97000C208054900F0070001238340885C20EAD3
:10C9800003008854704700BF18000020014BD3E912
:10C990000001704718000020054B1868C0F3C02242
:10C9A000C0F30020400040EA820040F001007047E0
:10C9B0001800002008B50DF0F5FA0023074A32F8F8
:10C9C0002310814205D302EB83039B78044A137042
:10C9D00008BD01330C2BF2D10023F7E7680B0300ED
:10C9E000FE120020024B1878072828BF0720704746
:10C9F000FE12002010B54468238884F87B11A4F847
:10CA00007C3194F86C00FAF795FE84F87E0194F876
:10CA10006D00FAF78FFE054984F87F0104F5B970BF
:10CA200016F09AFF002384F8243110BD6924020017
:10CA3000406807490388A0F86E3190F8643080F8A8
:10CA4000703190F8653000F26510037316F07EBF08
:10CA5000A12402002DE9F04F0C4685B0054608469A
:10CA600016F0B9FD0646204616F0A9FD8046204680
:10CA700016F0A9FD8346204616F0ABFD6C6807460C
:10CA800094F8873094F886A0242B30D104F18709DC
:10CA9000002E4BD00BF0070B584615F050FD88B315
:10CAA00094F86C3098422DD094F82421012A0CBFC0
:10CAB00094F8262194F868201BEA020F36D0BAF1C8
:10CAC000220F1FD094F865201BEA020F1AD1461ED0
:10CAD000F6B2032E06D8013B5E4ADBB21644032BA6
:10CAE00031790BD940F21F210620F3F70DFFBAF17F
:10CAF000220F40F0AA8004F18609C9E713441B798C
:10CB00008B4213D808F00701084615F018FDC0B392
:10CB100094F86D30834234D094F82431012B0CBF4B
:10CB200094F8273194F8693019422AD194F82431C5
:10CB3000012B15D11E212846FFF75CFFBAF1220F09
:10CB400012D16B68182283F809210A2283F8862003
:10CB500093F8C230002B44D140F2B3217E20C4E7C9
:10CB6000002384F82431E9E70023284689F80030BF
:10CB700017F0F5F81821284605B0BDE8F04F17F07A
:10CB80001AB903AB20465A4600933B4615F01CFDEC
:10CB90006C6880BB94F82431012B29D1B4F8803023
:10CBA00004F5267294F86C10B4F8280115F06CFDA9
:10CBB0000446C0B901462846FFF71CFF89F800402B
:10CBC0006B6803F18702914502D1002283F8872028
:10CBD0006B68002403F18702914533D1284617F092
:10CBE000BEF8002032E06B68282283F88620E7E751
:10CBF00084F82401E4E7B4F8800047F6FD73A4F854
:10CC00009872C0430744BFB29F4206D928232846E2
:10CC100084F8A93001F050FEDAE794F887300E2B43
:10CC200002D00B3B012B01D82A23F0E79DF80C30F2
:10CC300084F89A329DF80D3084F89B32262389F8C7
:10CC40000030C5E783F8C240CBE7022005B0BDE85D
:10CC5000F08F00BF980B0300064B002283F8502092
:10CC60004FF6FF72A3F85220A3F85420A3F85620E1
:10CC7000704700BF00130020064BB3F852208242D9
:10CC800001BF002283F850204FF6FF72A3F8522014
:10CC9000704700BF00130020014BA3F854007047F9
:10CCA00000130020094A03464FF6FF71B2F8520004
:10CCB000884206D192F85010012905D001201A604F
:10CCC0007047002018607047002070470013002054
:10CCD000074B93F85020012A1BBF0120B3F85420C2
:10CCE000002083F8500018BFA3F85220704700BFFF
:10CCF00000130020014BA3F85600704700130020DA
:10CD0000074B0246B3F85610B3F85200884205D1DB
:10CD100093F8500018B1012013607047002070474D
:10CD2000001300200A4BB3F85210B3F8562091427A
:10CD300001D0002070474FF6FF72A3F8522093F8FD
:10CD40005020002AF5D00022012083F8502070479F
:10CD500000130020064BB3F85210B3F8562091424E
:10CD600003BF93F85000B0FA80F0400901207047EB
:10CD70000013002050B90A4A0120134603F8010BA2
:10CD80000868C2F801008A889A807047012805D196
:10CD9000034B0A68D8719A608A889A81704700BFED
:10CDA0005813002048B90A4B187880B1D3F80120F5
:10CDB000B3F805300A608B807047012806D1044B18
:10CDC000D87920B19A689B890A60F4E700207047FF
:10CDD0005813002020B9054B187800F00100704767
:10CDE00001280ABF014B0020D879F6E7581300202C
:10CDF000F7B58B8800228DF80600ADF8043008687E
:10CE00000B4B8DF8072001461C7803F5AC73019D90
:10CE1000D0B2844201D8082007E0D3E9007601327D
:10CE20000833AE4208BF8F42F2D103B0F0BD00BF5D
:10CE300068130020084B0146002230B55C7803F5EA
:10CE40008173D0B2844201D8082004E013F8015B5A
:10CE500001328D42F5D130BD68130020F8B52D4C5C
:10CE600063782218013B92F80251DBB2834263706F
:10CE700030D01A010101961C8F1C2644274406F16C
:10CE8000100C56F804EB664547F804EBF9D18232F2
:10CE900082312244214402F1100652F8047BB2424E
:10CEA00041F8047BF9D1E118221891F8026182F867
:10CEB000026106267343704303F5857300F58570A0
:10CEC000E618E35827182350B388BB8091F83A310D
:10CED00082F83A312846FFF7ADFF082818D12378A9
:10CEE000013BDBB29D42237012D02B3305F12B02A4
:10CEF00004EBC30304EBC20293E8030082E80300DF
:10CF00002078FFF797FF08281CBF241884F80251E7
:10CF1000F8BD00BF68130020F0B5254D89B095F825
:10CF2000984105F29911684622460EF0BFFD214650
:10CF3000684615F045FD0446B8B300EB400102A871
:10CF4000C9B2F4F791F8601E95F8A1610124C0B24E
:10CF500095F8982105E0731CB3FBF2F102FB113345
:10CF6000DEB206F120030DEB030111F8203C002B8B
:10CF7000F1D100EB400201F8204C06EB46032032D1
:10CF80002B446A4412F8187C83F8A27112F8177CBB
:10CF900012F8162C83F8A37183F8A4210138AB1979
:10CFA000C0B283F89941FF28D2D109B0F0BD00BFCB
:10CFB0006813002070B5064688B00C46002A4FD092
:10CFC0002A4A92F8A131D01890F8991121B94FF45A
:10CFD00080712820F3F798FC03EB430101331144DF
:10CFE00091F8A251E57091F8A35191F8A41125711F
:10CFF0006171002180F8991192F89811B3FBF1F05A
:10D0000001FB103382F8A13192F8C23123B91849DB
:10D0100002F5DD7016F09DFC65790D220021684651
:10D0200005F03F0545F0400565711AF002FEE37812
:10D0300004AA69468DF80F30304623798DF80D50DB
:10D040008DF80E3004231AF0E1FC9DF81F30237098
:10D050009DF81E3063709DF81D30A37008B070BD40
:10D0600003216018F4F700F8D6E700BF681300202A
:10D0700019CF0000044B5A78824286BF1B1893F8E0
:10D080004A010020704700BF68130020044B5A7803
:10D09000824286BF1B1893F842010020704700BFF0
:10D0A00068130020064B00224FF461711A8083F848
:10D0B000C32183F8C421A3F8C61183F8C2217047A5
:10D0C00068130020014B83F8C401704768130020E7
:10D0D000014B93F8C40170476813002010B5144643
:10D0E000FFF786FE082803D1012000F0010010BDE3
:10D0F000FFF7A0FE064B5A788242F5D904B12070A2
:10D10000184490F83A31012BEED090F84A01ECE740
:10D11000681300202DE9F047824689461746984655
:10D12000FFF766FE08280546064603D0FFF782FE95
:10D13000082863D1334C6378072B61D8082D18D1A8
:10D140002678731C072E237003D96B212820F3F750
:10D15000DBFB06F12B03D9F80000DAB204EBC303C2
:10D1600044F8320004EBC201B9F804208A8083F845
:10D1700006A0657807F110026B1C290163704B1C37
:10D18000234412F8010DBA4203F8010FF9D181319D
:10D1900008F11003214413F8012D984501F8012FDF
:10D1A000F9D125441021404615F06AFC102185F87C
:10D1B0004201384615F064FC002385F80261667868
:10D1C00085F84A0185F83A3131460F4815F0F8FBE9
:10D1D000054631460D4815F0F3FB012D03D8002814
:10D1E00018BF0135EDB284F898510025284684F81F
:10D1F000A151FFF791FE2846BDE8F0871220FBE71A
:10D200000720F9E768130020AA140020B2140020B8
:10D21000064B10B55878013840B2002800DA10BD2E
:10D22000C4B22046FFF71AFE601EF5E7681300201F
:10D23000014B83F8C301704768130020014B93F83A
:10D24000C301704768130020431E4AF2B7129BB215
:10D2500093429DBF024BA3F8C601012000207047F6
:10D2600068130020014BB3F8C60170476813002013
:10D270000A4B30B55C7884420ED9184490F802010C
:10D280002B3003EBC004A5790D7053F8300010600B
:10D290000120A388938030BD0020FCE768130020A4
:10D2A00070B506460D460BF0C9FA0AF033FA0A4B80
:10D2B00093F8C3415CB1597859B1981C8233324616
:10D2C000002D08BF18460AF0CBF90AF055FA20469F
:10D2D00070BD0C46FBE700BF6813002008B5064B85
:10D2E000024603EB0113012103F182000AF0B8F9B1
:10D2F000BDE808400AF040BA68130020024607481B
:10D3000010B590F8C34124B1417821B102300AF040
:10D31000A7F9204610BD0C46FBE700BF68130020AC
:10D3200008B5084B5A7882420AD91A1892F8422155
:10D3300032B903EB00108230FFF73CFE012008BD3C
:10D340000020FCE76813002008B5084B5A78824299
:10D350000AD91A1892F84A2132B903EB00100230A8
:10D36000FFF728FE012008BD0020FCE7681300201D
:10D370002DE9F74F2F4C9A468046894663788342C1
:10D3800056D9231893F8425185F00105F9B193F865
:10D390004A31E3B945F002070135BAF1000F18D15F
:10D3A000FA070AD5062104EB0810524601FB084192
:10D3B000823001F58571FFF7FDFDBB0734D504EB25
:10D3C0000810524649460230FFF7F4FD2CE02F4684
:10D3D000E3E794F8A1614FF0010B002DE0D0A31911
:10D3E00093F89911019399B90092DAB100F086FD92
:10D3F000019B06EB4601009A4FEA102C83F899B185
:10D40000214481F8A201000C81F8A3C181F8A40194
:10D41000013694F89831013DB6FBF3F103FB116638
:10D42000F6B2DAE747F00407384603B0BDE8F08FFC
:10D430000027F9E768130020F8B50646174C48B3F3
:10D44000617804F5A17015F0BBFA94F8985107467D
:10D4500004F29910294615F0B3FA2D1AEDB2AF4235
:10D460001AD8002506270FE0E21892F8422152B997
:10D4700007FB034104EB0313324601F5857103F109
:10D480008200FFF797FD01356278EBB29A42EBD844
:10D490000120F8BD0546E5E70020FAE76813002003
:10D4A000F0B51B4E89B007460D46737883422CD9E0
:10D4B000331893F8424144BB0D22214668461AF0C6
:10D4C000B8FBEB7806EB071004AA8DF80F3069461D
:10D4D0002B7982308DF80E306B798DF80D30042366
:10D4E0001AF094FA2A789DF81F309A420AD16A7885
:10D4F0009DF81E309A4205D1AC789DF81D00231A84
:10D500005C425C41204609B0F0BD0020FBE700BF53
:10D5100068130020074B5A78824209D91A1892F8EA
:10D5200042212AB9062202FB003000F585707047BF
:10D530000020704768130020064B5A78824281BF52
:10D540001B1893F83A01B0FA80F0400998BF002008
:10D55000704700BF68130020F8B50E460746062145
:10D560001546304615F08CFA044640B10A48294663
:10D57000427800F59D701AF05CFB2046F8BD3146FC
:10D58000384615F039FA08281FBF034B0124C0188C
:10D5900080F83A51F1E700BF6813002030B500244D
:10D5A00042F21075A0F84040B0F844404C43B4FB40
:10D5B000F2F4A0F84440541E05FB0343B3FBF2F31E
:10D5C000A0F84230084BB3FBF2F30133A0F8483027
:10D5D000838F05FB0344436B5943B4FBF2F4B1FB67
:10D5E000F2F28463426330BD005A620270B50446B1
:10D5F0000D4651BB4FF434721AF01BFB012384F823
:10D60000DE5084F88E306FF0360384F8D93004236E
:10D6100084F8DA306FF03B0384F8DB306F2384F852
:10D62000DC306FF03C0384F8DD30062384F8DF3013
:10D630002B2384F8D830FE2384F80E317F2384F81E
:10D640008530202384F81C3270BD012917D10023B6
:10D65000A0F8DC3180F8D3310D4BC2691344114678
:10D66000B3FBF2F3C0F8B03040F6B833A0F8B430F2
:10D67000C38C04F17800BDE87040FFF78FBF02292A
:10D68000E2D1B0F8A632D0F8A022C169F1E700BF1C
:10D690007FC3C90170B504460D4651BB4FF41672E5
:10D6A0001AF0C7FA012384F8DE5084F88E306FF048
:10D6B000360384F8D930042384F8DA306FF03B0362
:10D6C00084F8DB306F2384F8DC306FF03C0384F89F
:10D6D000DD30062384F8DF302B2384F8D830FE2396
:10D6E00084F80E317F2384F88530202384F8E931D3
:10D6F00070BD012912D1C2690C4B11461344B3FB12
:10D70000F2F3C0F8B03040F6B833A0F8B430C38CB0
:10D7100004F17800BDE87040FFF740BF0229E7D16F
:10D72000B0F81232D0F80C22C169F1E77FC3C90109
:10D73000034B80F874101B680BB1008818477047C2
:10D7400064020020074B93F900301844142804DCCD
:10D7500010F17F0F03DB40B27047142070476FF069
:10D760007E00704730150020084B1B785B425BB28F
:10D770001844142804DC10F17F0F03DB40B270471B
:10D78000142070476FF07E00704700BF30150020F6
:10D790007F2307B50DF107008DF807300BF05CF81B
:10D7A0009DF9073068B10A4A5078404240B21844A7
:10D7B000142808DC10F17F0F07DB40B203B05DF8DE
:10D7C00004FB1846FAE71420F8E76FF07E00F5E74F
:10D7D00030150020014B187059707047301500202B
:10D7E000024B00221A705A70704700BF301500209B
:10D7F000014B93F90000704730150020014B93F95D
:10D800000100704730150020054B1B7833B9054BDC
:10D810001A681B790260037101207047002070476D
:10D820003215002020000020054BFF221A70054A07
:10D83000016811600179117100221A70704700BFF0
:10D840003215002020000020064B07B518681B7910
:10D85000009068468DF80430FFF7E6FF03B05DF8EE
:10D8600004FB00BF592603000346407898B1DB78DB
:10D870003C2B05D8084AD35C1B1A584258417047C4
:10D8800003F11602D2B2042A04D8034A134413F84F
:10D89000AD3CF1E701207047A00B03003C2908B51F
:10D8A000C17003D80B4B5B5C437008BD01F11603DC
:10D8B000DBB2042B04D8074B194411F8AD3CF3E755
:10D8C000FF2904D040F259412A20F3F71DF8012323
:10D8D000EAE700BFA00B03002DE9F04385B08946BD
:10D8E0001446984602A915F09DF8054600283DD13A
:10D8F000039E34B9012486F88D40204605B0BDE86A
:10D90000F0837769214638460EF019FF014678B357
:10D91000194B5B88A3422DD301AA38460FF07EF83D
:10D9200096F88D300198002B0CBF4946022115F066
:10D9300020FD01982246414603300EF0B7F82146FB
:10D9400038460EF041FF044618B97D212B20F2F72E
:10D95000DBFF9DF808302BB102A815F0AEFF039B4A
:10D96000A3F8CA51002386F88D30C6E70124C4E726
:10D970000446C2E72C46C0E734150020024B987FCE
:10D98000C04300F00100704734150020034B987F1E
:10D9900080F00200C0F34000704700BF3415002043
:10D9A00083230B70014B1B78CB70704754150020FC
:10D9B0002DE9F743876981460D4638460FF020F878
:10D9C000014618B9FC211020F2F79EFF01AA384643
:10D9D0000FF024F8064610B94FF48071F3E7019B6D
:10D9E000B9F8000003F103081D4B1B687BB9B9F8B7
:10D9F00000300198AB800023EE806B7215F0C1FC03
:10DA000001280ED002280CD04FF48D71DBE732468E
:10DA10004146984704460028E9D1204603B0BDE8B6
:10DA2000F083287238460FF001F8044610B940F22E
:10DA30002311C8E7FB2E02D94FF49671C3E728687B
:10DA400010B940F22D11BEE7324641460EF02EF8D5
:10DA500038460EF01CFF0028DFD140F23111B2E74A
:10DA60006C0200202DE9F34706460D460527DFF836
:10DA70006C81DFF86C912B694BB11B7A1BB97E214D
:10DA80001020F2F741FF2C6994B9002066E06C6821
:10DA9000237A012BF9D0EFF3108372B66A6812680B
:10DAA0006A6003B962B62C61237A0BB9A421E7E757
:10DAB00094F808A05FFA8AFA27720AF1FF330B2B59
:10DAC00077D8DFE803F073061027703D4E3D3D3DEB
:10DAD0003D61636813B94FF4D471D1E731462046F4
:10DAE000984704201EE0636813B940F2B111C7E7FC
:10DAF0003146204698470346ADF80400C0B2C3F350
:10DB00000723012B58D0022B0CD100232B610028B6
:10DB1000B1D023E0636813B940F2B911B0E72046F1
:10DB200098470020EFF3108372B6227A052AD1B20B
:10DB30004AD1002222722A61002BE8D162B6E6E7C0
:10DB4000D9F80030002BECD0524631466068984737
:10DB5000BAF10A0FC5D100232B61042002B0BDE841
:10DB6000F08763680BB9B3218AE70D220024327075
:10DB7000012219885869B270A6F803107271B47145
:10DB80000EF085FE2C61E8E7606810B940F2E11103
:10DB900076E7D8F8003031469847034660B1002355
:10DBA00002202B61DAE74FF4F97169E740F2F511D1
:10DBB00066E74FF4FC7163E784F808A00028CDD134
:10DBC000002B7FF458AF60E711B940F2192157E7F5
:10DBD000002B7FF450AF62B64DE700BF6802002013
:10DBE0007002002070B5144C14260021231D32460B
:10DBF00018461AF01EF803460125257404333246F0
:10DC0000002104F11800C4E901331AF012F884F875
:10DC1000245004F11C03094AC4E906330023E362DB
:10DC2000236384F83430C4F83530C4F8393084F8CC
:10DC30003D30136070BD00BF541500206C02002001
:10DC400010B5084C2378FF2B04D04FF49D711020A1
:10DC5000F2F75AFE0DF042FE2070BDE81040FFF7CB
:10DC6000C1BF00BF2500002010B5034C20780DF087
:10DC700051FEFF23237010BD25000020014B1878B2
:10DC80000DF058BE25000020014B024A1A60704773
:10DC900068020020B1D90000014B024A1A607047A7
:10DCA00068020020B1D9000010B506490446FFF70C
:10DCB000D9FE28B920460449BDE81040FFF7D2BE7E
:10DCC00010BD00BF6C15002058150020014B1860D6
:10DCD000704700BF6C020020134610B5027A22B1D3
:10DCE00040F295211020F2F70FFE0A460146024845
:10DCF000BDE8104015F00ABE58150020044890F801
:10DD000034301BB903492C3015F01DBE704700BFDD
:10DD100054150020FF3802000346064890F83E20C4
:10DD20003AB190F83D2022B9034900F8353B15F08F
:10DD30000ABE704754150020A1D900000A4610B54C
:10DD4000037A23B140F29D211020F2F7DDFD014658
:10DD500007230248BDE8104015F0D8BD6C1500201F
:10DD60001346027A0AB1037270470A460146014817
:10DD700015F0CCBD581500201B234FF01B128384D7
:10DD8000038482618382C260038541B94FF4A47326
:10DD9000094AC3844384C261C382026170474FF45D
:10DDA00029634FF4A472C384438403F12963C282BC
:10DDB000C3610361704700BF48014801034608463C
:10DDC000B3F85820B3F84C10B3F842C08A42F0B40C
:10DDD00093F86D4028BF0A46B3F85060B3F85A1064
:10DDE000033CB3F84870B142E4B2B3F8465028BFE0
:10DDF0003146012CA3F842208BBFB3F84A604FF4A0
:10DE000029660C464FF429649742A3F8464038BF70
:10DE100017468E4238BF0E469445A3F84870A3F8C3
:10DE20004A6026D12C1B18BF0124B3F85420B3F844
:10DE30004E50B3F840609542B3F8441028BF1546E1
:10DE400093F86C20033A012A15D9B3F85220B3F89D
:10DE50005670BA4228BF3A46AE42A3F84050A3F8E3
:10DE6000442002D1914200D144B10549F0BC15F0E3
:10DE700073BD0124D9E74FF42962EDE7F0BC704788
:10DE80006B3902000B8BA2F809001046A2F80B3088
:10DE90004B8BA2F80D308B8BA2F80F30CB8B024945
:10DEA000A2F8113015F052BDCD39020008B50B4A69
:10DEB0000B4B70B1492904D940F291212C20F2F783
:10DEC00023FD012010701A78914238BF1146197055
:10DED00008BD10701B221A70FAE700BF93150020CE
:10DEE00026000020014B1878704700BF93150020D2
:10DEF000014B1878704700BF26000020094AD2E97C
:10DF00000003434083EAB01181EA43214FEAF3431F
:10DF100011605360044B58434FEAF06000EB8000FF
:10DF2000704700BF94150020BB79379E094AD2E99B
:10DF30000003434083EAB01181EA43214FEAF343EF
:10DF400011605360044B58434FEAF06000EB8000CF
:10DF5000704700BF28000020BB79379E10B50A4CDF
:10DF600008210948F3F780F8D4E900231343F7D0D8
:10DF7000064CFFF7DBFF2060FFF7D8FF23686060E7
:10DF80000343F6D010BD00BF2800002094150020E8
:10DF9000A0F10C031046DBB2392B10B50C4696BF2E
:10DFA0000C49FE21C95C15F096FE88B984B1217830
:10DFB000342909D0EB2909D0272908BF262110468A
:10DFC000BDE8104015F087BE3221F8E7EA21F6E7F8
:10DFD00010BD00BFE20B0300174B184A9A60184AA5
:10DFE000DA62184A1A61184A5A61184A9A61184A3C
:10DFF0001A63184A5A62184ADA64184A9A64184A24
:10E000009A63184B184A9A60184A1A62184A5A605A
:10E01000184A1A60184A9A62184ADA62184ADA608C
:10E02000184A9A61184A1A63184A9A64184ADA64B4
:10E03000184A5A62704700BF74020020413E020035
:10E040006B42020035420200F9410200E1E90000A2
:10E0500029ED0000F9EB0000554402007D44020068
:10E060009DEB00007C030020633E0200FF430200A2
:10E07000CF3E0200F33F0200B54302008742020098
:10E08000D74302009743020023450200C344020025
:10E09000B144020019440200174B184A9A60184A0A
:10E0A0005A60184A1A60184A9A62184ADA62184A7C
:10E0B000DA60184A9A61184A1A63184A1A62184AAA
:10E0C000DA64184A9A64184A5A62184B184A9A60D5
:10E0D000184A5A62184ADA62184A1A61184A5A618A
:10E0E000184A9A61184A1A63184A9A64184ADA64F4
:10E0F000184A9A63704700BF84040020413E020022
:10E10000773E0200093F0200AB4202001D430200BD
:10E1100045EA00003343020029ED00009DEB0000BA
:10E12000554402007D440200F9EB00008C050020FC
:10E13000633E02001944020055430200F942020006
:10E1400079430200EDEA000023450200C3440200C7
:10E15000B1440200FF4302000C4B0D4A0D491A6006
:10E160000D4B0E4A1A600E4B0E4A1A600E4B0F4AA8
:10E17000DA670F4AC2F880100E49C3F884100E49BE
:10E18000C3F888100D4BC2F88830704798060020FD
:10E19000F5F40100BDF60100940600208FF70100A0
:10E1A000A006002035F301007C030020A1F6010049
:10E1B0007402002051F80100C9F4010049F4010083
:10E1C0000B4B0C4A0C491A600C4B0D4A1A600D4B54
:10E1D0000D4ADA670D4AC3F884200D4AC2F8801050
:10E1E0000C49C3F888100C4BC2F88830704700BF48
:10E1F0009C060020018E00005DF30100A0060020B7
:10E2000035F3010084040020598B00005D8F00006D
:10E210008C05002049F40100C9F40100054B064AB1
:10E220001A65064A5A65064B064A1A65064A5A6531
:10E23000704700BF74020020AD4002007F40020022
:10E240007C0300206540020053410200044B054A54
:10E250005A65054B054A1A65054A5A65704700BF5D
:10E2600084040020774102008C05002065400200F4
:10E27000A5410200054B064A9A65064ADA65064B37
:10E28000064A9A65064A1A66704700BF7402002063
:10E29000FD260200912802007C03002025250200B3
:10E2A000F3280200054B064A9A65064A1A66064B91
:10E2B000064A9A65064ADA65704700BF8404002062
:10E2C000E927020055CA00008C0500202525020020
:10E2D0005F29020010B5084B084C09485C67986735
:10E2E0000849094B094A59679A67094BC3E91D4018
:10E2F000084BC3E91D1210BD7C0300201765020006
:10E30000316502005F65020074020020A965020009
:10E310008C05002084040020024B034A1367034A43
:10E3200013677047612701007402002084040020F5
:10E33000024B034A1367034A13677047FB3D020011
:10E340007C0300208C0500203A2A73B505460C4654
:10E350003ED83A2A45D8DFE812F049008D009700F0
:10E36000A300BB00A100A100CA00CC00D200A10004
:10E37000A100D700E200CC0044004400E600A10068
:10E38000A1000101010108010F011B01440044002B
:10E390003A01570164016A0170017B017D017F012F
:10E3A00081018C019401C301C501440044009C011A
:10E3B00044004400B501AB01AD01AF01B101B701AB
:10E3C000BB01B901BF01A1004400BD01B301C101FE
:10E3D000EB2A00F08B81FF2A00F08A81EA2A00F004
:10E3E000838140F266415120F2F78EFA416841F292
:10E3F0007070D1F80C32B1F80622A3F57A75854217
:10E400000CD84FF47A70B3FBF0F303F550639BB272
:10E410006420B2FBF0F20120D2B20DE040F2E24003
:10E420006FF45065B3FBF0F39BB25D19062DEFD985
:10E43000B2FBF0F20020D2B22271D1F80822B0B1C2
:10E440006420E3711B0AB2FBF0F292B22372204601
:10E450006271120AA271B1F8103263721B0AA372C0
:10E46000B1F8121202B0BDE8704014F0B2BF40F231
:10E47000E240E6E743682046D3F8F811013102B0E4
:10E48000BDE8704014F0D9BF02784368012A02D178
:10E4900093F8103101E093F81931237102B070BD87
:10E4A0004568204605F5107114F0D6FF05F5127188
:10E4B000204614F0DBFF05F50871204614F0DCFF60
:10E4C000D5F80011204602B0BDE8704014F0E2BF5C
:10E4D0004168204601F5F37114F0E2FF6B682046B5
:10E4E000D3F8041102B0BDE8704014F0DDBF4368FA
:10E4F000CEE7084602B0BDE8704000F0CFBB02B0E6
:10E50000BDE8704000F0DABB0E230B7159234B714C
:10E5100000238B71F323CB7130230B72BEE743686A
:10E5200093F80A31B9E7037846687BB996F8103159
:10E5300063B196F80D11204615F05CF896F80C11B1
:10E54000204602B0BDE8704015F058B896F80B119F
:10E55000204615F04FF896F80A11F1E74168204679
:10E5600002B0BDE8704015F053BC436893F8262113
:10E57000227193F8273109E0436893F82421012A96
:10E58000F4D093F868200A7193F86930637185E7D5
:10E59000456895F8030214F08AF80146204615F004
:10E5A00010F895F80202C31E012B07D895F86C30BD
:10E5B000DA1E012A02D8984218BF002014F077F81A
:10E5C0000146204602B0BDE8704014F0F6BF456831
:10E5D0000023204601218DF8043014F0D6FE2A7C59
:10E5E00001A96B7C2046032A03F01F0308BF002209
:10E5F00043EA82139DF8042002F0200213438DF8B1
:10E60000043014F0CFFE49E7436811211888F2F76F
:10E61000C9FF00F15B01204602B0BDE8704014F074
:10E6200078BF084602B0BDE8704017F064BF0846E6
:10E6300002B0BDE8704017F066BF334B1B68002B7B
:10E640003FF42CAF2946204602B0BDE87040184781
:10E650002E4BF3E72E4BF1E72E4BEFE72E4B1B68CB
:10E66000002B3FF41BAF0246232002B0BDE87040F0
:10E670001847294B1B68002B3FF410AF024624209B
:10E68000F3E7254B1B68002B3FF408AF024625201B
:10E69000EBE7436811211888F2F784FF00F17D024F
:10E6A00000F15B01204602B0BDE8704014F03DBFB0
:10E6B0001A4BC3E71A4BC1E71A4BBFE71A4BBDE72A
:10E6C0001A4BBBE71A4BB9E71A4BB7E71A4BB5E73A
:10E6D0001A4BB3E71A4BB1E71A4BAFE71A4BADE74A
:10E6E0001A4BABE71A4BA9E71A4BA7E71A4BA5E75A
:10E6F0004368204693F88F22D3F8901202B0BDE809
:10E70000704014F052BE00BF980600209C06002006
:10E7100094060020A0060020E4060020A4060020A5
:10E72000A8060020B0060020B4060020C406002081
:10E73000C8060020BC060020B8060020C006002045
:10E74000AC060020CC060020D0060020E006002009
:10E75000DC060020D8060020D40600203C2803D880
:10E76000064B53F82000704700F11603DBB2042B70
:10E7700001D8AD38F4E70020704700BF74020020D4
:10E780003C2803D8064B53F82000704700F11603CD
:10E79000DBB2042B01D8AD38F4E70020704700BF8E
:10E7A000840400203C2803D8064B53F8200070470F
:10E7B00000F11603DBB2042B01D8AD38F4E70020DA
:10E7C000704700BF7C0300203C2803D8064B53F859
:10E7D0002000704700F11603DBB2042B01D8AD38DE
:10E7E000F4E70020704700BF8C05002030F8023CA1
:10E7F000F7B504460E467BB100238DF804308DF842
:10E80000053000209DF8043063F307009DF80530C3
:10E8100063F30F2003B0F0BD1B4B30F8A05C1B6806
:10E820000BB128389847194B1B680BB128469847FD
:10E83000174B1B680BB1284698470A230027A6F8F8
:10E8400003503370B770637A54F8880C73710EF00C
:10E8500030F818B9B1216320F2F756F82846FEF7D0
:10E860000BFA39462846F2F7B3FE02212846F2F7A2
:10E87000AFFE18B9074B1B6803B1984704238DF806
:10E8800004300223BBE700BFEC060020F4060020A2
:10E89000E8060020F0060020014B024A1A6070478B
:10E8A000EC060020CBF40100014B024A1A607047CD
:10E8B000F406002043510200F7B5456804464FF6C0
:10E8C000FF776E690DF102010DF101023046ADF8DE
:10E8D00002700DF095FF01A930460DF0B3FF40B175
:10E8E00001980EF0A1F8616800220272FFF726FA83
:10E8F000E8E7044905F1A00003B0BDE8F04015F0D9
:10E9000025B800BFEDE70000F0B5044685B00D4620
:10E91000FF2600F8C16C10F8C23CF3B1184F3B78E9
:10E920001BB148211F20F1F7EFFF0C21381DF2F732
:10E930009BFB3E70002304F8C13C09232A4602F8E1
:10E94000033BD4F80930C5F80330D4F80D305360D8
:10E95000D4F81130936005B0F0BD01A80C21F2F796
:10E9600083FBA4F52C73039AC3F8042101AB03CBFA
:10E9700044F8CA0C44F8C61C04F8C26CDAE700BFBD
:10E980009C15002010B5054C23782BB90C21201DB7
:10E99000F2F76AFBFF23237010BD00BF9C15002017
:10E9A000024690F8EE31BBB990F8EF3103F0FF0169
:10E9B0000BB100207047094B18780028F9D0197066
:10E9C000D9680433C2F8041103CBC2F8E601C2F8D7
:10E9D000EA11FF2382F8EE31012070479C150020D8
:10E9E00038B54368044693F886201C2A24D10022B7
:10E9F00083F8C72083F8C22083F84A22436893F83B
:10EA0000C81003F5D3701D8869B10C4983F8C8207C
:10EA1000A3F8B05183F8AF2114F095FF636800208C
:10EA200083F8860038BD012283F8AF11A3F8B051F6
:10EA3000034983F8B221EFE70220F3E7E541020042
:10EA4000D7410200426870B592F8873004460D46FF
:10EA50003BB1142B05D0123B0B2B94BF0820012097
:10EA600070BDD2F8143183BB92F8C83013B9204678
:10EA700015F065F96168284601F5EF7114F003FDA2
:10EA80002846666814F009FD6168C6F8000128464A
:10EA90000B8801F2BB2121F8023C14F0E2FC616812
:10EAA000284601F2C32114F0E4FC6368002583F8D2
:10EAB000EE5160680C4900F52C7014F044FF636857
:10EAC0001622284683F88720CAE70C220321204615
:10EAD00015F058F963683222204683F8872015F034
:10EAE0002EF90020BCE700BF09E9000038B54368F3
:10EAF000044693F887201D2A04D04FF4DE711F20AE
:10EB0000F1F702FF002293F8C8101D8803F5D370B7
:10EB100083F8C72069B10B4983F8C820A3F8B05126
:10EB200083F8AF2114F00FFF6368002283F8872079
:10EB300038BD012283F8AF11A3F8B051024983F820
:10EB4000B221EFE7E5410200D74102000B46072260
:10EB500010B503F8032B0446D0F80920C1F80320B0
:10EB6000D0F80D205A60B0F811201A81C27C9A7238
:10EB700010F8483C7BB1084B1B681BB935211C20A1
:10EB8000F1F7C2FEA0F5C072A0F58471683898470D
:10EB9000002304F8483C10BDF806002038B505787D
:10EBA000446825B994F8873023B1012518E0A36F94
:10EBB000DB07FAD44A680E4B896813400D4AC4F843
:10EBC000D830C3F307630A4043F00803C4F8DC20DD
:10EBD00084F8DB3015F0B3F825B9042384F88730C6
:10EBE000284638BDA36F002543F00103A367F7E76C
:10EBF0002FC904F76FDB0006436870B593F88620D1
:10EC0000042A30D14C681A4A8E6822400578194C83
:10EC1000C3F8D820C2F30762344042F00802C3F8B8
:10EC2000DC4083F8DB20002283F8C22083F88620B2
:10EC300015B9426882F82B5193F8882102F0FF043D
:10EC40009AB91A8803F5C07083F88941A3F88A211C
:10EC50004A68C3F88C218A680749C3F8902114F0E8
:10EC600072FE204670BD0124FBE70024F9E700BFD7
:10EC70002FC904F76FDB00064DEB0000406890F8E9
:10EC8000883143B9038800F5C070034943811A23D2
:10EC9000437214F058BE70474DEB000010B50446A7
:10ECA000FDF774FE034A044B02400B406260A36010
:10ECB00010BD00BF2FC904F76FDB000637B50C4647
:10ECC0004568FDF763FE084B084A03400A4095F883
:10ECD000D81000930B4001928DF800306B4603CBA7
:10ECE0006060A16003B030BD2FC904F76FDB000680
:10ECF000DB0410B5144604D5037D13B10023436330
:10ED000010BD436B0133436315F0ECFBD0E90D23D9
:10ED10009A42F5D30023034943632046BDE81040DF
:10ED200014F01ABE47440200F8B5446805460E4682
:10ED3000077894F88630012B08D027B994F88730EB
:10ED400023B1012040E0A36F9A07FAD494F8C930A8
:10ED50009B0719D4304614F0ABFB84F8D300B6F807
:10ED60000530A4F8D430B6F80730A4F8D63094F8BB
:10ED7000C93043F00202D80784F8C92010D51749DA
:10ED800004F1CA0014F0E8FD94F8C930D90712D490
:10ED9000DFB994F8873043B150214020F1F7B4FD3A
:10EDA00094F82A31002BEAD1EEE7012384F887306A
:10EDB000284614F0C4FF94F886300020012B03D1BC
:10EDC00084F8860084F8C200F8BDA36F9A0701D5C5
:10EDD0005521E2E743F00203A367E9E70545020096
:10EDE00070B545680446FEF7D3FC054B014685F82F
:10EDF00085001B681BB12046BDE87040184770BDF8
:10EE000000070020024B1B6803B11847704700BF82
:10EE1000FC060020F0B5204E054600243078147022
:10EE200080B1431E7768DBB2181B01280BDC07EBAF
:10EE3000C40057F834604068884208BFAE4212D11F
:10EE400014700120F0BD18194610C0F3470057F8A0
:10EE500036C007EBC60EAC45DEF804608E412CBF11
:10EE600003460446E0E7B54271EB000002D214709D
:10EE70000020E7E707EBC30057F8334040688842BB
:10EE800008BFAC4201D11370DBE7A542814128BF26
:10EE900001331370ECE700BFBC15002010F007022F
:10EEA00008B503D063214820F1F72EFD18B1034BBC
:10EEB000197258601A70C80008BD00BFBC15002048
:10EEC000014B00221A707047BC150020014B187AC4
:10EED000704700BFBC1500202DE9D34315F04BFB54
:10EEE0000DF1070207460E46FFF794FF98B9114C43
:10EEF0002278237A93420ED0616813466FF0604EF9
:10EF00009DF80700984209D301EBC00301320120AC
:10EF10002270C3E9007602B0BDE8D08303EB0E0097
:10EF2000013B01EBC000DBB2D0E90089C0E90289F6
:10EF3000E6E700BFBC15002037B515F01CFB0DF14E
:10EF40000702FFF767FF0446A0B10C4A9DF80700CF
:10EF500013785568411C013B05EBC101DBB213700E
:10EF60001A1AD2B2D200834238BF002205EBC00089
:10EF700018F047FE204603B030BD00BFBC1500208E
:10EF80000A460648822302F8033B0368C1F80330AF
:10EF90004368536083689360704700BFC5150020C5
:10EFA00016220021014818F044BE00BFC5150020FC
:10EFB00017B402AB03E903001B48437D83B30B4640
:10EFC0009DF8001009BB93F86C10184A52F82120E4
:10EFD0004FF47A7102F2E732B2FBF1F2D3E9701426
:10EFE0006E3144F100045218198844F10004426063
:10EFF00001808460B3F8803002220D490C3020F883
:10F000000A3C03B010BCFEF7ABBE520608D51A8806
:10F010000280D3F840224260D3F844228260E9E7BC
:10F0200003B010BC704700BFC51500201C0C0300C6
:10F0300081EF00000F4B4FF47A72042953F821300E
:10F0400010B503F2E73300F1FF34B3FBF2F34FEAFC
:10F05000C41409D003290AD002290CBF6022F0226F
:10F06000234400FB023010BD4FF4D262F8E740F2B7
:10F07000BE22F5E7300C0300264B1A6810B5D2F813
:10F080000F300362537D117D1B0443EA0123D17CC1
:10F090000B436FF450618362B2F819305918062996
:10F0A0008DBF40F2E241A3F550634FF47A714B43B8
:10F0B0008EBF00214B430121C36180F87610937D00
:10F0C000D9B103EB830303EB83039B000386B2F800
:10F0D0001730D9B164214B43C362B2F81B3083842B
:10F0E000B2F81D30C38492F8243003F01F025B098C
:10F0F00080F89A2080F8C03110BDC3EB431403EBB5
:10F10000840303EB83035B009BB2DFE740F2E24141
:10F11000E1E700BFDC150020042913B517D19B01DE
:10F1200003F53473417990F844400139C9B2032999
:10F130001AD81A480144087DD101CA3103FB0213D1
:10F14000174A934215D940F25B712D200FE0032935
:10F1500003D11B0103F5E773E4E702290BBF0B336F
:10F160000A339B00DB00DDE740F292310620F1F725
:10F17000CBFB1E2204F03F01B3FBF2F31A0A41F06D
:10F180004001DBB242EA4012002061F3070063F362
:10F190000F20D3B263F3174002B010BD300C030050
:10F1A000C3BF030038B5074D044600F16901286864
:10F1B00013F076FE94F868102868BDE8384013F024
:10F1C00084BE00BFDC150020D0F88030F7B50BB14D
:10F1D00001221A604388DB0727D50023056A144EF5
:10F1E00005F10A07CDE9003302238DF80630FF232D
:10F1F00086F820306846F2F70FFAB0B9009CA542B5
:10F20000F8D03B466A7A04F10A01607A13F0BAFB3F
:10F210000028EFD0A37886F82030D4F80330C6F861
:10F220002130044BB4F807209A8003B0F0BD00BF32
:10F23000DC150020FD15002038B5084D044600F10E
:10F24000690106232868002213F05FFF94F8681014
:10F250002868BDE8384013F038BE00BFDC15002038
:10F2600007B513F0A2FC8DF807000548012306221C
:10F270000DF10701006813F048FF03B05DF804FBCF
:10F28000DC15002008B5044B986910B1403016F029
:10F2900028FB00F0010008BDDC15002008B5044B78
:10F2A000D86910B1403016F01CFB00F0010008BD19
:10F2B000DC150020F8B504460E461346807F6588AD
:10F2C000324615F0040118BF04F17701FEF750F83B
:10F2D000C20705460BD50123A07F84F86830FEF7EE
:10F2E00019F90368C4F869308388A4F86D30AB0756
:10F2F0000CD50127084E04F17701306884F8767048
:10F3000013F0DCFD3946306813F0ECFD85F00400A5
:10F31000C0F38000F8BD00BFDC15002010B5044626
:10F32000084694F8D8306BBB2378082904F1DB0237
:10F3300084F8D93016D004F1DA01FDF799FF20B92D
:10F3400040F61A712D20F1F7DFFA94F8DA3043F025
:10F35000020384F8DA3004F1D0000B49BDE8104014
:10F3600014F0F1BA094B1868034613F8031BC1F3F4
:10F37000801184F8DA10D0F80310C4F8DB109B88F1
:10F380009380E8E710BD00BF37460200DC1500207F
:10F3900070B504460E461546FDF7D6FA98B923789F
:10F3A000A4F8C16084F8C030637C84F8BF500BB10E
:10F3B00094F8483004F1B60084F8C3300249BDE83F
:10F3C000704014F0C0BA70BD874A020010B5044600
:10F3D0000E498C3014F0B7FA0D4904F1C40014F052
:10F3E000B2FA94F89520B4F896102046FFF7D0FFB3
:10F3F000084B00221A71084B1B682BB12146206A6A
:10F400000222BDE81040184710BD00BF5549020058
:10F4100021460200DC1500204C07002038B5B0F86A
:10F4200048300446184D0133A0F84830AB7C2BB16E
:10F4300009F004FA08F06EF90023AB7400232B7175
:10F4400094F889302BB101212046BDE838400DF0F9
:10F450002CBF637CB3B1B4F848209A4212D3012187
:10F4600020460DF022FF63882046DB0747BF236A52
:10F47000432243224FF6FF7148BF1988BDE8384048
:10F48000FFF786BF0021DFE7DC15002010B5094C2F
:10F490002379012B02D02379022B05D1A37C1BB148
:10F4A00009F0CCF908F036F9A06ABDE81040FFF782
:10F4B000B5BF00BFDC1500200346074A906A03B9B8
:10F4C00009B9FFF7ABBF1379D26A03F18043126920
:10F4D000033B52F823301847DC15002003292DE99F
:10F4E000F043054685B090467BD090F888300529DA
:10F4F000DBB202D14288D60760D5002B5ED101274E
:10F50000DFF8E89099F81260B6B113F07FFA082896
:10F5100088F8000014D002AA0DF10701FDF7A8FE3B
:10F5200020B940F6A4612D20F1F7EEF902A99DF86B
:10F53000070015F02CF8064698F80030082B08D183
:10F54000D9F8001011F8030BC0F3801015F01FF864
:10F550000646D9F8001005F1700395F86F2011F8F0
:10F56000030BC0F3801013F00DFAD9F80010044615
:10F5700011F8030BC0F3801013F03EFA8146FDF73B
:10F58000DBFF014640B1B9F1080F1BD04846FDF73B
:10F5900071FD80F00101C9B298F80000082815D06B
:10F5A00094B9AB7F1C1A604260416B885A0706D43D
:10F5B00021B996B92B7D93B1BB4210D0002005B084
:10F5C000BDE8F0830021E7E70120EEE714B181F008
:10F5D0000104E4B204F00100E7E73046EFE7012060
:10F5E000EDE743889B07E9D5022789E7DC15002072
:10F5F0002DE9F341444C2379012B07D02379022BC9
:10F6000004D040F638412D20F1F77EF9A26A176A3E
:10F610000FB197F87570A8B90125A37C1BB109F04B
:10F620000DF908F077F8002D6BD0A06A0DF01FFEE1
:10F63000002860D008F078FFE36A9B6802B0BDE85C
:10F64000F0411847216802F1690392F8682011F827
:10F65000096BF00913F096F90028DDD006F00F06CB
:10F660002068052E2CD190F8243003F01F03102BB6
:10F6700026D9D4F8288098F812500DB308230DF13C
:10F680000702314640468DF80730FFF727FF002874
:10F69000C3D098F8E930002BBFD1226808F1EA0105
:10F6A000D31C233253F8040B934241F8040BF9D1D5
:10F6B0001B8808F1E1000B80144914F044F9ACE711
:10F6C000394613F037FC0028A6D02379A06A012B15
:10F6D00005D02379022B02D040F6114193E723791C
:10F6E0003146E26A03F180435269013B52F823300C
:10F6F0009847054691E7A06A02B0BDE8F041FFF7E0
:10F700008DBE02B0BDE8F081DC1500204F4602003E
:10F710002DE9FF4708230DF10702052104468DF866
:10F720000730FFF7DBFE054620B90025284604B068
:10F73000BDE8F087F9F750FF06460028F5D1DFF85D
:10F74000EC80216AD8F8002091F88E30104610F82D
:10F75000037B03EA571303F0010381F88E30D2F8DC
:10F760000330C1F803308388A1F807301346276AB5
:10F7700013F81F1BC1F38011B970D2F81F001B7959
:10F78000029038468DF80C30FFF776FC276A02A904
:10F7900094F913A007F18E0013F041FA40F201131F
:10F7A000A7F86C304FF0FF0987F86E90314607F1EB
:10F7B0003400FEF7E1FA51463846FDF7B9FF216AF9
:10F7C00084F8956020460B889DF80720A4F89630B1
:10F7D0004FF6FF7384F8B390A4F8B43015F0ECF84A
:10F7E000134904F18C0014F0AEF8FDF7ADF860B9E0
:10F7F000236A04F1C4000F491A88A4F8CD2093F8B5
:10F800008E3084F8CF3014F09EF8236A0022204610
:10F810001988FFF7BDFD084B00221B6888F80420FB
:10F82000002B83D02146206A98477FE7DC15002013
:10F8300055490200214602004C070020032973B5F8
:10F84000044604D005292BD0012002B070BD082346
:10F850000DF107028DF80730FFF740FE0028F3D0C6
:10F86000237C23B19DF807102046FFF757FD114D6B
:10F870000622042620462B685A701E70FFF792FC61
:10F8800094F85C20A16D286813F045FB28682E7160
:10F8900008F02CFF2868002116F079FF0020D4E73B
:10F8A000054B1B6823B1984780F00100C0B2CCE73C
:10F8B0001846CAE7DC15002048070020F8B50446C2
:10F8C0000F4619B300F13005284615F0ACFAA0B97F
:10F8D00063881A072ED5284615F0BAFA0646284638
:10F8E00015F0A1FA301AC0B215F0F3FA464A93683F
:10F8F00003442846936015F075FA284615F077FA08
:10F9000008F090FD2179252008F0AAFC3E4D002347
:10F9100094F876202868037043706388103B0D2BA1
:10F9200062D8DFE803F05D61590C61446161616197
:10F93000616161442046BDE8F840FFF76FBD0623D2
:10F940004370202303702046FFF72CFC638823F0CC
:10F9500008039BB2152B05D094F85420216D28681C
:10F9600013F0CAFA286808F0C1FE0021286816F0D2
:10F970000EFF0323217900202B7108F059FD064664
:10F9800007B9E86063881B0704D515F09FFA0644A1
:10F99000C4F820616388103B0D2B30D8DFE803F0FA
:10F9A000322F29292F292F2F2F2F2F2F2F290C23AB
:10F9B00043702123037042B104F1770113F07EFA02
:10F9C0000121286813F08EFABDE704F1700113F0ED
:10F9D00075FA94F86F10F4E7062303704370B2E7EA
:10F9E000022303700623F9E740F21F612D20F0F790
:10F9F0008BFF21790120BDE8F84008F039BF40F6BF
:10FA0000AB41F3E7F8BD00BFDC15002038B54388F3
:10FA10000446102B04D10121BDE83840FFF74EBF4A
:10FA20000B4DAB7C23B107F04DFE402008F0FAFEF1
:10FA3000286808F05BFE608810F0040002D121798C
:10FA400008F016FF002008F0B3FE01232B7138BD2B
:10FA5000DC15002003292DE9F743044605D00529CC
:10FA600000F08A80FFF7DAFC80E008230DF1030242
:10FA70008DF80330FFF732FD00287BD0237C23B1C3
:10FA80009DF803102046FFF749FC0123B4F80280DB
:10FA90003E4E00251F464FEA98123068294662F311
:10FAA000861707224370C8F380180270C57013F0E0
:10FAB00056FB2A463946306813F058FB2046FFF7BC
:10FAC000BBFB306813F0BCFBB4F85C30C0F1FE0542
:10FAD000AB42B4BFDDB2EDB2AB422AD947F010075A
:10FAE00000223068A5F10309394613F03FFB306866
:10FAF00013F031FBA91E5FFA89F9014420464D46F7
:10FB0000C9B214F019FF0422C0F307238DF80400D2
:10FB1000C0F307400DEB02018DF8053003238DF88B
:10FB20000600306813F0F1FA00223946306813F00D
:10FB30001DFBB8F1000F06D094F9132094F844107F
:10FB40006079FFF78DFB2A46A16D306813F042FB08
:10FB5000FF203582617908F083FB07233068337119
:10FB600008F0C4FD0021306816F011FE002003B03B
:10FB7000BDE8F083204675E7054B1B6823B1984725
:10FB800080F00100C0B2F2E71846F0E7DC15002073
:10FB90004407002010B5154CA37C1BB108F04EFEA5
:10FBA00007F0B8FDA06A0DF062FB20B1A06A43889F
:10FBB00003F0180323B9A06ABDE81040FFF72EBC7C
:10FBC0002379012B07D02379022B04D040F63B3157
:10FBD0002D20F0F799FE2379E26A03F18043D26881
:10FBE000013BBDE8104052F823301847DC150020D7
:10FBF0002DE9F04FB0F802B08BB0044616461BF06A
:10FC00000307019108D0012F06D0022F04D040F243
:10FC10004C612D20F0F778FE0BF00703052B08D17F
:10FC2000002E72D04FF000094FF0010A4D4601221C
:10FC300009E0022B5DD1002E67D04FF000094FF094
:10FC4000010A4D464A464FF001081BF0400B04D014
:10FC5000002E00F0FE804FF0010B48EA4202DFF870
:10FC60006C820121072042EACA03002243EA0513FD
:10FC700043EA491949EA8B1B0BF07B030093D8F840
:10FC800000309DF800B05A7018705970002E40F086
:10FC90000381B146DE703946D8F8000013F05FFAF0
:10FCA000D8F800004A469DF8001013F05FFA009B58
:10FCB0009DF80070D80702D52046FFF7BDFAB907B6
:10FCC00010D5019BD8F80000002B00F0F68004F15D
:10FCD00077010623012213F018FA0121D8F8000059
:10FCE00013F000F90023002B00F0F28040F62E0103
:10FCF0008FE7002B47D15EBB0BF02303B4F85420F1
:10FD0000134309D01BF0200913D04FF0000901253F
:10FD10004A46AA46C84698E7FFF7B4FA0028F1D148
:10FD2000FFF7BCFA02460028ECD1B1463546B24690
:10FD300089E794F804800125A8F10308AA46B8F1E0
:10FD4000010F94BF4FF000084FF001084A467CE7CE
:10FD5000FFF798FAA8B9FFF7A1FA1BF0200500F009
:10FD600001096CD194F804804FF0010A2A46A8F1E9
:10FD70000308B8F1010F8CBF4FF000084FF00108E5
:10FD800063E70120E9E7012B17D194F8048056B905
:10FD9000A8F10205B1469A463246D5F1000848EB73
:10FDA00005081D4651E7B8F102084FF000099A46D0
:10FDB00018BF4FF001084D46C8E7062B3FF430AF9F
:10FDC000042B39D126BB0BF02303B4F85420134382
:10FDD00011D022794FF000090125033A012A94BF7E
:10FDE000002201221BF0200F0CBF90464FF00008AC
:10FDF0004FF0010A29E7FFF745FA0028E9D1FFF79C
:10FE00004DFA82460028E4D14FF000094D460EE736
:10FE1000FFF738FA70B9FFF741FA227900F00109CB
:10FE2000033A012A8CBF002201221BF020050CD1CD
:10FE30009046DDE70120F0E740F2EF61E9E60025BA
:10FE40004FF0010A2A46A846FFE600254FF0010AB6
:10FE5000F9E7B4F8541059B194F804B0ABF1030BBE
:10FE6000BBF1010F94BF4FF0000B4FF0010BF4E614
:10FE7000618801F023010029EED10092FFF702FA18
:10FE8000009A0028E8D1FFF709FA009A0028E3D188
:10FE9000002F3FF4E0AEDFE7DA70FFF7FFF950B173
:10FEA000D8F81C3093F8BD30002B0CBF4FF0000980
:10FEB0004FF00A09EFE68146EDE604F170010623F2
:10FEC000012213F022F994F86F1007E7DC150020E7
:10FED0003A0716D5626C05A9D8F80000C2F30B22C8
:10FEE00062F30B0394F84620ADF814301209C3F303
:10FEF000072362F3071303228DF81530022313F052
:10FF000004F9BF0640F1B580D4F85031D8F81C7020
:10FF10000293D4F8543103930FB9D8F81870D7E985
:10FF200018A30193FFF7BAF980B1D8F81C3093F801
:10FF3000BD305BB107F1400015F0FDFD30B93B6FFE
:10FF400013EB0A0A019B43F100030193397C4FF044
:10FF5000000CA34BD8F8142053F821004FF47A7307
:10FF6000DDF808E000F2E730B0FBF3F0D2F16E0309
:10FF700061EB0101B3EB0E03DDF80CE061EB0E0168
:10FF8000C318019841F1000113EB0A0340EB010192
:10FF9000D4F84401B3F5161FA0EB020E9DF815002E
:10FFA00071F100024FEAEE7A00F0BF000ADB6CF359
:10FFB00045108DF81500BDF814306FF30C03ADF843
:10FFC000143026E0B3F5703F71F1000208DB9E4566
:10FFD0007AEB0102EBDA40F020008DF8150007E023
:10FFE0009E456CF345107AEB01028DF81500E2DABC
:10FFF0009DF8152012F0200FBDF8142014BF4FF407
:020000040001F9
:10000000967A4FF01E0AB3FBFAF363F30C02ADF8D5
:1000100014203B6F40F2E242B3FBF2F3ADF816302E
:10002000D7F81730FA7E06939DF81C3062F304036C
:100030008DF81C30FCF7D6FC9DF81C3060F347139C
:100040008DF81C309DF815306FF3C7138DF81530FF
:100050003B68CDF81D303B798DF821307B798DF8E8
:100060002230BB798DF82330B7F852300133ADF828
:100070002430012E4FD1B4F85430002B4BD063887C
:10008000980748D4DFF85CA1DAF8000013F063F8B1
:10009000421CB4F854100346D2B2BAF81070C2F140
:1000A000FF00CF1B8742A8BFD743FFB2B94227D971
:1000B0006288D10724D401934A46009B033FD8F8B5
:1000C0000000012543F01001FFB28B4613F04EF8FB
:1000D000019B2046191D3944C9B214F02DFCC0F310
:1000E00007238DF81000C0F307408DF8113004226B
:1000F0008DF81200032304A9D8F8000013F005F8C6
:100100003A46216DDAF8000013F064F8BAF81030BE
:100110001F44AAF8107065F3041B1BF0200F5FFA50
:100120008BF506D02F481223052205A9006812F08E
:10013000ECFF6A060CD5002E4AD104F13000267976
:1001400014F091FE014694F913203046FFF788F829
:10015000FFF7A4F8002836D0224CE36993F8BD30AD
:100160008BB30721206812F0EFFF092340F2E24130
:10017000037032234370E369D3F890308370E369EE
:10018000D3F890301B0AC370E369B3F8923003715F
:10019000E36993F893304371E36993F8A130837175
:1001A000E369D3F89420B2FBF1F2C2717D22E369D6
:1001B000D3F89830B3FBF1F30372E369D3F89C30C2
:1001C000B3FBF2F343722B0606D540F6930120E50C
:1001D000667994F84410B6E70BB0BDE8F08F00BF25
:1001E000300C0300DC1500202DE9F74F04460F46C4
:1001F00090F8440008F016F96179FF20764D08F078
:100200002FF8002F4CD1286812F048FE94F8048093
:10021000064604F1300014F01BFEB8F1040F30D193
:10022000B60106F53476EB6803EBC013CA3306FB60
:1002300000366388002019076E6142BFAB68F6186C
:100240006E616279696908F05BF963889A072ED05C
:100250007FBB6179012008F00BFB012294F8761036
:100260002046FFF7C5FC286808F040FA00212868FE
:1002700016F08DFA06232B7101236B7103B0BDE8D4
:10028000F08FB8F1030F03D1360106F5E776CAE720
:10029000B8F1020F0BBF0B360A36B600F600C2E704
:1002A00062794FF4A571002016F045FACDE7002FD2
:1002B000D3D066884FF0000A286806F00203C6F320
:1002C00080165146002B4FF007030EBF4FF0010977
:1002D0004FF00009D4F858804FEAC90912BFB4F8AA
:1002E0005C70D4F85080B4F8547049EA861B0370EF
:1002F000012380F803A0D946437012F030FF524624
:100300005946286812F032FF1BF0080F17D0626CB4
:1003100001A9BDF80430C2F30B22286862F30B0375
:1003200094F84620ADF804301209C3F3072362F3B2
:10033000071303228DF80530022312F0E6FE286829
:1003400012F07EFF2B8AC0F1FE06FA1AB242B4BF49
:10035000D6B2F6B233449F422ADD002249F01001A2
:10036000286812F003FF286812F06AFF2E8ABF1B6C
:10037000C0F1FE062868B742B4BFFEB2F6B212F072
:10038000EAFE811920460131C9B214F0D5FA0422DF
:10039000C0F307238DF80400C0F307400DEB020102
:1003A0008DF8053003238DF80600286812F0ADFEA5
:1003B00063885B0606D594F9132094F8441060799D
:1003C000FEF74EFF298A32462868414412F002FFA8
:1003D000288A06442E8246E7DC15002010B5084C1A
:1003E000B0F85C30228A9A4205D00121FFF7FCFE6A
:1003F0000723237110BDBDE81040FFF70FB800BF01
:10040000DC15002038B5438804461E4D13F0020F5A
:100410000FD1DB070DD42A8AB0F854309A4203D1A9
:10042000BDE83840FEF7FABF0121BDE83840FFF7CC
:10043000DBBE0020617908F01BFA6388617913F054
:10044000020F14BF0C20222007F00AFF02232B7199
:10045000AB7C4BB107F036F96379033B012B94BFBA
:100460004520402008F0DEF96379033B012B94BF5F
:100470002820002008F09CF92868BDE8384008F0E2
:1004800035B900BFDC150020094810B5037903F029
:10049000FF0453B924222146043017F0CAFB08F0A8
:1004A000CDF907F037F9204610BD0C24FBE700BF5B
:1004B000DC15002010B50023084C23712060FFF7E5
:1004C000E3FF20B140F2EA212D20F0F71DFAE36AA4
:1004D00013B940F2ED21F7E710BD00BFDC15002095
:1004E000014B024ADA627047DC1500202C0700201D
:1004F000044B054A1A60054B054A1A60054B064A2B
:100500001A6070474807002011F700004C070020D0
:10051000FD33000044070020BD0901002DE9F34729
:1005200004460E4600297FD000F13005284614F01D
:100530007AFC28B96388180770D5284614F052FC55
:10054000284614F054FC07F06DFF2179252007F0B0
:1005500087FE384D28680379D90623D5C3789A06D3
:1005600020D012F09BFC074604F1300094F8048080
:1005700014F059FC421C3B464146D2B22046FEF7DD
:10058000CBFD0422C0F307238DF80400C0F307401D
:100590000DEB02018DF8053003238DF80600286865
:1005A00012F0B3FD46B304F1300A2868D5F80C8088
:1005B00012F074FC8146504614F04AFC074650463F
:1005C000013F14F030FC1FFA89F2391A2079C9B2C0
:1005D00014F066FC638880441B0708D5AB680121D2
:1005E0002046984414F0D6FA4044C4F820012279F9
:1005F0004146002007F084FF286808F077F80021C2
:10060000286816F0C4F826B92179304607F010FFA3
:10061000E86005232B7102B0BDE8F087204602B0E8
:10062000BDE8F047FEF7FABE0A4690F87610FFF7ED
:10063000DFFA8EE7DC15002070B5174E0125044661
:100640003030B57114F0EFFBF8B96388DA0604D5E1
:100650002046BDE87040FEF7E1BEB279002AF7D02F
:1006600003F02303B4F85420134305D0204600219F
:10067000BDE87040FFF7B8BDFEF704FE0028F5D1D5
:10068000FEF70CFE0028F1D1E2E729462046BDE83E
:100690007040FFF743BF00BFDC15002070B5114D5F
:1006A0000026012104462E826E7114F073FAAB68A5
:1006B0000344AB60B4F848300133A4F84830FDF788
:1006C0001DFC4FF47F7394F87610B0FBF3F202FB3D
:1006D0001300AB6832461844A8602046BDE870405D
:1006E000FFF786BADC15002010B5094CA06A4388D4
:1006F000092B07D1FFF7D2FFA06A0121BDE8104006
:10070000FFF70CBF0121BDE81040FFF7D7B800BFCD
:10071000DC150020F8B5467D0446B31EDBB2012B84
:100720008CBF0027012796B3023E18BF0126012B7C
:100730002DD800F1700190F86F0012F05DF90546B8
:1007400063889B0605D4082D2CD02846FCF79EFC18
:1007500040BBA577677784F86860FCF783FD0546A2
:1007600017F027F8164B0022A5FB033584F87620F6
:100770001B18204645EB01051146C4E91835FEF764
:1007800099FD70B940F275412D20F0F7BDF80825AC
:10079000D6E704F169013046FCF704FB0028D8D104
:1007A0000020F8BD002EF4D0237F002BF8D0D4F821
:1007B0001630C4F86930638BA4F86D30C9E700BF08
:1007C00040420F002DE9F04F07469BB00C4605460E
:1007D0000EAE0FCF0FC60FCF0FC697E80F0086E8FB
:1007E0000F0006A86E7914F0E3FAA37A61780293F9
:1007F000237801F07F080393237D013BDBB2022BBA
:1008000000F288806C4AC90613441F7E06D4A37D7B
:10081000013BDBB2022B7DD813441E7E637E03F0C6
:10082000FD03012B02D1042F08BF0327A37E03F091
:10083000FD03012B02D1042E08BF0326617A06A80E
:1008400014F0BDFA237D227F06A8022B02F10102DB
:100850000CBF617D0121D2B204BF0131C9B214F0D5
:10086000B0FA18F0080F6CD106A814F0F1FA63780A
:100870008246DA0653D4F0F7DDFF8146394650460A
:10088000FEF7D8FB0123014632464846CDF80080EA
:1008900013F0ECFE40F27121227900F29920E37806
:1008A000B0FBF1F043EA02236279484343EA024392
:1008B0004B43984238D84FF0000B94F818A005939A
:1008C000A37CE86C04930AF1FF33D3F1000A4AEBEE
:1008D000030A0CF085FA8146E86C0CF091FA059B4E
:1008E000484538BF48460DF1180980B260B308A9E1
:1008F000CDF82090ADF824808DF830708DF83160FF
:10090000CDE90A3B13F0E2FF059BE8B945201BB097
:10091000BDE8F08F40F256310620EFF7F5FF2822B0
:10092000414600F01FFAB5E7E379A27942EA0322D3
:10093000237A42EA034201FB02F3984298BF03463E
:10094000B9E700239B46B8E7CDE9103B049B039A27
:100950008DF84C308DF83C700EAF029B8DF83D60E9
:100960002E468DF848A08DF84D308DF83820ADF822
:100970003A800FCF0FC60FCF0FC697E80F0086E85B
:100980000F0099E8030028630020A986E37A13F09A
:10099000FD0F14BF0123002385F86F30E3682B6738
:1009A000238AA5F8743095F84630E27D62F3071388
:1009B00085F84630ABE700BF300C03002DE9FF4758
:1009C00008230DF10702052104468DF80730FEF7D4
:1009D00085FD002800F09280F8F7FEFD002840F029
:1009E0008D80484D206AFEF747FB2B68D3F81F0027
:1009F00093F8232002908DF80C20226AD3F803107C
:100A0000C2F80310B3F80710A2F807101B78206A89
:100A1000C3F3801383703C4B1B6813B10122214642
:100A20009847266A0E2328684FF00808B7780021F7
:100A3000437080F8008012F092FB00224FF0030117
:100A4000286812F093FB2046FEF7F6FB394628682B
:100A500012F048FA06230122F11C286812F055FB17
:100A60006179FF2007F0FCFB286807F03FFE28684B
:100A7000002115F08CFE266A2046314614F036F926
:100A800007460DEB080106F18E0094F913A012F051
:100A9000C6F886F86C7086F86D704FF0FF0986F81E
:100AA0006E90F91E06F1340001298CBF002101214E
:100AB000FDF762F951463046FCF73AFE216A002301
:100AC0009DF80720204684F895300B8884F8B39071
:100AD000A4F896304FF6FF73A4F8B43013F06CFF0F
:100AE000236A1A8885F80480A4F8CD2093F88E3004
:100AF00084F8CF30012004B0BDE8F0872046FEF72F
:100B00008DFCF7E7DC1500204C0700202DE9FF41A4
:100B1000564E0446327902F0FF0312B90278FF2ADA
:100B200004D140F6A2112D20EFF7EEFE3382B36020
:100B30007371B37180F889304D4B684604F130050C
:100B400000934C4B01934C4B0293F36A5B68039305
:100B500007F0B6FD07F0D6FB07F070FE06F0DAFDF1
:100B6000464807F039FC464807F0A4FD284614F033
:100B700039F9284614F03BF907F054FC2179252077
:100B800007F06EFB94F9130007F020FC04F150010C
:100B9000E06C0CF0B4F8074604F15801E06C0CF07E
:100BA000D5F880461FB194F82430002B38D1B8F125
:100BB000000F37D094F82550637F13B963885B0723
:100BC00009D56FF00043D4E918129A4208BFB1F179
:100BD000FF3F29D185BB002F08BF474694F88B30D3
:100BE00003B9AFB1638813F0100511D1606CC0F385
:100BF0000B2014F086F894F8463084F84500C0F3D2
:100C0000032023F00F03184384F8460084F88B5028
:100C100030680330FCF772FBB07404B0BDE8F081BB
:100C20000125C9E74546C7E716F0C3FDD4E91823F7
:100C3000904271EB0303CDD30122204605EA020165
:100C4000FEF738FB68B1FCF70DFB054616F0B1FD69
:100C50000C4BA5FB03351B1845EB0105C4E9183502
:100C6000B9E7002DB7D040F6D7115CE7DC150020BE
:100C700095FB0000F1F50000B9F40000D6BE898EA6
:100C80005555550040420F0037B504461C4DFFF73F
:100C90003DFF04212078F0F785FC0621A86120782B
:100CA000F0F780FCAB69E8612BB120B140F60E2172
:100CB0002D20EFF729FE204613F030FE618811F059
:100CC000100118D000212046FEF7F8FD94F88A3074
:100CD0005BB16846FCF798FD38B1694604F136000F
:100CE00011F09DFF002384F88A30204603B0BDE850
:100CF0003040FEF769BA2046FFF710FCE6E700BF78
:100D0000DC150020024B9862DB6A1B68184700BFA5
:100D1000DC15002043881A0710B504460ED5036A77
:100D20003C220F498C3042721B884381FF2380F89C
:100D300027304FF6FF73038512F005FE63882046C7
:100D4000DB0747BF236A3C223C224FF6FF7148BFB6
:100D50001988FEF71DFBFF2384F8893010BD00BF02
:100D6000554902000138022808B503D9C3212F20B4
:100D7000EFF7CAFD13290A4B05D811290CD8102901
:100D800007D0D121F3E71529FBD103EB4003D88825
:100D900001E033F8100008BD03EB40039889FAE73F
:100DA0004C0C0300F8B52F4B40281A8842EA000289
:100DB0001A8005D104219868BDE8F840F2F78EBA90
:100DC000802801D10521F6E700F00302032A04D1AF
:100DD00040F60E213120EFF797FD10F0020418BF06
:100DE000D960C50705D5CA781961062A0DD00B2A26
:100DF00018D02CB1DA68D278052A1FD00B2A2AD055
:100E0000820644BF08221A75F8BD9A6892F88710C6
:100E10001929EED1002600270121C2E9386782F89E
:100E20008B10E6E79A6892F88710132901BF00211A
:100E300082F88B10012182F8C810DAE79A6892F8DC
:100E400087101729DCD1002400250121C2E93A4589
:100E500082F88C10D4E79A6892F887101229CFD1C3
:100E60000021F5E70C16002013B5044601A8FBF796
:100E700019FF20B940F60C013120EFF745FD502253
:100E80000021019816F0D5FE0321019812F071FAA5
:100E900001982146037823F010030370FCF7FEFC51
:100EA000224601990548FDF74FFAFBF711FF10B9EB
:100EB00040F61601E0E702B010BD00BF101600209A
:100EC00070B5274CA36893F89A6293F89B52002E52
:100ED0003FD193F86C10002D3DD193F86D2083F82D
:100EE0006C1083F86D20FF2283F86E201D4B1B6869
:100EF0000BB1A0689847A36893F82431012B02D066
:100F000056EA050303D000211748FBF773FDA068DC
:100F1000343012F0A7FD0546A06800F24911FCF735
:100F20004DFFA0680621F2F7D9F9A068343012F01D
:100F300099FD8542044610D209F0E4F80146601B91
:100F4000192838BF19200AF00BFAB0FA80F04009CE
:100F500070BD3146BFE72A46C1E70120F8E700BF70
:100F60000C16002070070020101600200A460146CB
:100F7000044808B515F050FB10B9024812F0D6FE2F
:100F8000002008BD1016002008B50C4B9B6893F894
:100F90000E21FE2A04D040F61B013120EFF7B4FCED
:100FA00083F80E0111B9A3F8C41008BD0022A3F8FC
:100FB000BE20012283F8C220F7E700BF0C160020F4
:100FC0000D4A117D99B940B99068B0F85C10B0F83D
:100FD000402091420BD8F2F7F7B813881B0708D5C9
:100FE000936893F88800083818BF012070470020E4
:100FF00070470120704700BF0C16002043689B6FAC
:1010000013F0300F2DE9F74304460D4652D1084640
:1010100012F068FA30B9E978204603B0BDE8F04331
:1010200012F0C9BE2846666812F058FA07462846EC
:10103000343612F04FFA8046284612F051FA8146B3
:10104000284612F049FA4B4642460090394630464F
:1010500012F03DFD184B1A8892070FD5DA68D27846
:10106000142A0BD16268936F43F0100393672046F4
:1010700012F065FE002003B0BDE8F083626892F8CC
:1010800086101E29EED092F81B21002AEAD1626850
:1010900092F81A21002AE5D161688A6F42F0200295
:1010A0008A679A68114602F5A97231F8340BFCF789
:1010B000E9FEDCE70120DEE70C160020154BDB68BB
:1010C00010B51979436893F886200A2A09D193F854
:1010D00009218A4205D1002283F8862083F8C220A4
:1010E00010BD9A6F12F0080406D022F00802BDE885
:1010F00010409A6712F033BEFF2905D1342283F8DD
:101100008C4283F88620EBE740F204513120EFF760
:10111000FBFB00BF0C1600200029134608BF1F214F
:10112000362810B51CD80D281CD9A0F10E02282A8B
:1011300018D8DFE802F019171717191719171F1910
:1011400017171717174217174817173B3B3B52172C
:101150001717171717175A175A175A17175A5A00E7
:10116000EA284BD0002010BD1A460021BDE81040EF
:1011700013F005BF254CA36893F88620222A09D1D5
:10118000201DFBF737FCA368002283F8862083F834
:10119000C220E7E72F2AE5D193F88730A3F1210297
:1011A000062AF0D92F2BEED02A21E9E7184B1B682D
:1011B000002BD7D0BDE810401847164B1B68002BFA
:1011C000D0D01D20F6E7144B1B68002BCAD00A466E
:1011D00012482021BDE810401847114B1B68002B16
:1011E000C0D00E48BDE8104018470E4A1468002CC5
:1011F000B8D00A46014618462346EBE70A4A126869
:10120000002AAFD01846BDE8104010470C16002049
:101210006C070020940700205407002010160020BF
:10122000A407002060070020880700201C4B02460E
:1012300009799B6893F8860022281DD02F281BD09F
:1012400029281BD004281BD010281BD01E281BD0F7
:1012500093F88730242B19D0302819D0352819D08D
:10126000362807D0372817D03B2817D0412814BF7D
:10127000FE203520FFF750BF1620FBE72320F9E7BB
:101280000E20F7E71220F5E71420F3E71720F1E727
:101290002620EFE72E20EDE73020EBE73220E9E7CC
:1012A0000C16002038B50D7904464268362D92F8A8
:1012B00086305DD8222D06D8A5F10E02D0B20F28B7
:1012C00030D9002038BD233D132DFAD801A252F8A1
:1012D00025F000BFD3130100C3120100C3120100A7
:1012E000F3130100C3120100C3120100C312010075
:1012F000C3120100C3120100C3120100C312010096
:101300000B140100C312010039140100C3120100C3
:101310004D140100C3120100C31201006114010049
:10132000231401000F2ACCD801A050F822F000BFEE
:1013300089130100C3120100C3120100C31201008E
:1013400089130100C312010089130100C3120100B7
:101350009713010089130100C3120100C312010099
:10136000C3120100C3120100C3120100E9130100FE
:10137000EA2D45D0FF2DA4D13E4B9B69002BA0D078
:10138000012382F88E329CE7224628460121BDE8DF
:10139000384013F0F4BD222B01D02F2B91D12046E1
:1013A00012F0C4FC636893F88720232A89D093F84D
:1013B000D9201A21204622F0010283F8D920626840
:1013C00092F8D93023F0080382F8D930FBF712FBEA
:1013D00077E7292B7FF475AF274B1B68002B3FF471
:1013E00070AF204698476CE7332B7FF46AAF234BEE
:1013F000F3E7234B1B68002B3FF463AF984760E78C
:10140000204B1B68002BF9D15BE7352B7FF459AFDC
:101410001D4B1B68002B3FF454AF2E2120469847EC
:101420004FE7362B7FF44DAF174A1268002A3FF47E
:1014300048AF1946904744E7372B7FF442AF124B31
:101440001B68002B3FF43DAF3021E7E73B2B7FF4D7
:1014500038AF0D4B1B68002B3FF433AF3221DDE773
:10146000412B7FF42EAF084B1B68002B3FF429AFB4
:101470003521D3E70C1600207407002098070020C0
:101480009C0700208C07002064070020F7B5054664
:10149000934C002840F0E08023881F0752D5A368B2
:1014A00093F80E21222A13D02A2A01D01C2A05D112
:1014B000002283F82C218B4812F038FCA36893F8A3
:1014C0000E21FE2A11D140F276513120EFF71CFA9D
:1014D00083F82E01844B1B68002BECD0A06800F52C
:1014E000977100F58A709847E5E7FE2283F80E2190
:1014F00093F887201B2A08D100267A4883F8C76012
:1015000012F02DFCA36883F88760A36893F8862007
:10151000342A3BD0402A42D0212A0AD193F887208E
:10152000A2F12101062901D92F2A2DD12F2283F8DA
:101530008620A36893F88820082A02BF0222227717
:1015400083F80E212388DE075AD5A368276993F80C
:101550008730123B0B2B0DD8FB78023BDBB2092BFB
:1015600000F2BA80012202FA03F340F2333213424E
:1015700000F0B2803846FCF777F9FE78B0B9314612
:10158000584812F018FC89E02222D0E7012283F8A3
:101590008D22002283F8862083F8C220C9E700222A
:1015A00083F83D214F4812F0C1FBC2E7012E01D95B
:1015B000162E0FD1A36893F8860012F0E9FB48B10C
:1015C000A36893F88620212A04D0222A40D12F2212
:1015D00083F88620112E65D058D8072E64D00D2EA2
:1015E00064D03046FDF7CCF80346002853D1FF2ED7
:1015F0005ED1A369002B5BD0A368012283F88E2201
:101600002388580706D5A26892F88820072A04BFC5
:101610000122227799070FD5E368DE780D2E49D095
:10162000112E49D0072E49D03046FDF7CDF803469C
:10163000002845D02B4898472388DA060CD5A368A4
:1016400093F887200B2A07D10C2283F8872003E028
:10165000162E0CBF20250225237D1B0713D5A3685A
:1016600093F88730123B0B2B38D9002601A90320B1
:101670000196F0F7F1FE019B2BB11E720C22A168BE
:101680000198FCF729FB284603B0F0BD142EA8D121
:10169000164B1B6863B12169124898470028AFD0E8
:1016A0000546D9E7124BF6E7124BF4E7124BF2E787
:1016B000F97865E7114BBDE7114BBBE7114BB9E773
:1016C000FF2E06D1A268342182F88C0282F886109F
:1016D000B2E740F26A51F8E60825BDE70825D2E7EF
:1016E0000C1600201016002058070020900700203C
:1016F0001B500200A51201002D120100ED4E020048
:101700000B4F0200BD100100024B002098611862CF
:10171000704700BF0C16002008B50022044B9A61E8
:101720001A62FCF7B9FCBDE80840FDF72BB900BF11
:101730000C160020024B9869003818BF0120704732
:101740000C1600202DE9F047814C0E4686B0074666
:10175000B4F80080A16818F4007F01F178050CBF8F
:10176000B1F8B820002328460DBF0132A1F8B830E7
:1017700081F8D731A1F8B82013F0DFFB28B1434638
:1017800001F5A0722846FDF7B3FA238803F4C0637D
:1017900043B1A06890F88A30002B00F0AF80032B93
:1017A00000F0B280A168238891F88A20012A04D130
:1017B0001D0544BF022281F88A20002F40F071816C
:1017C000580657BFB1F8F0213A46013292B2A1F85B
:1017D000F02103F00A020A2A0DD1E268D278022A27
:1017E00009D123F0080330462380FFF74FFE06435C
:1017F0000823F6B223803046FFF748FEA36906436C
:10180000F6B2002B5FD01422002101A816F011FAC5
:10181000A36893F86D0007F0BBF9A368054693F839
:101820006D0007F0ADF905F5FA754FF47A71A2680D
:10183000B5FBF1F51388054441F27070ADF8043042
:10184000B2F88030ADF80A50ADF80830D369A3F58E
:101850007A75854295BFB3FBF1F340F2E24103F59F
:101860005063B3FBF1F39BB2ADF8063092F88E32C1
:1018700033B12069C31C049311F079FD8DF8140075
:10188000A26801A89DF80C3092F88D2262F3000343
:101890008DF80C30A3699847A3680022049983F857
:1018A0008E2283F88D2271B193F88C225AB993F865
:1018B0008620342A07D09DF8142022B10878FF280A
:1018C00027D11B2A2CD9A36893F80E21FE2A4FD1C9
:1018D000002E4DD193F88820073A012A48D993F871
:1018E00018312BB3A3680121022093F81921A3F822
:1018F000BC6083F81021FFF747FB39E0012180F835
:101900008A10F1F7EBFC4DE70223012180F88A30C1
:10191000F7E70728D7D1022AD5D14878FF28D2D1B6
:101920000120C3F8901283F88F2283F88C02CAE753
:10193000A06890F88730A3F11105EDB20C2D40F2AC
:101940007881836FDA0705D531460920D3E700BFD8
:101950000C160020990740F1038131460C20FFF757
:1019600013FBA26892F8C93043F0010382F8C93032
:10197000A568B5F8D03195F8D4810133A5F8D031F8
:10198000B8F1000F00F0F382F0F758FD10B100231A
:10199000A5F8D031A368188814F060FEA1688246CB
:1019A00091F88A30B1F83280012B40F2258391F80A
:1019B0008830082B40F0F382B1F8B830022B40F2A7
:1019C0001B83B1F8BA500135ADB2B1F88030DFF801
:1019D00090922B44A1F8C831D9F80030002B00F0C8
:1019E0000F83B8F1010F40F20B83F0F71BFD0246A5
:1019F000A068D9F80090B0F88010C84700F101093C
:101A00001FFA89F9A36893F8D521002A3DD1012D49
:101A10003BD993F887200AB10C2A36D193F8862057
:101A20009ABB93F8882082BB93F88A20022A2CD193
:101A300093F8D7214ABB58690AF03BFF28B3A36843
:101A400093F80E21FE2A20D1B3F8CA21012A1CD90D
:101A5000B3F8D0119A8C914217D2BAF1000F02D08C
:101A6000BAF80E0088B9013D521AADB292B2B5FB78
:101A7000F8F5954228BF154605FB0899003D1FFA69
:101A800089F918BF012583F8D251764B1B6813B131
:101A9000484698478146A368B3F880008144A3F87C
:101AA000CC912288A368550657BFB3F8DC210022E9
:101AB000B3F8CE115218A3F8DC2193F818312BB9E2
:101AC000A36893F88830073B012B07D8A368B3F8C5
:101AD000BC20B3F8CE110A44A3F8BC20A36893F845
:101AE000C20030B1B3F8BE20B3F8CE110A44A3F857
:101AF000BE2093F9C6100029C1BFB3F8C420B3F8C3
:101B0000CE515219A3F8C42093F8A9205AB9002F36
:101B100040F0C082227F022A40F0758293F81021A3
:101B2000062A18BF1622A36893F8A8302BB9A36819
:101B30004D4883F8A920FCF7BFFEA06813F0ABFA6C
:101B40004A4B1B681BB14A4AA06811689847A368B2
:101B5000002283F8D32106B0BDE8F047FBF7E2B8D6
:101B60005A0702D531461320C5E6190706D590F865
:101B70000831314680F810310720BCE61A0602D53C
:101B800000211B20B7E613F030013CD090F81B3148
:101B9000002B40F08582A36893F81A31E3B1A06866
:101BA00090F8873000F58D7100F29A22262B28D00C
:101BB00090F88630A3F1260CDCF1000343EB0C0314
:101BC00011F059FFA268936F23F0200343F0100334
:101BD0009367002382F81A31A068836FDA0640F118
:101BE0005F8200F24911FCF7E9F8A3680021152093
:101BF000B3F85620A3F81021B3F85A20A3F8122105
:101C000079E60123DCE713F0400201D0242072E6DC
:101C100013F4807102D011461E206CE613F400729A
:101C200001D02F2067E65B0540F13A821146312052
:101C300061E6123B0B2B57D8DFE803F006565656E9
:101C4000091C56565656564700210B2053E6FCF702
:101C5000A7FE00283FF48CAE002104204BE600BF15
:101C6000A007002068070020101600205007002061
:101C70003000002090F88832012B08D10021052087
:101C8000FFF782F9A368002283F8882270E6A36830
:101C900093F88832022BD8B27FF46AAEA36806228A
:101CA00093F8C8501DB1002183F81021E8E7AA4835
:101CB000032112F067F8A368294693F8D83013F08F
:101CC000040F14BF11200D20DAE70021062012E6D0
:101CD000002111200FE692F82431012B04D192F853
:101CE0002531002B00F0F181A36893F88620B2B96A
:101CF00093F88720113A0C2A40F2F78193F8B62026
:101D0000002A00F0F28101211220F4E500212D20AB
:101D1000F1E500213320EEE500212020EBE50A2A41
:101D200040F0DF8193F80921012183F8102123E796
:101D3000A36893F82A319BB1A36893F8C93013F0D4
:101D400003050DD101210C20FFF71EF9A36893F8BC
:101D5000C92042F0010283F8C92083F82A5195E78F
:101D6000A36893F81A3153B3A36893F81B3133BBBC
:101D7000A06890F8873000F58D7100F29A22262B2A
:101D80001BD090F88630A3F1260CDCF1000343EB66
:101D90000C0311F070FEA368002283F81A210121C0
:101DA0001420FFF7F1F8A368B3F85620A3F8102128
:101DB000B3F85A20A3F81221DAE50123E9E7A36872
:101DC00093F82421012A74D193F82531002B70D186
